:100000000C946B470C948C470C9447D00C948C4701
:100010000C948C470C948C470C948C470C948C4714
:100020000C948C470C948C470C948C470C9472D293
:100030000C948C470C948C470C947AB40C948C4799
:100040000C948C470C948C470C948C470C948C47E4
:100050000C948C470C948C470C948C470C948C47D4
:100060000C948C470C9461D00C94F0CF0C948C477A
:100070000C94C7C90C9469C90C94A5C90C948C47FD
:100080000C9412D10C948C470C948C470C948C4794
:100090000C948C470C948C470C948C470C948C4794
:1000A0000C948C470C948C470C948C470C9455BB47
:1000B0000C94F9BB0C948C470C948C470C946BB645
:1000C0000C948C470C948C470C948C470C948C4764
:1000D0000C948C470C948C470C948C470C948C4754
:1000E0000C940DA60C948C470C948C470C948C4764
:1000F0000C948C470C948C470C948C470C948C4734
:100100000C942CBB0C94D0BB0C9403BB0C94A7BBDD
:100110000C948C470C948C470C948C470C948C4713
:100120000C948C470C948C470C948C470C948C4703
:100130000C948C470C94CFB50C948C470C948C4742
:100140000C948C470C948C470C948C470C948C47E3
:100150000C948C470C948C470C9403A60C948C47FD
:100160000C948C470C948C470C948C470C948C47C3
:100170000C948C470C948C470C948C470C948C47B3
:100180000C948C470C948C470C948C470C948C47A3
:100190000C948C470C948C470C948C470C948C4793
:1001A0000C947EBB0C9422BC0C948C470C948C4712
:1001B0000C941DB60C948C470C948C470C948C4773
:1001C0000C948C470C948C470C948C470C948C4763
:1001D0000C948C470C948C470C948C470C948C4753
:1001E0000C948C470C948C476F71797183718D716D
:1001F00098719E779E779E779E779E779E719E7769
:100200009E779E779E779E779E77A071AA71B47134
:10021000BE71C8719E779E779E779E779E779E77F8
:10022000D2719E7728729E779E779E779E779E7773
:100230009E779E7767729E7783759E779E779E776F
:100240009E779E779E779E779E7783759E779E7723
:100250009E7794729972A372AD72AF72B972C472C2
:100260009E77CF729E779E770C739E779E779E7750
:100270009E779E779E779E779E779E779E779E77D6
:100280009E779E779E779E7716739E779E779E7752
:100290009E779E779E779E779E779E7720735D737D
:1002A0009A73E373ED730674067410741A742474ED
:1002B0002E7438743D74477451749C779C779C7786
:1002C0009C779C779C779C779C779C779C779C7796
:1002D0009C779C779C779C779C779C779C779C7786
:1002E0009C7710749C779C779C779C779C779C7705
:1002F0009C779C779C779C779C779C779C779C7766
:100300009C779C779C775B7465746F7479749C7729
:100310009C779C779C779C779C779C779C770674DE
:100320002977E876EC76F476D076D476DC76E076CB
:10033000007715771D77217725778177F876F47424
:10034000057516759E779E778E7460719E772775FA
:10035000387549758375F7736B759E779F749E77B3
:100360005A75B07483749E779E779E77C174D274E9
:10037000E3749CBAA4BAACBAB4BABCBAC4BACCBA24
:10038000D4BAB4BD18BD20BD28BD30BD38BD40BDF8
:1003900048BD50BD58BD60BD68BD70BD78BD80BD55
:1003A00098BD98BD98BD98BD98BD98BD98BD98BDA5
:1003B00098BD98BD98BD98BD98BD98BD98BD98BD95
:1003C00098BD98BD98BD98BD98BD98BD98BD98BD85
:1003D00098BD98BD98BD98BD98BD98BD98BD98BD75
:1003E00098BD98BD98BD88BD90BD084AD73B3BCE0F
:1003F000016E84BCBFFDC12F3D6C74319ABD568324
:100400003DDA3D00C77F11BED9E4BB4C3E916BAADB
:10041000AABE000000803F05A84CCDB2D44EB9382A
:1004200036A9020C50B9918688083CA6AAAA2ABE11
:10043000000000803F07634236B79BD8A71A39688F
:100440005618AEBAAB558C1D3CB7CC5763BD6DED9D
:10045000FD753EF6177231BF000000803F080000B6
:1004600000BE922449123EABAAAA2ABECDCCCC4CE7
:100470003E00000080BEABAAAAAA3E00000000BF5A
:10048000000000803F0000000000084178D3BB431B
:1004900087D1133D190E3CC3BD4282AD2B3E68ECA3
:1004A0008276BED98FE1A93E4C80EFFFBE01C4FF2A
:1004B0007F3F0000000000000C94CCBA0C940D5754
:1004C0000C9472AD0C9472A70C945ABA0C94DC760E
:1004D0000C941F570C94D4BA0C942E7A0C94257754
:1004E0000C9476AD0C949A5A0C94037A0C94CA5ED0
:1004F0000C94945B0C9413640C94725A0C942557CE
:100500000C9446800C94A5C80C94765A0C941A74DA
:100510000C942ECD0C949C770C94D2710C94605B4F
:100520000C94155E0C9442BA0C9417C80C942D6868
:100530000C9486630C94A2470C94A5AE0C94AD72F7
:100540000C94D0760C949E770C9442800C9498472F
:100550000C9436570C941CC00C948D710C949A59C1
:100560000C94C4720C94AA5E0C94A65A0C947974E0
:100570000C948E740C949A570C948E470C940674B9
:100580000C9476A70C94B4BA0C94405D0C949A73B6
:100590000C94CEAE0C9400770C94D76E0C945AAD9C
:1005A0000C94F15E0C94675D0C9405750C94926349
:1005B0000C94BE590C948A5A0C9478BD0C944B68D8
:1005C0000C94C5630C94965A0C948A630C94805BCB
:1005D0000C9438750C9413570C9455570C9458BDC3
:1005E0000C94EBAB0C94DCCC0C94E0770C94E9B954
:1005F0000C9430BD0C9433AD0C940C6E0C94E1CD86
:100600000C945EBA0C945B740C94E3730C94D879DC
:100610000C947C5B0C94D55A0C94B9C50C94607105
:100620000C946EAD0C9476570C942D4B0C94925AFE
:100630000C9433580C94B0590C9480BD0C94005712
:100640000C94A25A0C9420BD0C94785B0C943484C6
:100650000C94A9580C94EFAB0C94C0AB0C9441577C
:100660000C9481770C946A5E0C9465540C94195721
:100670000C94C4BA0C941D770C949E710C947971EF
:100680000C94AA5A0C9483740C94E8620C946C5BDE
:100690000C943ABA0C942A5F0C94F9630C9495B9B3
:1006A0000C9466A70C9428720C94F45A0C9460571E
:1006B0000C9498BD0C94B65A0C94E1470C9446AD3A
:1006C0000C946A5A0C940C730C94B4BD0C94095895
:1006D0000C94E9AB0C9456BA0C9445CE0C94387437
:1006E0000C9467720C945E640C9484C80C94157717
:1006F0000C94276E0C94F7730C94C6620C940EB98C
:100700000C94AA710C9450BD0C949C580C94ADB9E7
:100710000C9452A70C94B8670C9452790C94CCBFEB
:100720000C94EB590C943E800C9449750C943163F5
:100730000C94936E0C947E5A0C94556B0C94FE673B
:100740000C9440BD0C94C5590C94EEBC0C94F6B8B6
:100750000C9448BD0C94845B0C94DCCB0C94FEC5CB
:100760000C945C5B0C94CC590C94F2470C9424745C
:100770000C946EA70C94C8710C9410740C946AA716
:100780000C9460BD0C9483750C9451740C9429776F
:100790000C94E05C0C9462BA0C9490CF0C94297980
:1007A0000C94F8760C94E8760C94C2600C94B55DC9
:1007B0000C949C5B0C94495E0C9400800C946959D9
:1007C0000C948A5E0C9400690C94E1C00C946F74D4
:1007D0000C9465CD0C94F0770C94BCBA0C944D6BD2
:1007E0000C94985B0C94DC5D0C9499790C94A4BAED
:1007F0000C94865A0C9465740C943E640C94E076C8
:100800000C945AA70C94AF720C94B9720C945D734B
:100810000C94A0710C94B0740C944AC00C949CBAC3
:100820000C9478680C940A5A0C94A3720C948E5D04
:100830000C9447BA0C9416C90C945E790C94305EF3
:100840000C9416750C9427750C9468BD0C9447A8ED
:100850000C94296D0C9420730C94175E0C94D25751
:100860000C94665A0C943C5D0C94ED730C9478C017
:100870000C94F4BC0C9402B90C946E5A0C94A85BC2
:100880000C947A5A0C94B35B0C94D2740C94CF727F
:100890000C948E630C948E5A0C94D4760C9470BD88
:1008A0000C9406BD0C94195E0C946B750C943D74FD
:1008B0000C94AE5A0C944A570C946B570C94477492
:1008C0000C9490BD0C945A750C945EA70C946F71A7
:1008D0000C94C2AB0C94885B0C9411590C948263F9
:1008E0000C9428BD0C942E790C94EC760C942B5718
:1008F0000C94ACBA0C9470CC0C9494720C94F47666
:100900000C947AAD0C949E5A0C940ABD0C940CBABB
:100910000C9456790C9416730C9485B90C944E79FA
:100920000C948D680C94DF630C945A790C94A64E49
:100930000C94905B0C9469920C94685B0C94175B1C
:100940000C94825A0C9438BD0C9495590C94B25A5C
:100950000C94705B0C9488BD0C948C5B0C94E374C9
:100960000C94F85A0C94DA810C94C1740C94895745
:100970000C9418BD0C9498710C94BE710C94B471C5
:100980000C94C4AB0C9435670C94745B0C94645B4E
:100990000C9462A70C9421770C94D6780C946C5824
:1009A0000C940ACB0C9483710C947E640C94997211
:1009B0000C94B7590C943EBA0C942E740C9404C940
:1009C0000C94F4740C9456A70C949F745B257325B7
:1009D000735D20257320257320706F736974696FB0
:1009E0006E2531382E336625730A005B2573257317
:1009F0005D202573202573206F666673657425322C
:100A0000302E336625730A005B257325735D202520
:100A100073207A65726F206261636B6F6666253141
:100A2000392E336625730A005B257325735D2025F7
:100A300073206C61746368206261636B6F66662506
:100A400031382E336625730A005B257325735D20CC
:100A50002573206C617463682076656C6F636974BC
:100A6000792531332E306625732F6D696E0A005B50
:100A7000257325735D20257320736561726368207B
:100A800076656C6F636974792531322E3066257313
:100A90002F6D696E0A005B257325735D2025732019
:100AA000737769746368206D617825313764205BE2
:100AB000303D6F66662C313D686F6D696E672C3214
:100AC0003D6C696D69742C333D6C696D69742B687C
:100AD0006F6D696E675D0A005B257325735D202568
:100AE0007320737769746368206D696E253137648C
:100AF000205B303D6F66662C313D686F6D696E67B7
:100B00002C323D6C696D69742C333D6C696D697470
:100B10002B686F6D696E675D0A005B257325735DD9
:100B2000202573207261646975732076616C756528
:100B30002532302E346625730A005B257325735DDC
:100B4000202573206A756E6374696F6E2064657604
:100B5000696174696F6E2531342E346625732028DF
:100B60006C61726765722069732066617374657267
:100B7000290A005B257325735D202573206A657241
:100B80006B20686F6D696E672531362E3066257370
:100B90002F6D696E5E33202A2031206D696C6C697F
:100BA0006F6E0A005B257325735D202573206A65CF
:100BB000726B206D6178696D756D2531352E3066EB
:100BC00025732F6D696E5E33202A2031206D696C8C
:100BD0006C696F6E0A005B257325735D2025732099
:100BE00074726176656C206D696E696D756D253105
:100BF000372E336625730A005B257325735D202528
:100C0000732074726176656C206D6178696D756DA5
:100C10002531372E336625730A005B257325735DF6
:100C20002025732076656C6F63697479206D617817
:100C3000696D756D2531312E306625732F6D696EA6
:100C40000A005B257325735D202573206665656446
:100C500072617465206D6178696D756D2531312E15
:100C6000306625732F6D696E0A005B257325735DF1
:100C70002025732061786973206D6F646525313894
:100C8000642025730A005B6D615D20206D696E2014
:100C9000617263207365676D656E742531382E331C
:100CA0006625730A005B736C5D2020736F66742089
:100CB0006C696D697420656E61626C6525313264A2
:100CC0000A005B63745D202063686F7264616C204E
:100CD000746F6C6572616E63652531372E346625DD
:100CE000730A005B6A615D20206A756E6374696FC8
:100CF0006E20616363656C65726174696F6E25381F
:100D00002E306625730A005B6764695D2064656642
:100D100061756C742067636F6465206469737461C6
:100D20006E6365206D6F6465253264205B303D47DE
:100D300039302C313D4739315D0A005B6770615DA8
:100D40002064656661756C742067636F64652070EC
:100D500061746820636F6E74726F6C253364205BFE
:100D6000303D4736312C313D4736312E312C323D26
:100D70004736345D0A005B67636F5D2064656661BA
:100D8000756C742067636F646520636F6F72642095
:100D900073797374656D253364205B312D3620289B
:100DA0004735342D473539295D0A005B67756E5D1F
:100DB0002064656661756C742067636F6465207577
:100DC0006E697473206D6F6465253564205B303DFA
:100DD0004732302C313D4732315D0A005B67706C21
:100DE0005D2064656661756C742067636F6465205F
:100DF000706C616E6525313064205B303D47313762
:100E00002C313D4731382C323D4731395D0A0025C0
:100E10006320776F726B206F66667365743A253155
:100E2000322E336625730A002563206D616368697D
:100E30006E6520706F736E3A2531312E33662573DF
:100E40000A00256320706F736974696F6E3A2531EB
:100E5000352E336625730A00546F6F6C206E756DE6
:100E60006265722020202020202020202025640A76
:100E700000466565642072617465206D6F64653A33
:100E800020202020202025730A0044697374616E9D
:100E90006365206D6F64653A202020202020202586
:100EA000730A0050617468204D6F64653A202020F9
:100EB000202020202020202025730A00506C616E05
:100EC000653A2020202020202020202020202020C3
:100ED0002025730A004D6F74696F6E206D6F646515
:100EE0003A20202020202020202025730A00436F54
:100EF0006F7264696E6174652073797374656D3A9D
:100F000020202025730A00556E6974733A20202032
:100F100020202020202020202020202025730A00AF
:100F2000486F6D696E672073746174653A20202084
:100F3000202020202025730A0046656564686F6CB8
:100F4000642073746174653A20202020202025736A
:100F50000A004D6F74696F6E2073746174653A2076
:100F60002020202020202025730A004379636C650F
:100F70002073746174653A202020202020202020D6
:100F800025730A00526177206D616368696E652080
:100F900073746174653A20202025730A004D6163E3
:100FA00068696E652073746174653A202020202082
:100FB000202025730A004C696E65206E756D626590
:100FC000723A2531306C750A00466565642072619D
:100FD00074653A2531362E336625732F6D696E0A96
:100FE0000056656C6F636974793A2531372E336624
:100FF00025732F6D696E0A004F101E10FE0F4739C2
:1010000035202D20756E6974732D7065722D726593
:10101000766F6C7574696F6E206D6F64650047390B
:1010200034202D20756E6974732D7065722D6D6975
:101030006E757465206D6F64652028692E652E209D
:101040006665656472617465206D6F64652900472B
:101050003933202D20696E76657273652074696D51
:1010600065206D6F6465008B106B10473931202D42
:1010700020696E6372656D656E74616C206469735E
:1010800074616E6365206D6F646500473930202D93
:10109000206162736F6C7574652064697374616E2E
:1010A0006365206D6F646500DC10C410AE104736B8
:1010B00034202D20636F6E74696E756F7573206DAB
:1010C0006F6465004736312E31202D2065786163CD
:1010D000742073746F70206D6F6465004736312023
:1010E0002D2065786163742070617468206D6F6471
:1010F000650016110711F810473139202D20595A73
:1011000020706C616E6500473138202D20585A20C0
:10111000706C616E6500473137202D205859207062
:101120006C616E6500A2119011771156112F114755
:101130003830202D2063616E63656C206D6F74699B
:101140006F6E206D6F646520286E6F6E6520616321
:10115000746976652900473320202D20636F756EF2
:1011600074657220636C6F636B776973652061725D
:1011700063206665656400473220202D20636C6F14
:10118000636B7769736520617263206665656400CF
:10119000473120202D206C696E656172206665657F
:1011A0006400473020202D206C696E6561722074C8
:1011B0007261766572736520287365656B290069B5
:1011C000124F1235121B120112E711CD114735399A
:1011D000202D20636F6F7264696E6174652073796E
:1011E0007374656D203600473538202D20636F6F8E
:1011F0007264696E6174652073797374656D2035EE
:1012000000473537202D20636F6F7264696E6174FB
:10121000652073797374656D203400473536202D51
:1012200020636F6F7264696E617465207379737483
:10123000656D203300473535202D20636F6F726454
:10124000696E6174652073797374656D203200472F
:101250003534202D20636F6F7264696E6174652070
:1012600073797374656D203100473533202D206DFF
:10127000616368696E6520636F6F7264696E617423
:10128000652073797374656D009C1296128F1248F5
:101290006F6D696E6700486F6D6564004E6F7420F6
:1012A000486F6D656400D012CB12C612C012BB121B
:1012B000B212456E6420486F6C6400486F6C640025
:1012C000446563656C00506C616E0053796E630019
:1012D0004F666600E312DF12DA12486F6C64005248
:1012E000756E0053746F70000D130313FD12F61228
:1012F000F2124A6F6700486F6D696E670050726F37
:101300006265004D616368696E696E67004F66666D
:101310000043133D13371332132E1328131F135397
:10132000687574646F776E004379636C6500456E11
:10133000640053746F7000416C61726D005265619E
:10134000647900496E697469616C697A696E6700D5
:10135000A613A0139A13951391138D138813821358
:101360007C1375137113681353687574646F776E0B
:10137000004A6F6700486F6D696E67004379636C60
:10138000650050726F626500486F6C640052756E44
:1013900000456E640053746F7000416C61726D00A3
:1013A000526561647900496E697469616C697A6932
:1013B0006E6700CD13B713473231202D206D696C55
:1013C0006C696D65746572206D6F646500473230BD
:1013D000202D20696E63686573206D6F646500075A
:1013E00014FC13F013E7135B7261646975735D009D
:1013F0005B696E686962697465645D005B737461E2
:101400006E646172645D005B64697361626C6564E3
:101410005D0021141D1418142064656700206D6D93
:101420000020696E002A2A2A204E4F544943452045
:101430002A2A2A20526573657474696E6720626176
:101440007564207261746520746F202573005B627F
:101450006175645D2055534220626175642072613C
:10146000746525313564205B313D393630302C329E
:101470003D31393230302C333D33383430302C3438
:101480003D35373630302C353D3131353230302C2A
:10149000363D3233303430305D0A005B72786D5D3A
:1014A0002073657269616C205258206D6F646525E8
:1014B000313564205B303D636861725F6D6F6465D8
:1014C0002C313D6C696E655F6D6F64655D0A005B14
:1014D00065785D2020656E61626C6520666C6F7753
:1014E00020636F6E74726F6C25313064205B303D09
:1014F0006F66662C313D584F4E2F584F46462C3262
:101500003D5254532F4354535D0A005B65655D2083
:1015100020656E61626C65206563686F2531386493
:10152000205B303D6F66662C313D6F6E5D0A005B5F
:1015300065635D2020657870616E64204C46207480
:101540006F2043524C46206F6E205458253664203D
:101550005B303D6F66662C313D6F6E5D0A00911504
:101560008C15861580157A1573156C153233303449
:1015700030300031313532303000353736303000E0
:101580003338343030003139323030003936303091
:101590000030007379730066620000000017024E8D
:1015A00079DC5D155E763CCD2CDC43737973006687
:1015B000760000000017035279DC5D155E7A3CEC82
:1015C00051783F737973006870000000000700567F
:1015D000798E5D195E7E3C0000803F7379730068F0
:1015E000760000000017005A79DC5D2E797F3C0000
:1015F0000000417379730069640000000004005E1C
:1016000079D678155E723C00000000000000006E84
:1016100000000000000000665A8E5D495EED340057
:10162000000000000000006C696E650000000066AC
:101630005A8957495EED3400000000000000007632
:10164000656C0000001002CC599A57155E723C0080
:10165000000000000000006665656400001002EBF9
:1016600059D257155E723C00000000000000007364
:10167000746174000000006A5A0057155E723C00E5
:10168000000000000000006D616373000000006E48
:101690005A0D57155E723C00000000000000006308
:1016A00079637300000000725A1357155E723C0094
:1016B000000000000000006D6F74730000000076F1
:1016C0005A1957155E723C000000000000000068C7
:1016D0006F6C64000000007A5A1F57155E723C0060
:1016E00000000000000000756E69740000000082B8
:1016F0005A2B57155E723C0000000000000000638A
:101700006F6F7200000000865A3657155E723C00FB
:10171000000000000000006D6F6D6F000000008A87
:101720005A4157155E723C00000000000000007036
:101730006C616E000000008E5A4A57155E723C00C4
:10174000000000000000007061746800000000925A
:101750005A5557155E723C000000000000000064FE
:1017600069737400000000965A6057155E723C0061
:101770000000000000000066726D6F000000009A1B
:101780005A6B57155E723C000000000000000074A8
:101790006F6F6C000000009E5A7657155E723C0019
:1017A0000000006D706F006D706F7800001003A86E
:1017B0005B3358155E723C000000006D706F006D69
:1017C000706F7900001003A85B3358155E723C00FF
:1017D0000000006D706F006D706F7A00001003A83C
:1017E0005B3358155E723C000000006D706F006D39
:1017F000706F6100001003A85B3358155E723C00E7
:101800000000006D706F006D706F6200001003A823
:101810005B3358155E723C000000006D706F006D08
:10182000706F6300001003A85B3358155E723C00B4
:10183000000000706F7300706F7378000010039CDD
:101840005B0958155E723C00000000706F730070F9
:101850006F7379000010039C5B0958155E723C00A1
:10186000000000706F7300706F737A000010039CAB
:101870005B0958155E723C00000000706F730070C9
:101880006F7361000010039C5B0958155E723C0089
:10189000000000706F7300706F7362000010039C93
:1018A0005B0958155E723C00000000706F73007099
:1018B0006F7363000010039C5B0958155E723C0057
:1018C0000000006F6673006F66737800001003B34A
:1018D0005B6C58155E723C000000006F6673006F11
:1018E00066737900001003B35B6C58155E723C00A0
:1018F0000000006F6673006F66737A00001003B318
:101900005B6C58155E723C000000006F6673006FE0
:1019100066736100001003B35B6C58155E723C0087
:101920000000006F6673006F66736200001003B3FF
:101930005B6C58155E723C000000006F6673006FB0
:1019400066736300001003B35B6C58155E723C0055
:10195000000000686F6D00686F6D65000000007E1C
:101960005A25579A59723C00000000686F6D006854
:101970006F6D78000010009C5B405D155EC2340006
:10198000000000686F6D00686F6D79000010009CAA
:101990005B405D155EC33400000000686F6D006839
:1019A0006F6D7A000010009C5B405D155EC43400D2
:1019B000000000686F6D00686F6D61000010009C92
:1019C0005B405D155EC53400000000686F6D006807
:1019D0006F6D62000010009C5B405D155EC63400B8
:1019E000000000686F6D00686F6D63000010009C60
:1019F0005B405D155EC734000000007072620070CD
:101A000072626500000000CCBF405D155EC8340006
:101A1000000000707262007072627800001003CCE7
:101A2000BFDC5D155EC9340000000070726200709A
:101A300072627900001003CCBFDC5D155ECD34000E
:101A4000000000707262007072627A00001003CCB5
:101A5000BFDC5D155ED13400000000707262007062
:101A600072626100001003CCBFDC5D155ED53400EE
:101A7000000000707262007072626200001003CC9D
:101A8000BFDC5D155ED9340000000070726200702A
:101A900072626300001003CCBFDC5D155EDD3400B4
:101AA0000000006A6F67006A6F677800001000CC62
:101AB000BF3C5DB059E734000000006A6F67006A00
:101AC0006F677900001000CCBF3C5DB759E7340068
:101AD0000000006A6F67006A6F677A00001000CC30
:101AE000BF3C5DBE59E734000000006A6F67006AC2
:101AF0006F676100001000CCBF3C5DC559E7340042
:101B00000000007077720070777231000000006290
:101B1000BA95B9155E723C000000007077720070D3
:101B20007772320000000062BA95B9155E723C000F
:101B3000000000707772007077723300000000625E
:101B4000BA95B9155E723C000000007077720070A3
:101B50007772340000000062BA95B9155E723C00DD
:101B600000000031000000316D6100000003003E04
:101B7000BA405D195EF05A000000003100000031EB
:101B80007361000000130342BADC5DF6B8FB5A66CD
:101B900066E63F310000003174720000001B04470C
:101BA000BADC5D02B9FF5A0000204231000000316A
:101BB0006D69000000030056BA405D0EB9F15A008D
:101BC0000000413100000031706F00000003005A36
:101BD000BA405D6A5EF55A0000803F310000003176
:101BE000706D00000003005EBA405D85B9F65A00D2
:101BF00000004032000000326D6100000003003E32
:101C0000BA405D195E0F5B0000803F320000003279
:101C10007361000000130342BADC5DF6B81A5B661C
:101C200066E63F320000003274720000001B044779
:101C3000BADC5D02B91E5B000020423200000032B7
:101C40006D69000000030056BA405D0EB9105B00DC
:101C50000000413200000032706F00000003005AA3
:101C6000BA405D6A5E145B0000803F3200000032C3
:101C7000706D00000003005EBA405D85B9155B0021
:101C800000004033000000336D6100000003003E9F
:101C9000BA405D195E2E5B0000803F3300000033C8
:101CA0007361000000130342BADC5DF6B8395B666D
:101CB00066E63F330000003374720000001B0447E7
:101CC000BADC5D02B93D5B00002042330000003306
:101CD0006D69000000030056BA405D0EB92F5B002D
:101CE0000000413300000033706F00000003005A11
:101CF000BA405D6A5E335B000000003300000033D1
:101D0000706D00000003005EBA405D85B9345B0071
:101D100000004034000000346D6100000003003E0C
:101D2000BA405D195E4D5B00000040340000003495
:101D30007361000000130342BADC5DF6B8585B66BD
:101D400066E63F340000003474720000001B044754
:101D5000BADC5D02B95C5B60760740340000003499
:101D60006D69000000030056BA405D0EB94E5B007D
:101D70000000413400000034706F00000003005A7E
:101D8000BA405D6A5E525B0000803F340000003460
:101D9000706D00000003005EBA405D85B9535B00C2
:101DA0000000407800000078616D0000000300171B
:101DB0005B9C58A9587E330000803F780000007873
:101DC000766D0000001B00605BDC5D3163833300D7
:101DD000007A46780000007866720000001B005C04
:101DE0005BDC5D31637F3300007A46780000007869
:101DF000746E0000001B03685BDC5D31638B330095
:101E00000000007800000078746D0000001B03647F
:101E10005BDC5D316387330000914378000000781C
:101E20006A6D0000001B006C5BDC5D11598F330094
:101E3000409C4578000000786A680000001B007034
:101E40005BDC5D6959933300401C467800000078E4
:101E50006A640000001B04745BDC5D31639B330A21
:101E6000D7233C7800000078736E00000003007CEC
:101E70005B405DF4BCA2320000803F780000007837
:101E800073780000000300805B405DF4BCA3320067
:101E9000000000780000007873760000001B0084CA
:101EA0005BDC5D3163A33300803B45780000007844
:101EB0006C760000001B00885BDC5D3163A733009B
:101EC00000C84278000000786C620000001B038CA0
:101ED0005BDC5D3163AB33000020417800000078AB
:101EE0007A620000001B03905BDC5D3163AF33005E
:101EF0000000407900000079616D000000030017C8
:101F00005B9C58A958B3330000803F7900000079EA
:101F1000766D0000001B00605BDC5D3163B8330050
:101F2000007A46790000007966720000001B005CB0
:101F30005BDC5D3163B43300007A467900000079E0
:101F4000746E0000001B03685BDC5D3163C033000E
:101F50000000007900000079746D0000001B03642C
:101F60005BDC5D3163BC330000A043790000007985
:101F70006A6D0000001B006C5BDC5D1159C433000E
:101F8000409C4579000000796A680000001B0070E1
:101F90005BDC5D6959C83300401C4679000000795C
:101FA0006A640000001B04745BDC5D3163D0330A9B
:101FB000D7233C7900000079736E00000003007C99
:101FC0005B405DF4BCA4320000803F7900000079E2
:101FD00073780000000300805B405DF4BCA5320014
:101FE000000000790000007973760000001B008477
:101FF0005BDC5D3163D83300803B457900000079BC
:102000006C760000001B00885BDC5D3163DC330014
:1020100000C84279000000796C620000001B038C4C
:102020005BDC5D3163E03300002041790000007922
:102030007A620000001B03905BDC5D3163E43300D7
:102040000000407A0000007A616D00000003001774
:102050005B9C58A958E8330000803F7A0000007A62
:10206000766D0000001B00605BDC5D3163ED3300CA
:10207000007A447A0000007A66720000001B005C5F
:102080005BDC5D3163E93300007A447A0000007A5A
:10209000746E0000001B03685BDC5D3163F5330088
:1020A00000F0C27A0000007A746D0000001B036427
:1020B0005BDC5D3163F133000000007A0000007AE0
:1020C0006A6D0000001B006C5BDC5D1159F9330088
:1020D0000048427A0000007A6A680000001B007025
:1020E0005BDC5D6959FD3300007A447A0000007AB8
:1020F0006A640000001B04745BDC5D316305340A14
:10210000D7233C7A0000007A736E00000003007C45
:102110005B405DF4BCA632000000007A0000007A4B
:1021200073780000000300805B405DF4BCA73200C0
:1021300000803F7A0000007A73760000001B008464
:102140005BDC5D31630D3400007A447A0000007A74
:102150006C760000001B00885BDC5D31631134008D
:1021600000C8427A0000007A6C620000001B038CF9
:102170005BDC5D31631534000020417A0000007A99
:102180007A620000001B03905BDC5D316319340050
:102190000040406100000061616D00000003001715
:1021A0005B9C58A9581D340000404061000000614C
:1021B000766D0000001300605BDC5DF15E22340090
:1021C00080CA466100000061667200000013005C76
:1021D0005BDC5DF15E1E3400804A466100000061F8
:1021E000746E0000001303685BDC5D31632A340009
:1021F0000080BF6100000061746D00000013036483
:102200005BDC5DF15E2634000080BF610000006190
:102210006A6D00000013006C5BDC5D11592E340008
:10222000349E4861000000616A680000001300707D
:102230005BDC5D6959323400349E48610000006106
:102240006A640000001304745BDC5DF15E3A34CD17
:10225000CCCC3D610000006172610000001B03787E
:102260005BDC5DF15E3E34DFC3A9406100000061CC
:10227000736E00000003007C5B405DF4BCA832007C
:1022800000803F610000006173780000000300805F
:102290005B405DF4BCA932000000006100000061F9
:1022A00073760000001300845BDC5DF15E42340055
:1022B00000FA4461000000616C76000000130088A1
:1022C0005BDC5DF15E46340000FA446100000061B1
:1022D0006C6200000013038C5BDC5DF15E4A34002D
:1022E00000A04061000000617A62000000130390CA
:1022F0005BDC5DF15E4E3400000040620000006275
:10230000616D0000000300175B9C58A9585234000F
:102310000000006200000062766D000000130060A3
:102320005BDC5DF15E5734000061456200000062D5
:10233000667200000013005C5BDC5DF15E533400EC
:102340000061456200000062746E000000130368C3
:102350005BDC5D31635F34000080BF6200000062BF
:10236000746D0000001303645BDC5DF15E5B3400A0
:102370000080BF62000000626A6D00000013006C04
:102380005BDC5D115963340000A041620000006213
:102390006A640000001300745BDC5DF15E6F340A58
:1023A000D7233C620000006272610000001B0378CA
:1023B0005BDC5DF15E73340000803F63000000630E
:1023C000616D0000000300175B9C58A9588734001A
:1023D0000000006300000063766D000000130060E1
:1023E0005BDC5DF15E8C34000061456300000063DE
:1023F000667200000013005C5BDC5DF15E883400F7
:102400000061456300000063746E00000013036800
:102410005BDC5D31639434000080BF6300000063C7
:10242000746D0000001303645BDC5DF15E903400AA
:102430000080BF63000000636A6D00000013006C41
:102440005BDC5D115998340000A04163000000631B
:102450006A640000001300745BDC5DF15EA4340A62
:10246000D7233C630000006372610000001B037807
:102470005BDC5DF15EA8340000803F7031000070CD
:102480003166727100130052A7DC5DF15ECC590019
:1024900000C84270310000703163736C0013005645
:1024A000A7DC5DF15ED05900007A44703100007005
:1024B000316373680013005AA7DC5DF15ED45900E4
:1024C00000FA4470310000703163706C0013035ED9
:1024D000A7DC5DF15ED8590000003E70310000704D
:1024E0003163706800130362A7DC5DF15EDC59CDD7
:1024F000CC4C3E70310000703177736C0013006675
:10250000A7DC5DF15EE05900007A44703100007094
:10251000317773680013006AA7DC5DF15EE459004F
:1025200000FA4470310000703177706C0013036E54
:10253000A7DC5DF15EE8590000003E7031000070DC
:102540003177706800130372A7DC5DF15EEC59CD42
:10255000CC4C3E703100007031706F660013037612
:10256000A7DC5DF15EF059CDCCCC3D67353400671A
:1025700035347800001B03945BDC5D3163EE320080
:10258000000000673534006735347900001B039480
:102590005BDC5D3163F232000000006735340067B8
:1025A00035347A00001B03945BDC5D3163F6320046
:1025B000000000673534006735346100001B039468
:1025C0005BDC5DF15EFA32000000006735340067C5
:1025D00035346200001B03945BDC5DF15EFE32006B
:1025E000000000673534006735346300001B039436
:1025F0005BDC5DF15E02330000000067353500678B
:1026000035357800001B03945BDC5D3163063300D5
:10261000001143673535006735357900001B039499
:102620005BDC5D31630A33000020436735350067AA
:1026300035357A00001B03945BDC5D31630E33009B
:10264000000000673535006735356100001B0394D5
:102650005BDC5DF15E12330000000067353500671A
:1026600035356200001B03945BDC5DF15E163300C0
:10267000000000673535006735356300001B0394A3
:102680005BDC5DF15E1A33000000006735360067E1
:1026900035367800001B03945BDC5D31631E33002C
:1026A000000000673536006735367900001B03945B
:1026B0005BDC5D3163223300000000673536006764
:1026C00035367A00001B03945BDC5D3163263300F2
:1026D000000000673536006735366100001B039443
:1026E0005BDC5DF15E2A3300000000673536006771
:1026F00035366200001B03945BDC5DF15E2E330017
:10270000000000673536006735366300001B039410
:102710005BDC5DF15E323300000000673537006737
:1027200035377800001B03945BDC5D316336330082
:10273000000000673537006735377900001B0394C8
:102740005BDC5D31633A33000000006735370067BA
:1027500035377A00001B03945BDC5D31633E330048
:10276000000000673537006735376100001B0394B0
:102770005BDC5DF15E4233000000006735370067C7
:1027800035376200001B03945BDC5DF15E4633006D
:10279000000000673537006735376300001B03947E
:1027A0005BDC5DF15E4A330000000067353800678E
:1027B00035387800001B03945BDC5D31634E3300D9
:1027C000000000673538006735387900001B039436
:1027D0005BDC5D3163523300000000673538006711
:1027E00035387A00001B03945BDC5D31635633009F
:1027F000000000673538006735386100001B03941E
:102800005BDC5DF15E5A330000000067353800671D
:1028100035386200001B03945BDC5DF15E5E3300C3
:10282000000000673538006735386300001B0394EB
:102830005BDC5DF15E6233000000006735390067E4
:1028400035397800001B03945BDC5D31636633002F
:10285000000000673539006735397900001B0394A3
:102860005BDC5D31636A3300000000673539006767
:1028700035397A00001B03945BDC5D31636E3300F5
:10288000000000673539006735396100001B03948B
:102890005BDC5DF15E723300000000673539006774
:1028A00035396200001B03945BDC5DF15E7633001A
:1028B000000000673539006735396300001B039459
:1028C0005BDC5DF15E7A330000000067393200673F
:1028D00039327800001103945BDC5D155E5F3500D2
:1028E0000000006739320067393279000011039423
:1028F0005BDC5D155E633500000000673932006700
:1029000039327A00001103945BDC5D155E67350097
:10291000000000673932006739326100001103940A
:102920005BDC5D155E6B35000000006739320067C7
:1029300039326200001103945BDC5D155E6F350077
:1029400000000067393200673932630000110394D8
:102950005BDC5D155E733500000000673238006790
:1029600032387800001103985BDC5D155E77350026
:102970000000006732380067323879000011039890
:102980005BDC5D155E7B3500000000673238006758
:1029900032387A00001103985BDC5D155E7F3500EC
:1029A0000000006732380067323861000011039878
:1029B0005BDC5D155E833500000000673238006720
:1029C00032386200001103985BDC5D155E873500CC
:1029D0000000006732380067323863000011039846
:1029E0005BDC5D155E8B35000000006733300067EF
:1029F00033307800001103985BDC5D155E8F350085
:102A0000000000673330006733307900001103980D
:102A10005BDC5D155E9335000000006733300067B6
:102A200033307A00001103985BDC5D155E9735004A
:102A300000000067333000673330610000110398F5
:102A40005BDC5D155E9B350000000067333000677E
:102A500033306200001103985BDC5D155E9F35002A
:102A600000000067333000673330630000110398C3
:102A70005BDC5D155EA335000000006A6964006AD6
:102A800069646100000000CCBFB55DCA5E923C0085
:102A90000000006A6964006A69646200000000CC9A
:102AA000BFB55DCA5E963C000000006A6964006ABA
:102AB00069646300000000CCBFB55DCA5E9A3C004B
:102AC0000000006A6964006A69646400000000CC68
:102AD000BFB55DCA5E9E3C00000000737973006A5A
:102AE00061000000001F00B65ADC5D3163BC32009B
:102AF00024F449737973006374000000001F04D547
:102B00005ADC5D3163C0320AD7233C73797300739A
:102B10006C000000000700F45A405D195EC43200EA
:102B20000000007379730073740000000007000652
:102B3000BD405DEEBC97320000803F737973006D3D
:102B4000740000000007023ABADC5DADB9EC5A002F
:102B5000000040000000006D650000000000001C47
:102B6000C00CBA0CBA723C00000000000000006DFE
:102B7000640000000000001CC0E9B9E9B9723C0023
:102B800000000073797300656A0000000007003ED2
:102B900080405D6A5E843C0000803F737973006A08
:102BA000760000000007004280405D00805C3F002E
:102BB00000A040737973006A7300000000070046AC
:102BC00080405D6A5E5D3F0000803F7379730074F2
:102BD00076000000000700E1C0405D6A5E5F5C00B7
:102BE00000803F7379730071760000000007007A5F
:102BF000AD405DAA5E255A00000000737973007332
:102C000076000000000700EFAB405D8A5E325A009C
:102C100000803F737973007369000000000700EBC8
:102C2000AB8E5DC4AB335A00007A43737973006591
:102C3000630000000007008263405D7E6474320020
:102C400000000073797300656500000000070086CE
:102C500063405D5E64753200000000737973006547
:102C6000780000000007008A63405D3E6476320011
:102C70000000407379730072786D00000007008EC9
:102C800063405D6A5E77320000803F737973006253
:102C9000617564000004009263405DE86272320076
:102CA00000A040000000007372000000000000E976
:102CB000ABC0ABC2AB723C00000000000000007172
:102CC000720000000000006EAD33AD155E723C0076
:102CD00000000000000000716900000000000072A8
:102CE000AD46AD155E723C000000000000000071B2
:102CF0006F00000000000076AD5AAD155E723C001A
:102D0000000000000000006572000000000000CC20
:102D1000BF47A8155E723C00000000000000007173
:102D200066000000000000CCBF3C5D9559723C007D
:102D30000000000000000072780000000000004A5F
:102D4000C0C662155E723C00000000000000006D0D
:102D5000736700000000001CC03C5D155E723C0003
:102D600000000000000000636C656172000000CC90
:102D7000BFA64EA64E723C0000000000000000748A
:102D800078740000000000CCBF3C5D175E723C0010
:102D90000000000000000074696400000001004AA7
:102DA000C08E5D495EA23C0000000000000000747F
:102DB00065737400000000CCBFD8790ABD723C0076
:102DC000000000000000006465666100000000CCA7
:102DD000BF037AE05C723C0000000000000000626B
:102DE0006F6F7400000000CCBF2E7A2979723C000E
:102DF0000000000000000068656C7000000000CC5E
:102E0000BF9979155E723C00000000000000006868
:102E100000000000000000CCBF9979155E723C00F4
:102E20000000007379730067706C0000000700A257
:102E30005A405D8A5ED232000000007379730067E9
:102E4000756E0000000700A65A405D6A5ED332002E
:102E500000803F7379730067636F0000000700AA6A
:102E60005A405D195ED1320000803F73797300676C
:102E700070610000000700AE5A405D8A5ED43200E7
:102E8000000040737973006764690000000700B2B6
:102E90005A405D6A5ED53200000000000000006705
:102EA00063000000000000CCBFE077F077723C00C8
:102EB000000000000000006D61000000001B04F82D
:102EC0005ADC5D3163C932CDCCCC3D0000000066D8
:102ED000640000000003004AC0405D6A5E5E3F007F
:102EE0000000007564610075646130000003004AF1
:102EF000C0B55DCA5E2E3C000000007564610075BF
:102F0000646131000003004AC0B55DCA5E323C0016
:102F10000000007564610075646132000003004ABE
:102F2000C0B55DCA5E363C00000000756461007586
:102F3000646133000003004AC0B55DCA5E3A3C00DC
:102F40000000007564620075646230000003004A8E
:102F5000C0B55DCA5E3E3C0000000075646200754D
:102F6000646231000003004AC0B55DCA5E423C00A5
:102F70000000007564620075646232000003004A5C
:102F8000C0B55DCA5E463C00000000756462007515
:102F9000646233000003004AC0B55DCA5E4A3C006B
:102FA0000000007564630075646330000003004A2C
:102FB000C0B55DCA5E4E3C000000007564630075DC
:102FC000646331000003004AC0B55DCA5E523C0034
:102FD0000000007564630075646332000003004AFA
:102FE000C0B55DCA5E563C000000007564630075A4
:102FF000646333000003004AC0B55DCA5E5A3C00FA
:103000000000007564640075646430000003004AC9
:10301000C0B55DCA5E5E3C0000000075646400756A
:10302000646431000003004AC0B55DCA5E623C00C2
:103030000000007564640075646432000003004A97
:10304000C0B55DCA5E663C00000000756464007532
:10305000646433000003004AC0B55DCA5E6A3C0088
:103060000000005F7465005F7465780000100278EE
:10307000C0DC5D155E9557000000005F7465005F61
:103080007465790000100278C0DC5D155E99570008
:103090000000005F7465005F74657A0000100278BC
:1030A000C0DC5D155E9D57000000005F7465005F29
:1030B0007465610000100278C0DC5D155EA15700E8
:1030C0000000005F7465005F7465620000100278A4
:1030D000C0DC5D155EA557000000005F7465005FF1
:1030E0007465630000100278C0DC5D155EA95700AE
:1030F0000000005F7472005F747278000010027844
:10310000C0DC5D155EBA58000000005F7472005F9D
:103110007472790000100278C0DC5D155EBE580044
:103120000000005F7472005F74727A000010027811
:10313000C0DC5D155EC258000000005F7472005F65
:103140007472610000100278C0DC5D155EC6580024
:103150000000005F7472005F7472620000100278F9
:10316000C0DC5D155ECA58000000005F7472005F2D
:103170007472630000100278C0DC5D155ECE5800EA
:103180000000005F7473005F7473310000100278F8
:10319000C0DC5D155E2558000000005F7073005FA5
:1031A0007073310000100278C0DC5D155E35580088
:1031B0000000005F6373005F6373310000100278EA
:1031C000C0DC5D155E4558000000005F6573005F60
:1031D0006573310000100278C0DC5D155E55580043
:1031E0000000005F7873005F787331000010027890
:1031F000C0DC5D155E875B000000005F6665005FF8
:103200006665310000100278C0DC5D155E6558000F
:103210000000005F7473005F747332000010027866
:10322000C0DC5D155E2958000000005F7073005F10
:103230007073320000100278C0DC5D155E395800F2
:103240000000005F6373005F637332000010027858
:10325000C0DC5D155E4958000000005F6573005FCB
:103260006573320000100278C0DC5D155E595800AD
:103270000000005F7873005F7873320000100278FE
:10328000C0DC5D155E9F5B000000005F6665005F4F
:103290006665320000100278C0DC5D155E6958007A
:1032A0000000005F7473005F7473330000100278D5
:1032B000C0DC5D155E2D58000000005F7073005F7C
:1032C0007073330000100278C0DC5D155E3D58005D
:1032D0000000005F6373005F6373330000100278C7
:1032E000C0DC5D155E4D58000000005F6573005F37
:1032F0006573330000100278C0DC5D155E5D580018
:103300000000005F7873005F78733300001002786C
:10331000C0DC5D155EB75B000000005F6665005FA6
:103320006665330000100278C0DC5D155E6D5800E4
:103330000000005F7473005F747334000010027843
:10334000C0DC5D155E3158000000005F7073005FE7
:103350007073340000100278C0DC5D155E415800C7
:103360000000005F6373005F637334000010027835
:10337000C0DC5D155E5158000000005F6573005FA2
:103380006573340000100278C0DC5D155E61580082
:103390000000005F7873005F7873340000100278DB
:1033A000C0DC5D155ECF5B000000005F6665005FFE
:1033B0006665340000100278C0DC5D155E7158004F
:1033C000000000000000005F64616D00000000CCA0
:1033D000BF0A5A0A5A723C00000000000000007345
:1033E00065303000000200CCBF675D305E3E5A00A1
:1033F000000000000000007365303100000200CCC6
:10340000BF675D305E405A0000000000000000739E
:1034100065303200000200CCBF675D305E425A006A
:10342000000000000000007365303300000200CC93
:10343000BF675D305E445A0000000000000000736A
:1034400065303400000200CCBF675D305E465A0034
:10345000000000000000007365303500000200CC61
:10346000BF675D305E485A00000000000000007336
:1034700065303600000200CCBF675D305E4A5A00FE
:10348000000000000000007365303700000200CC2F
:10349000BF675D305E4C5A00000000000000007302
:1034A00065303800000200CCBF675D305E4E5A00C8
:1034B000000000000000007365303900000200CCFD
:1034C000BF675D305E505A000000000000000073CE
:1034D00065313000000200CCBF675D305E525A009B
:1034E000000000000000007365313100000200CCD4
:1034F000BF675D305E545A0000000000000000739A
:1035000065313200000200CCBF675D305E565A0064
:10351000000000000000007365313300000200CCA1
:10352000BF675D305E585A00000000000000007365
:1035300065313400000200CCBF675D305E5A5A002E
:10354000000000000000007365313500000200CC6F
:10355000BF675D305E5C5A00000000000000007331
:1035600065313600000200CCBF675D305E5E5A00F8
:10357000000000000000007365313700000200CC3D
:10358000BF675D305E605A000000000000000073FD
:1035900065313800000200CCBF675D305E625A00C2
:1035A000000000000000007365313900000200CC0B
:1035B000BF675D305E645A000000000000000073C9
:1035C00065323000000200CCBF675D305E665A0095
:1035D000000000000000007365323100000200CCE2
:1035E000BF675D305E685A00000000000000007395
:1035F00065323200000200CCBF675D305E6A5A005F
:10360000000000000000007365323300000200CCAF
:10361000BF675D305E6C5A00000000000000007360
:1036200065323400000200CCBF675D305E6E5A0028
:10363000000000000000007365323500000200CC7D
:10364000BF675D305E705A0000000000000000732C
:1036500065323600000200CCBF675D305E725A00F2
:10366000000000000000007365323700000200CC4B
:10367000BF675D305E745A000000000000000073F8
:1036800065323800000200CCBF675D305E765A00BC
:10369000000000000000007365323900000200CC19
:1036A000BF675D305E785A000000000000000073C4
:1036B00079730000000000CCBFC2602A5F723C003A
:1036C000000000000000007031000000000000CC8D
:1036D000BFC2602A5F723C000000000000000031A1
:1036E00000000000000000CCBFC2602A5F723C00F6
:1036F000000000000000003200000000000000CCCC
:10370000BFC2602A5F723C0000000000000000336E
:1037100000000000000000CCBFC2602A5F723C00C5
:10372000000000000000003400000000000000CC99
:10373000BFC2602A5F723C000000000000000078F9
:1037400000000000000000CCBFC2602A5F723C0095
:10375000000000000000007900000000000000CC24
:10376000BFC2602A5F723C00000000000000007AC7
:1037700000000000000000CCBFC2602A5F723C0065
:10378000000000000000006100000000000000CC0C
:10379000BFC2602A5F723C000000000000000062AF
:1037A00000000000000000CCBFC2602A5F723C0035
:1037B000000000000000006300000000000000CCDA
:1037C000BFC2602A5F723C0000000000000000677A
:1037D00035340000000000CCBFC2602A5F723C009C
:1037E000000000000000006735350000000000CC3C
:1037F000BFC2602A5F723C0000000000000000674A
:1038000035360000000000CCBFC2602A5F723C0069
:10381000000000000000006735370000000000CC09
:10382000BFC2602A5F723C00000000000000006719
:1038300035380000000000CCBFC2602A5F723C0037
:10384000000000000000006735390000000000CCD7
:10385000BFC2602A5F723C000000000000000067E9
:1038600039320000000000CCBFC2602A5F723C0009
:10387000000000000000006732380000000000CCAB
:10388000BFC2602A5F723C000000000000000067B9
:1038900033300000000000CCBFC2602A5F723C00E1
:1038A000000000000000006D706F0000000000CC00
:1038B000BFC2602A5F723C00000000000000007080
:1038C0006F730000000000CCBFC2602A5F723C0032
:1038D000000000000000006F66730000000000CCD4
:1038E000BFC2602A5F723C00000000000000006858
:1038F0006F6D0000000000CCBFC2602A5F723C0008
:10390000000000000000007072620000000000CCA7
:10391000BFC2602A5F723C0000000000000000701F
:1039200077720000000000CCBFC2602A5F723C00CA
:10393000000000000000006A6F670000000000CC7B
:10394000BFC2602A5F723C00000000000000006AF5
:1039500069640000000000CCBFC2602A5F723C00B6
:10396000000000000000007564610000000000CC51
:10397000BFC2602A5F723C000000000000000075BA
:1039800064620000000000CCBFC2602A5F723C008D
:10399000000000000000007564630000000000CC1F
:1039A000BFC2602A5F723C0000000000000000758A
:1039B00064640000000000CCBFC2602A5F723C005B
:1039C000000000000000005F74650000000000CCF3
:1039D000BFC2602A5F723C00000000000000005F70
:1039E00074720000000000CCBFC2602A5F723C000D
:1039F000000000000000005F74730000000000CCB5
:103A0000BFC2602A5F723C00000000000000005F3F
:103A100070730000000000CCBFC2602A5F723C00DF
:103A2000000000000000005F63730000000000CC95
:103A3000BFC2602A5F723C00000000000000005F0F
:103A400065730000000000CCBFC2602A5F723C00BA
:103A5000000000000000005F78730000000000CC50
:103A6000BFC2602A5F723C00000000000000005FDF
:103A700066650000000000CCBFC2602A5F723C0097
:103A8000000000000000006D00000000000000CCFD
:103A9000BFF963155E723C00000000000000007179
:103AA00000000000000000CCBFDF63155E723C0028
:103AB000000000000000006F00000000000000CCCB
:103AC000BFC563155E723C000000000000000024CA
:103AD00000000000000000CCBF1364155E723C00C3
:103AE000000000486F6D696E67206572726F72200A
:103AF0002D20256320617869732073657474696E65
:103B00006773206D6973636F6E666967757265644C
:103B10000050726F62696E67206572726F72202D3D
:103B200020256320617869732063616E6E6F742055
:103B30006D6F766520647572696E672070726F6252
:103B4000696E67005B69645D202054696E79472067
:103B50004944253330730A005B68765D2020686134
:103B60007264776172652076657273696F6E253154
:103B7000362E32660A005B68705D202068617264D0
:103B80007761726520706C6174666F726D25313279
:103B9000640A005B66765D20206669726D776172EB
:103BA000652076657273696F6E2531362E32660A2E
:103BB000005B66625D20206669726D7761726520C8
:103BC0006275696C642531382E32660A00456E7460
:103BD00065722024626F6F743D3120746F20656EB2
:103BE0007465722074686520626F6F74206C6F61F9
:103BF0006465722E0A000A0A0A2323232054696E80
:103C0000794720424F4F54204C4F41444552204861
:103C1000656C70202323230A00456E74657220248E
:103C2000646566613D3120746F2072657365742030
:103C30007468652073797374656D20746F2074687F
:103C40006520666163746F72792064656661756C66
:103C5000742076616C7565732E0A546869732077D9
:103C6000696C6C206F766572777269746520616E1D
:103C700079206368616E67657320796F752068616C
:103C80007665206D6164652E0A000A0A0A232323E3
:103C90002054696E794720524553544F5245204471
:103CA000454641554C54532048656C7020232323CE
:103CB0000A00496E766F6B652073656C66207465CB
:103CC000737420627920656E746572696E67202452
:103CD000746573743D4E207768657265204E206967
:103CE00073206F6E65206F663A0A20202474657316
:103CF000743D312020736D6F6B6520746573740A99
:103D0000202024746573743D322020686F6D696EC5
:103D100067207465737420202028796F75206D7575
:103D20007374207472697020686F6D696E67207398
:103D300077697463686573290A2020247465737435
:103D40003D33202073717561726520746573742032
:103D50002020286120736572696573206F66207367
:103D6000717561726573290A202024746573743D2E
:103D70003420206172632074657374202020202019
:103D80002028736F6D65206C6172676520636972AE
:103D9000636C6573290A202024746573743D352093
:103DA000206477656C6C2074657374202020202853
:103DB0006D6F76657320737061636564206279202E
:103DC00031207365636F6E64206477656C6C732952
:103DD0000A202024746573743D362020666565646E
:103DE000686F6C6420746573742028656E746572E6
:103DF000202120616E64207E20746F20686F6C64C7
:103E000020616E6420726573746172742C20726517
:103E100073706563746976656C79290A202024744F
:103E20006573743D3720204D20636F646573207483
:103E30006573742020284D20636F64657320696E5C
:103E40007465726D696E676C65642077697468204B
:103E50006D6F766573290A202024746573743D386C
:103E600020204A534F4E2074657374202020202058
:103E7000286D6F74696F6E20746573742072756E2F
:103E8000207573696E67204A534F4E20636F6D6DC6
:103E9000616E6473290A202024746573743D39208F
:103EA00020696E76657273652074696D652074652E
:103EB00073740A202024746573743D313020726F4E
:103EC00074617279206D6F74696F6E20746573749C
:103ED0000A202024746573743D313120736D616C48
:103EE0006C206D6F76657320746573740A202024CE
:103EF000746573743D313220736C6F77206D6F760B
:103F0000657320746573740A202024746573743D8E
:103F1000313320636F6F7264696E617465207379E9
:103F20007374656D206F6666736574207465737451
:103F300020284739322C204735342D473539290A76
:103F40000A546573747320617373756D6520612005
:103F500063656E7465726564205859206F72696775
:103F6000696E20616E64206174206C6561737420D9
:103F700038306D6D20636C656172616E63652069B8
:103F80006E20616C6C20646972656374696F6E7316
:103F90000A546573747320617373756D65205A20BC
:103FA000686173206174206C656173742034306DB6
:103FB0006D20706F7369697469766520636C6561E3
:103FC00072616E63650A54657374732073746172F1
:103FD0007420776974682061204730205830205958
:103FE00030205A30206D6F76650A486F6D696E67B4
:103FF0002069732074686520657863657074696FE3
:104000006E2E204E6F20696E697469616C20706F2E
:10401000736974696F6E206F7220636C6561726181
:104020006E636520697320617373756D65640A0042
:104030000A0A0A2323232054696E79472053454CEA
:104040004620544553542048656C70202323230A8E
:104050000045616368202420636F6D6D616E64208C
:1040600061626F766520616C736F20646973706C38
:104070006179732074686520746F6B656E20666F5C
:104080007220656163682073657474696E67206966
:104090006E205B205D20627261636B6574730A54ED
:1040A0006F20766965772073657474696E67732015
:1040B000656E746572206120746F6B656E3A0A0AD2
:1040C0002020243C746F6B656E3E0A0A466F722096
:1040D0006578616D706C65202479667220746F203C
:1040E000646973706C6179207468652059206D6112
:1040F00078206665656420726174650A0A546F20D1
:104100007570646174652073657474696E6773207B
:10411000656E74657220746F6B656E206571756174
:104120006C732076616C75653A0A0A2020243C7411
:104130006F6B656E3E3D3C76616C75653E0A0A4666
:104140006F72206578616D706C6520247966723DB0
:1041500038303020746F207365742074686520597E
:10416000206D6178206665656420726174652074D5
:104170006F20383030206D6D2F6D696E7574650A53
:10418000466F7220636F6E66696775726174696FDE
:104190006E2064657461696C73207365653A20688C
:1041A000747470733A2F2F6769746875622E636F29
:1041B0006D2F73796E746865746F732F54696E799F
:1041C000472F77696B692F54696E79472D436F6E5E
:1041D00066696775726174696F6E0A005468657309
:1041E0006520636F6D6D616E64732061726520611F
:1041F000637469766520666F7220636F6E666967A7
:1042000075726174696F6E3A0A2020247379732085
:1042100053686F772073797374656D202867656EB6
:104220006572616C292073657474696E67730A2006
:1042300020243120202053686F77206D6F746F72B7
:1042400020312073657474696E677320286F722043
:104250007768617465766572206D6F746F7220790E
:104260006F752077616E7420312C322C332C3429F9
:104270000A2020247820202053686F77205820615E
:104280007869732073657474696E677320286F7220
:10429000207768617465766572206178697320792A
:1042A0006F752077616E7420782C792C7A2C612CB4
:1042B000622C63290A2020246D20202053686F7708
:1042C00020616C6C206D6F746F72207365747469FB
:1042D0006E67730A2020247120202053686F772096
:1042E000616C6C20617869732073657474696E67A2
:1042F000730A2020246F20202053686F7720616C80
:104300006C206F66667365742073657474696E677C
:10431000730A2020242420202053686F7720616CAA
:104320006C2073657474696E67730A20202468209A
:10433000202053686F7720746869732068656C70FB
:104340002073637265656E0A0A000A0A0A23232332
:104350002054696E794720434F4E46494755524194
:1043600054494F4E2048656C70202323230A000ACD
:10437000466F722064657461696C65642054696E6F
:10438000794720696E666F207365653A206874749A
:1043900070733A2F2F6769746875622E636F6D2F83
:1043A00073796E746865746F732F54696E79472FD3
:1043B00077696B692F0A466F7220746865206C619B
:1043C00074657374206669726D77617265207365B8
:1043D000653A2068747470733A2F2F676974687532
:1043E000622E636F6D2F73796E746865746F732FAF
:1043F00054696E79470A506C65617365206C6F670C
:1044000020616E792069737375657320617420680B
:104410007474703A2F2F7777772E73796E7468657E
:10442000746F732E636F6D2F666F72756D730A48AC
:104430006176652066756E0A000A4E6F74653A20D3
:1044400054696E79472067656E6572617465732083
:104450006175746F6D6174696320737461747573D1
:10446000207265706F727473206279206465666172
:10447000756C740A546869732063616E20626520EC
:1044800064697361626C656420627920656E74652D
:1044900072696E67202473763D300A536565207417
:1044A00068652077696B692062656C6F7720666F3D
:1044B00072206D6F72652064657461696C732E0A79
:1044C00000546865736520636F6D6D616E64732061
:1044D000617265206163746976652066726F6D2014
:1044E00074686520636F6D6D616E64206C696E65C4
:1044F0003A0A205E78202020202020202020202022
:10450000202052657365742028636F6E74726F6C1F
:10451000207829202D20736F667477617265207270
:10452000657365740A20203F202020202020202051
:1045300020202020204D616368696E6520706F73B4
:104540006974696F6E20616E642067636F646520B3
:104550006D6F64656C2073746174650A202024207B
:1045600020202020202020202020202053686F772A
:1045700020616E642073657420636F6E6669677571
:10458000726174696F6E2073657474696E67730A03
:10459000202021202020202020202020202020201A
:1045A00046656564686F6C64202D2073746F70209D
:1045B0006D6F74696F6E20776974686F7574206CA5
:1045C0006F73696E6720706F736974696F6E0A200C
:1045D000207E20202020202020202020202020435A
:1045E00079636C65205374617274202D2072657339
:1045F000746172742066726F6D2066656564686FA1
:104600006C640A20206820202020202020202020E8
:1046100020202053686F7720746869732068656C68
:10462000702073637265656E0A2020246820202044
:1046300020202020202020202053686F7720636FC7
:104640006E66696775726174696F6E2068656C70FB
:104650002073637265656E0A20202474657374206C
:1046600020202020202020204C6973742073656C4A
:10467000662D74657374730A202024746573743D09
:104680004E2020202020202052756E2073656C66FD
:104690002D74657374204E0A202024686F6D653D6B
:1046A000312020202020202052756E206120686F4C
:1046B0006D696E67206379636C650A2020246465E8
:1046C00066613D3120202020202020526573746FC8
:1046D000726520616C6C2073657474696E677320F9
:1046E000746F2022666163746F727922206465663C
:1046F00061756C74730A000A0A0A23232320546923
:104700006E79472048656C70202323230A0022001D
:104710007B2272223A7B226D7367223A22007B72DF
:104720003A7B6D73673A22005B6A735D20206A737F
:104730006F6E2073657269616C697A652073747934
:104740006C65253964205B303D72656C6178656409
:104750002C313D7374726963745D0A005B6A765D27
:1047600020206A736F6E20766572626F7369747948
:1047700025313564205B303D73696C656E742C3176
:104780003D666F6F7465722C323D6D657373616742
:1047900065732C333D636F6E666967732C343D6CB3
:1047A000696E656E756D2C353D766572626F7365E9
:1047B0005D0A005B656A5D2020656E61626C652044
:1047C0006A736F6E206D6F646525313364205B30D2
:1047D0003D746578742C313D4A534F4E5D0A002D6F
:1047E00059275920591B5912590759FC58F058E4B8
:1047F00058D658BF58B058A3589758835876586120
:10480000584D584A584758385823580E58FF57EFB4
:1048100057DD57C657A9578C5773575D574C573AB2
:10482000572D571B570157FE56FB56F856F556F2B3
:1048300056EF56EC56E956E656E356E056DD56DAA4
:1048400056D756D456D156CE56CB56C856C556C254
:1048500056BF56BC56B956B656B356B056AD56AA04
:1048600056A756A456A1569E569B569856955692B4
:10487000568F568C5689568656835680567D567A64
:10488000567756745671566E566B56685665566214
:10489000563B561756F755DD55C355A955855568EE
:1048A0005550553A552055FC54DF54CD54AD5496CF
:1048B000547D545B54425424540854F053DE53C086
:1048C00053AB538A53865382537E537A5376537233
:1048D000536E536A53665362535E535A5356535240
:1048E000534E5334531A530753EB52D952C252A169
:1048F0005290527052505236521C520552D251A50B
:1049000051855163513D511651FA50DB50C150A7AA
:10491000508250595041501650EA4FB44F7F4F6D5E
:104920004F5B4F4C4F394F204FFE4EEC4EDA4EC886
:104930004EB64EA44E924E804E6E4E5C4E4A4E384F
:104940004E264E144E024EFE4DFA4DF64DF24DEEF1
:104950004DEA4DE64DE24DDE4DDA4DD64DD24DCE0F
:104960004DCA4DC64DC24DBE4DBA4DB64DB24D9E0F
:104970004D804D644D394D144DEF4CEB4CE74CE3FD
:104980004CDF4CDB4CD74CD34CCF4CCB4CC74CC33F
:104990004CBF4CBB4CB74CA34C874C6B4C4F4C336F
:1049A0004C174CFB4BDF4BC34BA74B8B4B6F4B5305
:1049B0004B4F4B4B4B474B434B3F4B3B4B374B23A7
:1049C0004BFB4AD44AAE4A814A5B4A2E4A2A4A26BF
:1049D0004A224A0F4AEE49D9494A6F6767696E67AA
:1049E000206379636C65206661696C656400507250
:1049F0006F626520656E64706F696E7420697320E4
:104A00007374617274696E6720706F696E740050A0
:104A1000726F6265206379636C65206661696C659D
:104A20006400323439003234380032343700486F91
:104A30006D696E67204572726F72202D20486F6D10
:104A4000696E67207377697463686573206D697335
:104A5000636F6E6669677572656400486F6D696E35
:104A600067204572726F72202D204E6567617469F0
:104A70007665206C61746368206261636B6F666643
:104A800000486F6D696E67204572726F72202D202D
:104A900054726176656C206D696E2026206D617898
:104AA00020617265207468652073616D6500486FD0
:104AB0006D696E67204572726F72202D204C617493
:104AC00063682076656C6F63697479206973207AF6
:104AD00065726F00486F6D696E67204572726F7204
:104AE000202D205365617263682076656C6F636961
:104AF0007479206973207A65726F00486F6D696EF2
:104B000067204572726F72202D20426164206F729F
:104B1000206E6F20617869732073706563696669C0
:104B2000656400486F6D696E67206379636C65200A
:104B30006661696C656400323339003233380032A3
:104B400033370032333600323335003233340032FB
:104B5000333300536F6674206C696D697420657817
:104B6000636565646564202D2043206D6178005382
:104B70006F6674206C696D6974206578636565641F
:104B80006564202D2043206D696E00536F6674208C
:104B90006C696D6974206578636565646564202D52
:104BA0002042206D617800536F6674206C696D69D6
:104BB00074206578636565646564202D2042206DEE
:104BC000696E00536F6674206C696D697420657836
:104BD000636565646564202D2041206D6178005314
:104BE0006F6674206C696D697420657863656564AF
:104BF0006564202D2041206D696E00536F6674201E
:104C00006C696D6974206578636565646564202DE1
:104C1000205A206D617800536F6674206C696D694D
:104C200074206578636565646564202D205A206D65
:104C3000696E00536F6674206C696D6974206578C5
:104C4000636565646564202D2059206D617800538B
:104C50006F6674206C696D6974206578636565643E
:104C60006564202D2059206D696E00536F66742095
:104C70006C696D6974206578636565646564202D71
:104C80002058206D617800536F6674206C696D69DF
:104C900074206578636565646564202D2058206DF7
:104CA000696E00536F6674206C696D697420657855
:104CB0006365656465640032313900323138003231
:104CC0003137003231360032313500323134003282
:104CD0003133003231320032313100323130003282
:104CE000303900323038003230370032303600543C
:104CF000726170657A6F696420706C616E6E657246
:104D0000206661696C656420746F20636F6E7665E0
:104D1000726765004C696D697420737769746368A4
:104D200020686974202D2053687574646F776E2035
:104D30006F63637572726564004D616368696E6567
:104D400020697320616C61726D6564202D20436F52
:104D50006D6D616E64206E6F742070726F63657329
:104D6000736564004D6F7665206C6573732074689D
:104D7000616E206D696E696D756D2074696D650079
:104D80004D6F7665206C657373207468616E206D5D
:104D9000696E696D756D206C656E67746800476536
:104DA0006E657269632054696E7947206572726F0F
:104DB0007200313939003139380031393700313931
:104DC0003600313935003139340031393300313969
:104DD0003200313931003139300031383900313861
:104DE0003800313837003138360031383500313845
:104DF0003400313833003138320031383100313845
:104E000030005420776F726420697320696E766178
:104E10006C6964005420776F7264206973206D6937
:104E20007373696E67005220776F72642069732014
:104E3000696E76616C6964005220776F72642069D4
:104E400073206D697373696E67005120776F7264A8
:104E500020697320696E76616C6964005120776FF8
:104E60007264206973206D697373696E67004C20EA
:104E7000776F726420697320696E76616C69640073
:104E80004C20776F7264206973206D697373696E4B
:104E900067004820776F726420697320696E7661BD
:104EA0006C6964004820776F7264206973206D69B3
:104EB0007373696E67004520776F72642069732091
:104EC000696E76616C6964004520776F7264206951
:104ED00073206D697373696E67004420776F726425
:104EE00020697320696E76616C6964004420776F75
:104EF0007264206973206D697373696E6700502056
:104F0000776F7264206973206E6F74206120766100
:104F10006C696420746F6F6C206E756D62657200D1
:104F20005020776F7264206973206E6F7420616EF9
:104F300020696E7465676572005020776F72642017
:104F40006973206E65676174697665005020776FBC
:104F50007264206973207A65726F005020776F72D7
:104F60006420697320696E76616C696400502077F3
:104F70006F7264206973206D697373696E67004195
:104F800072632073706563696669636174696F6ECB
:104F9000206572726F72202D20656E64706F696E6D
:104FA00074206973207374617274696E6720706F06
:104FB000696E74004172632073706563696669632A
:104FC0006174696F6E206572726F72202D2072613C
:104FD0006469757320617263206F7574206F662039
:104FE000746F6C6572616E636500417263207370EB
:104FF0006563696669636174696F6E206572726F5B
:1050000072202D206D697373696E67206F666673F9
:105010006574287329004172632073706563696643
:1050200069636174696F6E206572726F72202D20E2
:105030006D697373696E6720617869732865732978
:1050400000417263207370656369666963617469A6
:105050006F6E206572726F72005370696E646C655A
:10506000206D757374206265207475726E696E6749
:1050700020666F72207468697320636F6D6D616E56
:1050800064005370696E646C65206D757374206282
:1050900065206F666620666F72207468697320638E
:1050A0006F6D6D616E64005370696E646C65205342
:1050B00020776F726420697320696E76616C696411
:1050C000005370696E646C65205320776F726420A2
:1050D0006973206D697373696E67005370696E64DC
:1050E0006C652073706565642065786365656465CB
:1050F00064206D6178696D756D005370696E646CC4
:10510000652073706565642062656C6F77206D69DA
:105110006E696D756D0050726F6772616D6D65645B
:1051200020706F696E742073616D652061732063F8
:10513000757272656E7420706F696E740043757459
:1051400074657220636F6D70656E736174696F6EE4
:105150002063616E6E6F7420626520656E61626CA3
:105160006564005265717565737465642076656C5D
:105170006F636974792065786365656473206C6911
:105180006D697473004730206F72204731206D7550
:1051900073742062652061637469766520666F723E
:1051A0002047353300526F746172792061786573DE
:1051B0002063616E6E6F7420626520757365642074
:1051C00077697468207468697320636F6D6D616EB0
:1051D0006400496E76657273652074696D65206D33
:1051E0006F64652063616E6E6F74206265207573F5
:1051F00065642077697468207468697320636F6DD3
:105200006D616E64004665656472617465206E6FE1
:1052100074207370656369666965640053656C65C5
:105220006374656420706C616E6520697320696EBB
:1052300076616C69640053656C65637465642070A5
:105240006C616E65206973206D697373696E6700A8
:10525000417869732074617267657420706F736937
:1052600074696F6E20697320696E76616C69640081
:10527000417869732074617267657420706F736917
:1052800074696F6E206973206D697373696E67004E
:10529000417869732069732064697361626C656425
:1052A000004178697320697320696E76616C696466
:1052B00020666F72207468697320636F6D6D616E14
:1052C0006400417869732063616E6E6F742062655B
:1052D0002070726573656E74004178697320776F12
:1052E0007264206D697373696E670047636F6465EC
:1052F000206D6F64616C2067726F75702076696FC6
:105300006C6174696F6E004D20636F646520756E0B
:10531000737570706F727465640047636F646520A5
:10532000636F6D6D616E6420756E737570706F72F2
:105330007465640047656E657269632047636F64D6
:105340006520696E707574206572726F72003132FB
:1053500039003132380031323700313236003132E3
:1053600035003132340031323300313232003132E3
:1053700031003132300031313900313138003131D2
:10538000370031313600313135004A534F4E2074E9
:105390007874206669656C64732063616E6E6F74E7
:1053A000206265206E6573746564004A534F4E2019
:1053B000737472696E6720746F6F206C6F6E670014
:1053C0004A534F4E20696E70757420686173207463
:1053D0006F6F206D616E79207061697273004A533E
:1053E0004F4E2073796E746178206572726F72000F
:1053F000496E7075742076616C75652072616E6798
:1054000065206572726F7200496E707574206578E0
:105410006365656473206D6178696D756D20766173
:105420006C756500496E707574206C6573732074BB
:1054300068616E206D696E696D756D2076616C7541
:105440006500496E707574206578636565647320C6
:105450006D6178206C656E67746800436F6D6D6177
:105460006E64206E6F742061636365707465642080
:10547000617420746869732074696D65005061728D
:10548000616D657465722063616E6E6F7420626514
:10549000207265616400506172616D65746572208F
:1054A000697320726561642D6F6E6C7900556E733F
:1054B0007570706F72746564206E756D62657220B0
:1054C0006F72204A534F4E207479706500426164B8
:1054D000206E756D62657220666F726D6174004931
:1054E0006E76616C6964206F72206D616C666F729C
:1054F0006D656420636F6D6D616E6400556E7265DD
:10550000636F676E697A656420636F6D6D616E6449
:10551000206F7220636F6E666967206E616D650033
:1055200047656E6572696320617373657274696F34
:105530006E206661696C757265004D656D6F72797C
:10554000206661756C7420646574656374656400BD
:10555000537461636B206F766572666C6F7720643D
:105560006574656374656400436F6E74726F6C6C10
:10557000657220617373657274696F6E206661690C
:105580006C7572650043616E6F6E6963616C206D4E
:10559000616368696E6520617373657274696F6EAB
:1055A000206661696C75726500506C616E6E657223
:1055B00020617373657274696F6E206661696C75C2
:1055C00072650053746570706572206173736572E3
:1055D00074696F6E206661696C75726500456E63F3
:1055E0006F64657220617373657274696F6E206693
:1055F00061696C75726500494F207375622D73790E
:105600007374656D20617373657274696F6E206663
:1056100061696C75726500436F6E666967207375AA
:10562000622D73797374656D20617373657274692B
:105630006F6E206661696C75726500494F206D65FB
:105640006D6F727920616C6C6F636174696F6E202D
:10565000617373657274696F6E206661696C7572CF
:1056600065003838003837003836003835003834AF
:105670000038330038320038310038300037390014
:1056800037380037370037360037350037340037C2
:1056900033003732003731003730003639003638C2
:1056A00000363700363600363500363400363300E3
:1056B00036320036310036300035390035380035A5
:1056C0003700353600353500353400353300353296
:1056D00000353100353000343900343800343700BB
:1056E000343600343500343400343300343200347E
:1056F000310034300033390033380033370033366B
:105700000042616420737461747573207265706FF8
:1057100072742073657474696E6700506572736982
:105720007374656E6365206572726F7200466C6F8C
:105730006174206973204E414E00466C6F61742085
:10574000697320696E66696E697465004D6F766570
:105750002074696D65206973204E414E004D6F764F
:10576000652074696D6520697320696E66696E696C
:1057700074650047656E657269632065786365705E
:1057800074696F6E207265706F7274004661696C27
:10579000656420746F2067657420706C616E6E653F
:1057A00072206275666665720053797374656D2048
:1057B000616C61726D202D207368757474696E67F9
:1057C00020646F776E00496E697469616C697A61F3
:1057D00074696F6E206661696C75726500526561EF
:1057E000642D6F6E6C792061646472657373004917
:1057F0006E76616C69642041646472657373004401
:105800006976696465206279207A65726F00466CFA
:105810006F6174696E6720706F696E742065727253
:105820006F7200496E7465726E616C2072616E6792
:1058300065206572726F7200496E7465726E616C7C
:10584000206572726F720031390031380046756E12
:105850006374696F6E206973207374756262656426
:1058600000456E746572696E6720626F6F74206C9C
:105870006F6164657200496E697469616C697A6907
:105880006E67004275666665722066756C6C202DC9
:1058900020666174616C004275666665722066758B
:1058A0006C6C0042756666657220656D7074790077
:1058B0004E6F207375636820646576696365004D7B
:1058C00061782066696C652073697A652065786304
:1058D00065656465640046696C65206E6F74206F51
:1058E00070656E00456E64206F662066696C6500A9
:1058F000456E64206F66206C696E65004861726455
:10590000207265736574005465726D696E617465AB
:105910006400436F6D706C657465004E6F6F70004E
:1059200045616761696E004572726F72004F4B008E
:105930005B7031706F665D2070776D207068617389
:1059400065206F66662020202531352E3366205B6A
:10595000302E2E315D0A005B70317770685D2070EB
:10596000776D2063637720706861736520686925AF
:1059700031352E3366205B302E2E315D0A005B7090
:105980003177706C5D2070776D206363772070686D
:10599000617365206C6F2531352E3366205B302EA8
:1059A0002E315D0A005B70317773685D2070776D12
:1059B00020636377207370656564206869253135DD
:1059C0002E30662052504D0A005B703177736C5D4B
:1059D0002070776D20636377207370656564206C39
:1059E0006F2531352E30662052504D0A005B7031E4
:1059F0006370685D2070776D2063772070686173D5
:105A000065206869202531352E3366205B302E2EC7
:105A1000315D0A005B703163706C5D2070776D20C2
:105A20006377207068617365206C6F202531352E97
:105A30003366205B302E2E315D0A005B703163735C
:105A4000685D2070776D20637720737065656420D2
:105A50006869202531352E30662052504D0A005B92
:105A6000703163736C5D2070776D20637720737085
:105A7000656564206C6F202531352E3066205250CC
:105A80004D0A005B70316672715D2070776D206623
:105A900072657175656E63792020202531352E3051
:105AA0006620487A0A0053595354454D20524541C7
:105AB0004459004C6F6164696E6720636F6E66695C
:105AC00067732066726F6D20454550524F4D0049F7
:105AD0006E697469616C697A696E6720636F6E665E
:105AE00069677320746F2053686170656F6B6F32E4
:105AF000203530306D6D2070726F66696C65007B8B
:105B0000226572223A7B226662223A25302E326664
:105B10002C227374223A25642C226D7367223A2258
:105B20002573227D7D0A007B65723A7B66623A2589
:105B3000302E32662C73743A25642C6D73673A22CA
:105B40002573227D7D0A005B71765D20207175656D
:105B50007565207265706F727420766572626F73FE
:105B6000697479253764205B303D6F66662C313D62
:105B700073696E676C652C323D747269706C655D1B
:105B80000A00716F3A25640A0071693A25640A00B7
:105B900071723A25640A005B73765D20207374612C
:105BA000747573207265706F727420766572626F9F
:105BB00073697479253664205B303D6F66662C31DD
:105BC0003D66696C74657265642C323D76657262FF
:105BD0006F73655D0A005B73695D20207374617487
:105BE000757320696E74657276616C2531342E3060
:105BF00066206D730A004D6F746F722025632070EC
:105C00006F77657220656E61626C65642073746184
:105C100074653A25322E30660A005B257325735D64
:105C2000206D257320706F776572206D616E6167DE
:105C3000656D656E7425313064205B303D64697339
:105C400061626C65642C313D616C77617973206FA2
:105C50006E2C323D696E206379636C652C333D7721
:105C600068656E206D6F76696E675D0A005B2573EF
:105C700025735D206D257320706F6C617269747976
:105C800025313864205B303D6E6F726D616C2C3154
:105C90003D726576657273655D0A005B25732573D9
:105CA0005D206D2573206D6963726F737465707309
:105CB00025313664205B312C322C342C385D0A00BF
:105CC0005B257325735D206D257320747261766585
:105CD0006C20706572207265766F6C7574696F6E7A
:105CE0002531302E346625730A005B257325735DDC
:105CF000206D2573207374657020616E676C652557
:105D000032302E336625730A005B257325735D20C0
:105D10006D2573206D617020746F20617869732523
:105D2000313564205B303D582C313D592C323D5A81
:105D30002E2E2E5D0A005B6D745D20206D6F746FDA
:105D4000722069646C652074696D656F75742531A6
:105D5000342E3266205365630A00695D655D605DBF
:105D60002064656700206D6D0020696E005B7374B0
:105D70005D202073776974636820747970652531BC
:105D80003864205B303D4E4F2C313D4E435D0A0060
:105D90005465737420232564206E6F7420666F75BC
:105DA0006E640A004E312054314D360A4E3220477F
:105DB00031370A4E33204732310A4E3820463138C7
:105DC00030300A4E392047310A4E313030204739C1
:105DD0003220582D32352E313737592D33342E306D
:105DE0003732205A2D312E303030202854454D5036
:105DF0002C2052454D4F5645204C41544552290ABE
:105E00004E33343320582D32352E353935592D3314
:105E1000342E3334390A4E33343420582D32352E53
:105E2000373031592D33342E3433360A4E3334352E
:105E300020582D32352E373931592D33342E353205
:105E4000300A4E33343620582D32352E38363459F8
:105E50002D33342E3630310A4E33343720582D321C
:105E6000352E393230592D33342E3637390A4E33E8
:105E7000343820582D32352E393630592D33342EC2
:105E80003735340A4E33343920582D32352E3938CF
:105E900032592D33342E3832360A4E3335302058AD
:105EA0002D32352E393837592D33342E3839350ABD
:105EB0004E33353120582D32352E393736592D3362
:105EC000342E3936310A4E33353220582D32352EA4
:105ED000393438592D33352E3032330A4E33353379
:105EE00020582D32352E393033592D33352E303858
:105EF000320A4E33353420582D32352E383431594C
:105F00002D33352E3133380A4E33353520582D3266
:105F1000352E373633592D33352E3139300A4E333D
:105F2000353620582D32352E363639592D33352E0B
:105F30003233390A4E33353720582D32352E353528
:105F400039592D33352E3238340A4E3335382058EE
:105F50002D32352E343333592D33352E3332350A25
:105F60004E33353920582D32352E323931592D33B3
:105F7000352E3336330A4E33363020582D32352EF7
:105F8000313334592D33352E3339370A4E333631C8
:105F900020582D32342E393633592D33352E3432A4
:105FA000380A4E33363220582D32342E373737598F
:105FB0002D33352E3435350A4E33363320582D32B5
:105FC000342E353737592D33352E3437370A4E3383
:105FD000363420582D32342E333637592D33352E62
:105FE0003439360A4E33363520582D32342E31347A
:105FF00034592D33352E3531310A4E33363620584B
:106000002D32332E393039592D33352E3532320A6F
:106010004E33363720582D32332E363631592D3304
:10602000352E3532390A4E33363820582D32332E3C
:10603000343033592D33352E3533320A4E33363919
:1060400020582D32332E313333592D33352E3533FD
:10605000320A4E33373020582D32322E38353359EC
:106060002D33352E3532370A2F4E32353138204711
:106070003058302E333237592D33332E3532315A92
:106080002D312E3030300A4E32353139204D3330FB
:10609000004E31204732300A4E35204734302047F9
:1060A00031370A4E3130205431204D30360A284ED7
:1060B00031352047393020473020583020593020A2
:1060C0005A30290A4E3230205335303030204D308E
:1060D00033200A4E32352058302E30363420593095
:1060E0002E333236205A300A4E3430204730312099
:1060F0004631362E300A4E35302058302E30363468
:106100002059302E3332360A4E35352058302E3055
:1061100036302059302E3239330A4E36302058303E
:106120002E3037372059302E3236370A4E3635204A
:1061300058302E3131312059302E3235370A4E3712
:10614000302058302E3134392059302E3235320A31
:106150004E37352058302E3138382059302E3235D0
:10616000350A4E38302058302E3232372059302EF2
:106170003236380A4E38352058302E3235372059CD
:10618000302E3237310A4E39302058302E333335E5
:106190002059302E3236350A4E39352058302E34BB
:1061A00031322059302E3237310A4E3130302058BA
:1061B000302E3437342059302E3238370A4E3130B1
:1061C000352058302E3439312059302E3238390AA2
:1061D0004E3131302058302E3531372059302E3263
:1061E00037330A4E3131352058302E35343420596A
:1061F000302E3236330A4E3132302058302E353878
:10620000302059302E3236310A4E31323520583056
:106210002E3539352059302E3236330A4E3133304F
:106220002058302E3632312059302E3237340A4E33
:106230003133352058302E3635392059302E333011
:10624000360A4E3134302058302E3637332059300C
:106250002E3333350A4E3134352058302E36373907
:106260002059302E3336310A4E3135302058302EF9
:106270003637382059302E3338390A4E31353520EB
:1062800058302E3637302059302E3432300A4E31C5
:1062900036302058302E3637302059302E343436B0
:1062A0000A4E3136352058302E3638302059302EAF
:1062B0003437340A4E3137302058302E37303420BE
:1062C00059302E3439370A4E3137352058302E3771
:1062D00033322059302E3531350A4E31383020587E
:1062E000302E3739342059302E3533350A4E313877
:1062F000352058302E3837322059302E3536370A6F
:106300004E3139302058302E3935302059302E3624
:1063100030340A4E3139352058312E30333120593E
:10632000302E3634370A4E3230302058312E313448
:10633000392059302E3732320A4E3230352058311A
:106340002E3330382059302E3835340A4E32313021
:106350002058312E3433302059302E3938340A4EFB
:106360003231352058312E3434372059302E3938D7
:10637000360A4E3232302058312E363238205930DB
:106380002E3832320A4E3232352058312E373332DF
:106390002059302E3731340A4E3233302058322EC5
:1063A0003030392059302E3338310A4E32333520CF
:1063B00058322E3131362059302E3236360A4E328E
:1063C00034302058322E3232382059302E31353781
:1063D0000A4E3234352058322E3238302059302E81
:1063E0003132330A4E3235302058322E3333322098
:1063F00059302E3039340A4E3235352058322E3449
:1064000032332059302E3037300A4E323630205851
:10641000322E3438392059302E3036350A4E323645
:10642000352058322E3535372059302E3036360A41
:106430004E3237302058322E3632372059302E30F7
:1064400038340A4E3237352058322E3639332059F7
:10645000302E3130390A4E3238302058322E373310
:10646000302059302E3133330A4E323835205832ED
:106470002E3830352059302E3139300A4E323930ED
:106480002058322E3832392059302E3231360A4EC9
:106490003239352058322E3838302059302E3239A2
:1064A000310A4E3330302058322E383834205930AB
:1064B0002E3330300A4E3330352058322E383938AA
:1064C0002059302E3333320A4E3331302058322E99
:1064D0003930352059302E3336370A4E3331352096
:1064E00058322E3931302059302E3430370A4E335D
:1064F00032302058322E3930382059302E3434364C
:106500000A4E3332352058322E3930312059302E50
:106510003439350A4E3333302058322E383937204B
:1065200059302E3439350A4E3333352058322E380F
:1065300039302059302E3532340A4E333430205819
:10654000322E3834322059302E3630340A4E33341D
:10655000352058322E3831342059302E3636350A0F
:106560004E3335302058322E3739342059302E37BB
:1065700035300A4E3335352058322E3739312059CF
:10658000302E3833380A4E3336302058322E3831D8
:10659000392059302E3937360A4E333635205832A5
:1065A0002E3833372059312E3034340A4E333730B9
:1065B0002058322E3836322059312E3131320A4E9F
:1065C0003337352058322E3837372059312E313471
:1065D000350A4E3338302058322E39313220593175
:1065E0002E3231370A4E3338352058322E39313772
:1065F0002059312E3232360A4E3339302058322E5D
:106600003935312059312E3238310A4E333935205F
:1066100058322E3937302059312E3239350A4E341E
:1066200030302058322E3939362059312E32393512
:106630000A4E3430352058332E3031332059312E24
:106640003237350A4E3431302058332E3032342030
:1066500059312E3235340A4E3431352058332E30EC
:1066600037302059312E3135310A4E3432302058EE
:10667000332E3037372059312E3133340A4E3432ED
:10668000352058332E3132352059312E3033390AE6
:106690004E3433302058332E3133382059312E3098
:1066A00031390A4E3433352058332E3230352059A3
:1066B000302E3930380A4E3434302058332E3238A8
:1066C000322059302E3739370A4E3434352058337A
:1066D0002E3336312059302E3639310A4E3435308A
:1066E0002058332E3432362059302E3539320A4E66
:1066F0003435352058332E3435362059302E353444
:10670000330A4E3436302058332E3437392059303E
:106710002E3439330A4E3436352058332E3439343A
:106720002059302E3437320A4E3437302058332E29
:106730003530352059302E3434360A4E3437352032
:1067400058332E3531382059302E3431370A4E34F3
:1067500038302058332E3533302059302E333931EC
:106760000A4E3438352058332E3536342059302EE1
:106770003330300A4E3439302058332E35373720F5
:1067800059302E3235330A4E3439352058332E35B0
:1067900036382059302E3231320A4E3530302058BA
:1067A000332E3534342059302E3137360A4E3530B9
:1067B000352058332E3534312059302E3134360AB5
:1067C0004E3531302058332E3535332059302E3167
:1067D00031390A4E3531352058332E353736205968
:1067E000302E3130360A4E3532302058332E35397E
:1067F000372059302E3130320A4E35323520583359
:106800002E3631382059302E3130390A4E3533305A
:106810002058332E3633392059302E3132390A4E32
:106820003533352058332E3635302059302E31351A
:10683000390A4E3534302058332E3636332059300D
:106840002E3137380A4E3534352058332E36373806
:106850002059302E3139320A4E3535302058332EFA
:106860003639392059302E3139370A4E35353520F1
:1068700058332E3732332059302E3139360A4E35BF
:1068800036302058332E3736342059302E313739B0
:106890000A4E3536352058332E3830352059302EB3
:1068A0003136350A4E3537302058332E38383420BB
:1068B00059302E3135390A4E3537352058332E3977
:1068C00034392059302E3136350A4E35383020587B
:1068D000332E3936362059302E3137350A4E353879
:1068E000352058332E3937382059302E3139340A73
:1068F0004E3539302058332E3937382059302E3222
:1069000032330A4E3539352058332E393630205936
:10691000302E3234350A4E3630302058332E38334C
:10692000342059302E3331310A4E36303520583329
:106930002E3736322059302E3334350A4E36313028
:106940002058332E3732362059302E3338390A4EFC
:106950003631352058332E3730332059302E3435E8
:10696000380A4E3632302058332E363832205930DD
:106970002E3533300A4E3632352058332E363739DD
:106980002059302E3533340A4E3633302058332ECA
:106990003632362059302E3638310A4E36333520CD
:1069A00058332E3536382059302E3832380A4E3684
:1069B00034302058332E3434342059312E3038308E
:1069C0000A4E3634352058332E3430352059312E86
:1069D0003136370A4E3635302058332E3430342095
:1069E00059312E3136370A4E3635352058332E334D
:1069F00038372059312E3230380A4E36363020584A
:106A0000332E3338342059312E3230380A4E363650
:106A1000352058332E3336352059312E3236350A4B
:106A20004E3637302058332E3335352059312E32FB
:106A300038350A4E3637352058332E3334382059FE
:106A4000312E3330380A4E3638302058332E333317
:106A5000332059312E3335300A4E363835205833ED
:106A60002E3332312059312E3339310A4E363930F6
:106A70002058332E3331312059312E3432380A4EDA
:106A80003639352058332E3333392059312E3432AC
:106A9000330A4E3730302058332E343430205931B9
:106AA0002E3430360A4E3730352058332E353130BB
:106AB0002059312E3430380A4E3731302058332E99
:106AC0003538352059312E3432310A4E37313520A0
:106AD00058332E3631312059312E3433390A4E375E
:106AE00032302058332E3631312059312E34343162
:106AF0000A4E3732352058332E3631352059312E53
:106B00003434310A4E3733302058332E3633362062
:106B100059312E3438380A4E3733352058332E3613
:106B200033342059312E3531370A4E37343020581E
:106B3000332E3632322059312E3534330A4E373423
:106B4000352058332E3630352059312E3536330A1C
:106B50004E3735302058332E3537362059312E35C3
:106B600037350A4E3735352058332E3534342059D1
:106B7000312E3538310A4E3736302058332E3437DF
:106B8000392059312E3539320A4E373635205833AF
:106B90002E3435312059312E3539380A4E373730B9
:106BA0002058332E3338372059312E3632360A4E9C
:106BB0003737352058332E3339302059312E36337C
:106BC000360A4E3738302058332E3533322059317B
:106BD0002E3630320A4E3738352058332E36303183
:106BE0002059312E3539370A4E3739302058332E57
:106BF0003636382059312E3539380A4E3739352056
:106C000058332E3738322059312E3631320A4E3829
:106C100030302058332E3739342059312E36313820
:106C20000A4E3830352058332E3836382059312E18
:106C30003633360A4E3831302058332E3931382029
:106C400059312E3635350A4E3831352058332E39E4
:106C500034352059312E3636370A4E3832302058E6
:106C6000332E3936342059312E3638350A4E3832E3
:106C7000352058332E3936372059312E3638350ADB
:106C80004E3833302058332E3937342059312E3690
:106C900039390A4E3833352058332E393834205993
:106CA000312E3732350A4E3834302058332E3938A9
:106CB000342059312E3735380A4E38343520583380
:106CC0002E3937302059312E3739300A4E38353089
:106CD0002058332E3934352059312E3831370A4E69
:106CE0003835352058332E3931382059312E383245
:106CF000360A4E3836302058332E38393120593143
:106D00002E3832370A4E3836352058332E38343242
:106D10002059312E3830390A4E3837302058332E2A
:106D20003739382059312E3738340A4E3837352024
:106D300058332E3734362059312E3737320A4E38F1
:106D400038302058332E3639382059312E373634E2
:106D50000A4E3838352058332E3633352059312EE7
:106D60003736360A4E3839302058332E35353320F1
:106D700059312E3738350A4E3839352058332E34AC
:106D800037382059312E3832300A4E3930302058B9
:106D9000332E3430392059312E3836340A4E3930BA
:106DA000352058332E3334352059312E3931380AB5
:106DB0004E3931302058332E3236342059322E306D
:106DC00032330A4E3931352058332E323438205977
:106DD000322E3035310A4E3932302058332E32348B
:106DE000302059322E3038310A4E3932352058335E
:106DF0002E3331362059322E3038360A4E39333060
:106E00002058332E3339302059322E3130340A4E47
:106E10003933352058332E3431342059322E313223
:106E2000310A4E3934302058332E34333120593220
:106E30002E3135330A4E3934352058332E3433331E
:106E40002059322E3138300A4E3935302058332E01
:106E50003432372059322E3230350A4E393535200A
:106E600058332E3431332059322E3232340A4E39CF
:106E700036302058332E3339322059322E323432C4
:106E80000A4E3936352058332E3333352059322EB9
:106E90003234340A4E3937302058332E32373820C6
:106EA00059322E3233360A4E3937352058332E3286
:106EB00035362059322E3234320A4E393830205885
:106EC000332E3233392059322E3235310A4E393889
:106ED000352058332E3231312059322E3238300A93
:106EE0004E3939302058332E3137342059322E3331
:106EF00035360A4E3939352058332E313539205937
:106F0000322E3339370A4E313030302058332E315B
:106F100035302059322E3433380A4E313030352056
:106F200058332E3134302059322E3438310A4E3114
:106F30003031302058332E3133322059322E353112
:106F4000300A4E313031352058332E313138205906
:106F5000322E3534330A4E313032302058332E3011
:106F600039392059322E3537360A4E3130323520F4
:106F700058332E3035312059322E3633310A4E31C6
:106F80003033302058332E3030332059322E3636BD
:106F9000360A4E313033352058322E3935372059A4
:106FA000322E3638350A4E313034302058322E39B0
:106FB00030372059322E3639390A4E3130343520A7
:106FC00058322E3836302059322E3731310A4E3170
:106FD0003035302058322E3831392059322E373260
:106FE000370A4E313035352058322E373638205951
:106FF000322E3734350A4E313036302058322E3763
:1070000031362059322E3735370A4E313036352059
:1070100058322E3637352059322E3735370A4E3111
:107020003037302058322E3537392059322E373309
:10703000310A4E313037352058322E35373020590D
:10704000322E3732330A4E313038302058322E3516
:1070500035392059322E3732300A4E31303835200A
:1070600058322E3533302059322E3730310A4E31D6
:107070003039302058322E3530312059322E3639C1
:10708000330A4E313039352058322E3437312059B9
:10709000322E3638330A4E313130302058322E34C9
:1070A00034332059322E3636380A4E3131303520BD
:1070B00058322E3339362059322E3633340A4E3177
:1070C0003131302058322E3335342059322E353973
:1070D000310A4E313131352058322E333532205974
:1070E000322E3539310A4E313132302058322E337A
:1070F00032352059322E3534330A4E313132352073
:1071000058322E3331352059322E3532310A4E3134
:107110003133302058322E3330372059322E343923
:10712000380A4E313133352058322E323936205913
:10713000322E3436340A4E313134302058322E3229
:1071400039332059322E3432370A4E31313435201A
:1071500058322E3239352059322E3336360A4E31D6
:107160003135302058322E3332312059322E3330DF
:10717000330A4E313135352058322E3335382059C7
:10718000322E3234370A4E313136302058322E34D6
:1071900031392059322E3230330A4E3131363520D2
:1071A00058322E3431392059322E3137390A4E3186
:1071B0003137302058322E3430352059322E313587
:1071C000380A4E313137352058322E333632205975
:1071D000322E3132330A4E313138302058322E338C
:1071E00035342059322E3130340A4E313138352081
:1071F00058322E3335342059322E3039310A4E313F
:107200003139302058322E3338302059322E303632
:10721000350A4E313139352058322E34313020592B
:10722000322E3035310A4E313230302058322E3441
:1072300031302059322E3034370A4E313230352039
:1072400058322E3430352059322E3032380A4E31F1
:107250003231302058322E3430382059322E3031ED
:10726000300A4E313231352058322E3431362059E1
:10727000312E3939350A4E313232302058322E34DF
:1072800033332059312E3938320A4E3132323520DB
:1072900058322E3433382059312E3936330A4E3194
:1072A0003233302058322E3434372059312E39348D
:1072B000380A4E313233352058322E343631205987
:1072C000312E3933380A4E313234302058322E3490
:1072D00038302059312E3933310A4E31323435208D
:1072E00058322E3437382059312E3839390A4E3138
:1072F0003235302058322E3438372059312E383735
:10730000350A4E313235352058322E353034205939
:10731000312E3835340A4E313236302058322E353F
:1073200032372059312E3834380A4E313236352032
:1073300058322E3534392059312E3834390A4E31ED
:107340003237302058322E3537372059312E3836E3
:10735000310A4E313237352058322E3630342059EA
:10736000312E3836360A4E313238302058322E36E9
:1073700033312059312E3835340A4E3132383520E8
:1073800058322E3634302059312E3832370A4E31A9
:107390003239302058322E3634302059312E373998
:1073A000320A4E313239352058322E363239205990
:1073B000312E3735390A4E313330302058322E369F
:1073C00031322059312E3732370A4E3133303520A1
:1073D00058322E3537362059312E3639340A4E314F
:1073E0003331302058322E3533362059312E36364F
:1073F000320A4E313331352058322E34373020594D
:10740000312E3631360A4E313332302058322E3357
:1074100034352059312E3535310A4E31333235204D
:1074200058322E3330372059312E3532310A4E3111
:107430003333302058322E3236302059312E343802
:10744000320A4E313333352058322E3234332059FC
:10745000312E3437370A4E313334302058322E3201
:1074600032382059312E3436390A4E3133343520F2
:1074700058322E3232322059312E3434380A4E31BD
:107480003335302058322E3232382059312E3432B2
:10749000350A4E313335352058322E3235342059A5
:1074A000312E3430350A4E313336302058322E32B8
:1074B00036382059312E3337330A4E3133363520A2
:1074C00058322E3237392059312E3334320A4E3168
:1074D0003337302058322E3330382059312E32385D
:1074E000370A4E313337352058322E333430205955
:1074F000312E3235340A4E313338302058322E3462
:1075000030372059312E3230310A4E313338352060
:1075100058322E3434312059312E3135360A4E311D
:107520003339302058322E3435342059312E31330E
:10753000310A4E313339352058322E343630205905
:10754000312E3130360A4E313430302058322E341C
:1075500036342059312E3130320A4E313430352014
:1075600058322E3437312059312E3033360A4E31CD
:107570003431302058322E3436362059302E3937B7
:10758000310A4E313431352058322E3435312059BC
:10759000302E3839370A4E313432302058322E34BA
:1075A00031352059302E3739310A4E3134323520B9
:1075B00058322E3430332059302E3736370A4E3178
:1075C0003433302058322E3338382059302E373665
:1075D000350A4E313433352058322E333036205967
:1075E000302E3834310A4E313434302058322E3275
:1075F00032322059302E3931310A4E31343435206F
:1076000058322E3131342059302E3939350A4E3125
:107610003435302058322E3030322059312E303728
:10762000360A4E313435352058312E39303520590F
:10763000312E3133390A4E313436302058312E371D
:1076400035342059312E3232330A4E31343635201A
:1076500058312E3633372059312E3237380A4E31D1
:107660003437302058312E3538322059312E3330CE
:10767000310A4E313437352058312E3535382059BE
:10768000312E3331350A4E313438302058312E34D2
:1076900036302059312E3335320A4E3134383520C8
:1076A00058312E3339392059312E3336300A4E3184
:1076B0003439302058312E3333382059312E333578
:1076C000340A4E313439352058312E32383720596A
:1076D000312E3332390A4E313530302058312E3286
:1076E00034382059312E3239340A4E313530352074
:1076F00058312E3231372059312E3235340A4E313D
:107700003531302058312E3231342059312E323536
:10771000320A4E313531352058312E313732205929
:10772000312E3139350A4E313532302058312E3133
:1077300032382059312E3133390A4E313532352025
:1077400058312E3131302059312E3131370A4E31F6
:107750003533302058302E3935382059302E3934D1
:10776000310A4E313533352058302E3839312059D1
:10777000302E3837330A4E313534302058302E38D9
:1077800032352059302E3830380A4E3135343520D4
:1077900058302E3735352059302E3734370A4E3190
:1077A0003535302058302E3631392059302E363389
:1077B000330A4E313535352058302E34373720597D
:1077C000302E3532360A4E313536302058302E3490
:1077D00037372059302E3532340A4E313536352080
:1077E00058302E3431312059302E3437360A4E314C
:1077F0003537302058302E3333312059302E343540
:10780000340A4E313537352058302E32373820592A
:10781000302E3432370A4E313538302058302E323F
:1078200033312059302E3339370A4E31353835202F
:1078300058302E3138332059302E3337390A4E31F3
:107840003539302058302E3133352059302E3336EB
:10785000350A4E313539352058302E3037362059DB
:10786000302E3334310A4E31363035204730302017
:107870004633302E300A4E31363130204D303520EF
:107880000A4E3136313520473930205830205930B2
:10789000205A300A4E31363135204D33300A2845D2
:1078A0006E64206F6620434E432050726F67726192
:1078B0006D2900284D53472A2A2A2A204D696372D0
:1078C0006F737465702054657374205B76315D202E
:1078D0002A2A2A2A290A47303020473137204732BE
:1078E0003120473430204734392047383020473959
:1078F000300A6730783079307A300A7B22316D690E
:10790000223A317D0A7B22326D69223A317D0A7B2F
:1079100022336D69223A317D0A7B22346D69223A25
:10792000317D0A6730207831300A7B22316D69223F
:107930003A327D0A78300A7B22316D69223A347DF1
:107940000A7831300A7B22316D69223A387D0A7813
:10795000300A6730207931300A7B22326D69223A51
:10796000327D0A79300A7B22326D69223A347D0AEF
:107970007931300A7B22326D69223A387D0A7930BA
:107980000A6730207A31300A7B22336D69223A321D
:107990007D0A7A300A7B22336D69223A347D0A7A75
:1079A00031300A7B22336D69223A387D0A7A300AF7
:1079B0006730206131300A7B22346D69223A327D92
:1079C0000A61300A7B22346D69223A347D0A6131C2
:1079D000300A7B22346D69223A387D0A61300A6DA3
:1079E0003200284D53472A2A2A2A20436F6F726497
:1079F000696E617465206F66667365747320746563
:107A00007374205B76315D202A2A2A2A290A67307E
:107A1000306731376732316734306734396738302F
:107A20006739300A6735340A673932783079307A05
:107A3000300A663630300A284D53472A2A2A2A202F
:107A40007465737420473932206F6666736574738A
:107A50002A2A2A2A290A286D7367537465702031EF
:107A60003A204D6F76652066726F6D20302C302085
:107A7000746F2033302C30206D6D20696E20706F54
:107A800073697469766520582064697265637469E6
:107A90006F6E290A286D73675374657020323A201F
:107AA0005265736574206F726967696E20746F2008
:107AB000302E30207573696E6720473932290A28C5
:107AC0006D73675374657020333A204D6F7665206F
:107AD000746F2032302C302E2053686F756C642008
:107AE0006D6F7665203230206D6D20696E20706F6D
:107AF0007369746976652058206469726563746976
:107B00006F6E20616E64207374617475732072658A
:107B1000706F72742073686F756C64207374617217
:107B2000742066726F6D20302C30290A286D7367BF
:107B30005374657020343A204D6F766520746F2041
:107B4000302E3020202053686F756C64206D6F7666
:107B500065203230206D6D20696E206E656761741E
:107B6000697665205820646972656374696F6E2058
:107B7000616E6420737461747573207265706F72C6
:107B8000742073686F756C642073746172742066FE
:107B9000726F6D2032302C30290A67317833300A09
:107BA00067393278300A67317832300A6731783095
:107BB00079300A2473720A67393278300A67347070
:107BC000302E350A284D53472A2A2A2A20746573F5
:107BD0007420473535206F6666736574732A2A2AC8
:107BE0002A290A286D73675374657020313A20532F
:107BF000657420436F6F7264696E61746520737978
:107C00007374656D2032205B6735355D20746F209D
:107C10006F6666736574206F662035302C353029A9
:107C20000A286D73675374657020323A2053656C6F
:107C30006563742047353520636F6F7264696E61C8
:107C400074652073797374656D290A286D736753A1
:107C500074657020333A204D6F766520746F203044
:107C60002C302E20486561642073686F756C642029
:107C70006D6F766520646961676F6E616C6C7920E9
:107C8000696E202B5820616E64202B5920616E6430
:107C900020737461747573207265706F72742073D1
:107CA000686F756C642073746172742066726F6D96
:107CB00020302C30290A6731304C32703278353020
:107CC0007935300A6735350A6730783079300A6798
:107CD0003470302E350A284D53472A2A2A2A207418
:107CE00065737420473533206162736F6C757465FA
:107CF000206F7665727269646573202A2A2A2A29A0
:107D00000A286D73675374657020313A2052756E7E
:107D100020612073717561726520696E2047353569
:107D20002073797374656D290A286D7367537465C0
:107D30007020323A2052756E206120737175617225
:107D40006520772F473533206F76657272696465D9
:107D5000290A6730783079300A67307832307930E4
:107D60000A67307832307932300A673078307932C9
:107D7000300A6730783079300A673470302E350A2F
:107D80006735336730783079300A67353367307854
:107D9000323079300A6735336730783230793230B3
:107DA0000A673533673078307932300A67353367A0
:107DB00030783079300A6730783079300A6734703B
:107DC000302E350A284D53472A2A2A2A20746573F3
:107DD000742052657475726E20746F20686F6D65C3
:107DE000202A2A2A2A290A286D736753746570206D
:107DF000313A2052657475726E20746F20686F6D11
:107E000065207573696E6720473238290A286D73BB
:107E1000675374657020323A20526573657420741C
:107E20006F2047353420636F6F72642073797374E9
:107E3000656D290A6732380A6735340A6D333000B8
:107E4000284D53472A2A2A2A2054657374206163D7
:107E5000637572616379206F6620736C6F77206D34
:107E60006F766573205B76315D202A2A2A2A290ADB
:107E70006735350A6730783079300A673470302ECC
:107E8000350A673470302E350A6731783130663202
:107E9000320A6735340A6730783079300A6D33300A
:107EA00000284D53472A2A2A2A20546573742076C5
:107EB0006572792073686F7274206D6F76657320B8
:107EC0005B76315D202A2A2A2A290A6730783079A0
:107ED000300A673470302E350A673178302E3166BB
:107EE000313030300A78300A78302E310A78300A52
:107EF00078302E310A78300A78302E310A78300AFC
:107F000078302E310A78300A78302E310A78300AEB
:107F100078302E310A78300A78302E310A78300ADB
:107F200078302E310A78300A78302E310A78300ACB
:107F300078302E310A78300A78302E310A78300ABB
:107F400078302E310A78300A78302E310A78300AAB
:107F500078302E310A673470302E350A78300A783E
:107F6000302E30310A78300A78302E30310A7830AD
:107F70000A78302E30310A78300A78302E30310AC3
:107F800078300A78302E30310A78300A78302E3046
:107F9000310A78300A78302E30310A78300A783059
:107FA0002E30310A78300A78302E30310A78300A93
:107FB00078302E30310A78300A78302E30310A7815
:107FC000300A78302E30310A78300A78302E30314D
:107FD0000A78300A78302E30310A673078307930BC
:107FE0000A6D3200284D53472A2A2A2A20526F74DC
:107FF0006172792041786973204D6F74696F6E20CA
:1080000054657374205B76315D202A2A2A2A290A56
:1080100067303067313767323167343067343967FA
:1080200038306739300A6730783079307A306130EB
:10803000623063300A6735350A6730783079300A44
:108040006633363030300A6730613336300A623397
:1080500036300A633336300A61300A62300A6330E0
:108060000A673161313434300A62313434300A63A2
:10807000313434300A61300A62300A63300A6731C1
:10808000613134343062373230633336300A78301D
:1080900079307A306130623063300A673178363057
:1080A000613134343062373230633336300A7830FD
:1080B00079307A306130623063300A673178363037
:1080C00079353061313434306237323063333630B1
:1080D0000A783079307A306130623063300A673143
:1080E0007836307935307832356131343430623732
:1080F0003230633336300A783079307A306130622A
:108100003063300A6735340A6730783079300A6D69
:10811000333000284D53472A2A2A2A20496E766593
:108120007273652054696D65204D6F74696F6E20A0
:1081300054657374205B76315D202A2A2A2A290A25
:1081400067303067313767323167343067343967C9
:1081500038306739300A6735350A6730783079301A
:108160000A6739330A66302E30310A673178313088
:108170000A7931300A7A31300A6131300A78300AAE
:1081800079300A7A300A61300A67317831307931D2
:10819000307A2D31306131300A6730783079307A79
:1081A0003061300A66302E310A6732783130792DED
:1081B00031307A2D32306931300A67307830793099
:1081C0007A300A6733783130792D31307A2D323078
:1081D0006931300A6730783079307A300A6732781E
:1081E000323079307A2D32306931300A6730783068
:1081F00079307A300A673378323079306931300A31
:108200006730783079307A300A6732783079307A6E
:108210002D33306931300A6733783079307A3069FC
:1082200031300A6730783079307A300A6732783006
:108230007930693230202843572033363020646546
:108240006772656573290A6733783079306932302F
:1082500020284343572033363020646567726565B4
:1082600073290A6739340A6735340A6730783079F8
:10827000300A6D3330007B226763223A2267303048
:108280006731376732316734306734396738306780
:108290003930227D0A7B226763223A2267353522F4
:1082A0007D0A7B226763223A226730783079302258
:1082B0007D0A7B226763223A2266353030227D0AAE
:1082C0007B226763223A22284D534773717561728E
:1082D000657329227D0A7B226763223A2267307800
:1082E0003230227D0A7B226763223A2279323022A1
:1082F0007D0A7B226763223A227830227D0A7B2224
:108300006763223A227930227D0A7B226763223A10
:10831000226731783130227D0A7B226763223A223C
:10832000793130227D0A7B226763223A227830221B
:108330007D0A7B226763223A227930227D0A7B22E2
:108340006763223A22284D5347636972636C6573F1
:1083500029227D0A7B226763223A226732783130F4
:10836000792D3130693130227D0A7B226763223AD0
:1083700022673078307930227D0A7B226763223A87
:10838000226733783130792D3130693130227D0ADE
:108390007B226763223A22673078307930227D0A67
:1083A0007B226763223A2267327832307930693132
:1083B00030227D0A7B226763223A22673078307947
:1083C00030227D0A7B226763223A2267337832307B
:1083D0007930693130227D0A7B226763223A226735
:1083E0003078307930227D0A7B226763223A226717
:1083F0003278307930693130227D0A7B22676322FE
:108400003A22673378307930693130227D0A7B2215
:108410006763223A22673534227D0A7B2267632212
:108420003A22673078307930227D0A7B22676322D6
:108430003A226D3330227D00284D53472A2A2A2ABA
:10844000204D636F6465732074657374205B7631AF
:108450005D202A2A2A2A290A6735350A67307830AA
:1084600079300A6D330A673470310A6D350A673422
:1084700070310A6D340A673470310A6D350A673419
:1084800070310A6D370A673470310A6D390A673402
:1084900070310A6D380A673470310A6D390A6635F1
:1084A00030300A67307832300A7932300A6D330A58
:1084B00078300A6D340A79300A6D350A67317831BF
:1084C000300A6D370A7931300A6D380A78300A6D12
:1084D000390A79300A6732783130792D3130693193
:1084E000300A6D330A6730783079300A6D340A67A4
:1084F00033783130792D31306931300A6D350A6782
:1085000030783079300A6D370A6732783230793016
:108510006931300A6D380A6730783079300A6D3940
:108520000A673378323079306931300A6730783011
:1085300079300A6732783079306931300A673378B8
:108540003079306931300A6735340A6730783079EC
:10855000300A6D333000284D53472A2A2A2A2046F4
:10856000656564686F6C642054657374205B763154
:108570005D202A2A2A2A290A284D53472A2A2A2AEC
:10858000204D616E75616C6C7920656E746572202A
:108590002120616E64207E20647572696E67206D93
:1085A0006F76656D656E7420746F207465737420CA
:1085B0002A2A2A2A290A6735350A6730783079301D
:1085C0000A673470330A6730306731376732316792
:1085D00034306734396738306739300A66363030BE
:1085E0000A6730783130307637362E3736350A78AC
:1085F0003079300A6735340A6730783079300A6D5F
:10860000333000284D53472A2A2A2A204477656CA4
:108610006C2054657374205B76315D202A2A2A2AE7
:10862000290A6730306731376732316739300A6776
:1086300035350A6730783079300A663530300A6768
:10864000307831300A673470310A67307832300A56
:10865000673470310A67307831300A673470310A14
:1086600067307830300A673470310A79350A6735F7
:10867000340A6730783079300A6D330A67347031E4
:108680000A67307831307931300A6D350A673470D5
:10869000310A67307832307932300A6D340A673403
:1086A00070310A67307833307933300A6D380A67B1
:1086B0003470310A67307834307934300A6D390AD1
:1086C000673470310A67307835307935300A673071
:1086D000783079300A6D3330004E312067303067A2
:1086E000313767323167343067343967383067394A
:1086F000300A4E3130206730783079300A4E3230CF
:1087000020663530300A4E33302067327831307988
:108710002D313069313020284357203237302064E2
:10872000656772656573290A4E343020673078308A
:1087300079300A4E3530206733783130792D313039
:1087400069313020284343572039302064656772EF
:10875000656573290A4E3630206730783079300AE3
:108760004E38302067327832307930693130202805
:108770004357203138302064656772656573290A74
:108780004E3730206730783079300A4E38302067E5
:1087900033783230793069313020284343572031E3
:1087A00038302064656772656573290A4E39302058
:1087B0006730783079300A4E3939204631323030DE
:1087C0000A4E3130302067327830793069323020CB
:1087D00028435720333630206465677265657329F6
:1087E0000A4E3131302067327830793069323020AA
:1087F0002843572033363020616761696E290A4E5D
:10880000313230206637303020284368616E67652A
:1088100020666565642072617465207768696C659F
:1088200020696E204732206D6F74696F6E206D6F06
:108830006465290A4E3133302067327830793069E7
:10884000323020284357203336302033726420746E
:10885000696D65290A4E31343020673278307930BD
:108860006932302028435720333630203474682052
:1088700074696D65290A4E31353020663530300A0D
:108880004E313630206733783079307A343069327F
:1088900030202843435720333630206465677265A3
:1088A00065732077697468206C696E6561722074E5
:1088B000726176656C290A4E313730206733783023
:1088C00079307A30693230202843435720333630AC
:1088D00020616761696E290A4E3138302066373071
:1088E0003020286D73672A2A2A2A4368616E6765DB
:1088F00020666565642072617465207768696C65BF
:1089000020696E204733206D6F74696F6E206D6F24
:1089100064652A2A2A2A290A4E3139302067337899
:1089200030793069323020284343572033363020A5
:108930003372642074696D65290A4E3230302067C5
:10894000337830793069323020284343572033362A
:1089500030203474682074696D65290A4E323130D4
:1089600020286D73672A2A2A2A47313820457661E4
:108970006C20746573742A2A2A2A290A4E323230EE
:10898000204731205833302E373037205A35302E9B
:1089900037323720463530300A4E323330204731B7
:1089A0003820473032205836372E373338205A3265
:1089B000332E3631372052323520463235300A4E8A
:1089C000323430206738300A4E3235302067307804
:1089D0003079307A300A4E323630206D333000280C
:1089E0004D53472A2A2A2A205371756172657320D4
:1089F0004D6F74696F6E2054657374205B76315DC2
:108A0000202A2A2A2A290A6730306731376732310B
:108A10006734306734396738306739300A673078FF
:108A20003079300A67307832302028747261766588
:108A300072736520612032306D6D207371756172C3
:108A40006520696E205820616E642059290A7932A8
:108A5000300A78300A79300A67317831306635303B
:108A60003020286472617720612031306D6D207371
:108A7000717561726520696E205820616E6420599D
:108A80002061742046353030290A7931300A783037
:108A90000A79300A67307A3230202874726176653C
:108AA00072736520612032306D6D20737175617253
:108AB0006520696E205820616E64205A290A783238
:108AC000300A7A300A78300A6731783230793230B9
:108AD0007A32306635303020286665656420612042
:108AE00032306D6D20646961676F6E616C20696EF4
:108AF00020582C205920616E64205A290A78307938
:108B0000307A300A7834307934307A34302028742E
:108B10007261766572736520612034306D6D2063FB
:108B200075626520696E20582C205920616E642082
:108B30005A290A78343079307A300A7830793430EA
:108B40007A34300A7834307934307A300A783079AF
:108B5000307A34300A78307934307A300A783430E8
:108B600079307A34300A783079307A300A673830A0
:108B70000A6730783079300A673078310A673078A0
:108B8000300A6D333000284D53472A2A2A2A2048BC
:108B90006F6D696E672054657374205B76315D205C
:108BA0002A2A2A2A290A6732382E32783079307AEE
:108BB000300A6D333000284D53472A2A2A2A205381
:108BC0006D6F6B652054657374205B76315D202A70
:108BD0002A2A2A290A4730302047313720473231A4
:108BE0002047343020473439204738302047393047
:108BF0000A6D33673470310A6D35673470310A6D30
:108C000034673470310A6D33673470310A6D3567FB
:108C10003470310A6D37673470310A6D39673470DA
:108C2000310A6D38673470310A6D390A673078302F
:108C300079307A300A673030207832300A78300A5A
:108C40007932300A79300A7A32300A7A300A61325F
:108C5000300A61300A4730302078323020793230A3
:108C6000207A3230206132300A473030207830208C
:108C70007930207A302061300A4730312066333035
:108C8000207832207932207A322061320A783020FE
:108C90007930207A302061300A673078310A6730C5
:108CA00078300A6D32005B74765D202074657874CC
:108CB00020766572626F7369747925313564205B43
:108CC000303D73696C656E742C313D766572626FF0
:108CD00073655D0A0025660A00256C750A00257318
:108CE0000A0074696E7967205B25735D2065727276
:108CF0003A2025733A202573200074696E79672025
:108D00005B25735D206F6B3E2000456E64206F66AF
:108D100020636F6D6D616E642066696C650A001773
:108D2000C8B9C584C8A5C804C9FEC5DCCBB9C5701F
:108D3000CCDCCC0ACBFEC50000400640061040B893
:108D400000B8DCCBB9C570CCDCCC0ACBFEC50000CA
:108D5000400620060840B800B845CEB9C565CDE14B
:108D6000CD90CF2ECDA0084006050609010845CEBE
:108D7000B9C565CDE1CD16C9FEC5B00840060540B0
:108D8000B030800000000000F0E0D0C0100100CF43
:108D9000673322211F1B1301016E616E00696E662D
:108DA000004E414E494E495459494E46CDCCCC3DDA
:108DB0000AD7233C17B7D13877CC2B329595E624C8
:108DC0001FB14F0A000020410000C84200401C466D
:108DD00020BCBE4CCA1B0E5AAEC59D7400407A1012
:108DE000F35A00A0724E18090010A5D4E80000E85C
:108DF0007648170000E40B54020000CA9A3B0000BA
:108E000000E1F505000080969800000040420F0048
:108E10000000A08601000000102700000000E80309
:108E2000000000006400000000000A0000000000D4
:108E30000100000000002C76D888DC674F0823DF93
:108E4000C1DFAE59E1B1B796E5E3E453C63AE65166
:108E5000997696E8E6C28426EB898C9B62ED407C8D
:108E60006FFCEFBC9C9F40F2BAA56FA5F490055A29
:108E70002AF75C936B6CF9676DC11BFCE0E40D474E
:108E8000FEF520E6B500D0ED902E03009435770571
:108E90000080841E080000204E0A000000C80C3329
:108EA0003333330F986E12831141EF8D2114893BB8
:108EB000E65516CFFEE6DB18D1844B381BF77C1D38
:108EC000901DA4BBE424203284725E228100C9F18B
:108ED00024ECA1E53D2711241FBECFEFCDBFDFE578
:108EE000DEBF00E00CBF13E2A0E0B0E2E4E6F6EC87
:108EF00001E00BBF02C007900D92AA38B107D9F765
:108F00002CE5AAE8B3E201C01D92A237B207E1F74F
:108F10000E94E8800C9430E30C940000FC01608116
:108F20007181828193810E94DED460933F350895E0
:108F3000FC0160817181828193810E94DED4609303
:108F40003E350895AF92BF92CF92DF92EF92FF929B
:108F50000F931F93CF93DF937B018C0182ECC82E7C
:108F600084E3D82EE601AA24A394BC2EBC18F701F2
:108F700061917191819191917F012CEA35EC47E2E9
:108F800057E30E946DD618164CF4F80140815181C8
:108F9000628173818B2D0E941782A8820C5F1F4F04
:108FA0002196F4E3C83CDF0701F7DF91CF911F91D1
:108FB0000F91FF90EF90DF90CF90BF90AF900C9407
:108FC0002282FC0160817181828193810E94DED4C2
:108FD00060934035613019F481E00E94F57781E0BB
:108FE0000C941678CF93DF93CDB7DEB76897CDBFDB
:108FF000DEBFFC0160817181828193810E94DED499
:109000006093413581E0613019F40E94F5770CC01E
:109010000E941678CE01019628E1FC0111922A9552
:10902000E9F7BC010E94E1476896CDBFDEBFDF9142
:10903000CF9108950F931F93CF93DF93CDB7DEB7F2
:109040002D97CDBFDEBF27E0E8EDF0E28E010F5F88
:109050001F4FD80101900D922A95E1F7BC01660FD0
:10906000771F680F791F660F771F660F771F660FD0
:10907000771F69567A4E45E050E0CE0108960E946F
:10908000A4E0688570E0C8010E94D2E0009739F43E
:109090006B8570E0C8010E94D2E0009711F0801B40
:1090A00001C08FEF2D96CDBFDEBFDF91CF911F9115
:1090B0000F9108950F931F93CF93DF93CDB7DEB732
:1090C000C058D109CDBFDEBFFC010D9624852F937A
:1090D00023852F9322852F9321852F939F938F9301
:1090E0007196FF93EF939F938F937F936F938E016E
:1090F0000F5F1F4F1F930F930E945BE2C8010E94F6
:10910000CDBFCDBFDEBFC058DF4FCDBFDEBFDF91CB
:10911000CF911F910F910895EF92FF920F931F939C
:10912000CF93DF93CDB7DEB7C058D109CDBFDEBF37
:109130008C01F62EE72EFC01848195810E941A484D
:1091400083309CF58F3F09F03BC02FC09801235F0F
:109150003F4F9F938F93F80184858F9383858F93DF
:1091600082858F9381858F933F932F930F5E1F4F3F
:109170001F930F933F932F93EF92FF928E010F5FF8
:109180001F4F1F930F930E945BE2C8010E94CDBF47
:10919000CDBFDEBFC058DF4FCDBFDEBFDF91CF9167
:1091A0001F910F91FF90EF900895E6E1F4E1659132
:1091B00074914FE450E086E69FE30E94A4E0C6CF9E
:1091C000E0913835F0E0EE0FFF1FEE5EFB4E65914B
:1091D00074914FE450E086E69FE30E94A4E0B6CF8E
:1091E000EF92FF920F931F93CF93DF93CDB7DEB72C
:1091F000C058D109CDBFDEBF8C01F62EE72EFC0191
:10920000848195810E941A488330B4F58F3F09F01C
:109210003EC032C0A8014F5E5F4F9801235F3F4FB1
:109220009F938F93F80184858F9383858F93828595
:109230008F9381858F935F934F933F932F935F938A
:109240004F933F932F93EF92FF928E010F5F1F4F2B
:109250001F930F930E945BE2C8010E94CDBFCDBF58
:10926000DEBFC058DF4FCDBFDEBFDF91CF911F9172
:109270000F91FF90EF900895E6E1F4E1659174910C
:109280004FE450E086E69FE30E94A4E0C3CFE09164
:109290003835F0E0EE0FFF1FEE5EFB4E65917491E6
:1092A0004FE450E086E69FE30E94A4E0B3CFDF9254
:1092B000EF92FF920F931F93CF93DF93CDB7DEB75B
:1092C000C858D109CDBFDEBF8B01E42ED52E37E0C3
:1092D000EFEDF0E2DE01AF57BF4F01900D923A95EE
:1092E000E1F7C857DF4F2883C858D0400E941A487A
:1092F000F82EC857DF4F2881C858D04082E08F151C
:1093000018F0E22FF0E002C0E2E0F0E0EE0FFF1F05
:10931000EE5EFB4E659174914FE450E086E69FE36C
:109320000E94A4E09F938F93F80183818F938281A1
:109330008F9381818F9380818F93E1E8F0E0EC0F30
:10934000FD1FEF0DF11D80811F928F93DF92EF9231
:109350008E010F5F1F4F1F930F930E945BE2C801A6
:109360000E94CDBFCDBFDEBFC857DF4FCDBFDEBF30
:10937000DF91CF911F910F91FF90EF90DF900895B3
:109380004F925F926F927F92AF92BF92CF92DF9295
:10939000EF92FF920F931F93CF93DF93C2ECD4E32E
:1093A00007E813E35C018991813009F042C0F801BC
:1093B000C480D580E680F7804080518062807380D1
:1093C000A3019201C701B6010E94C1D29F772CEA86
:1093D00035EC47E257E30E946AD487FD2AC020E0BB
:1093E00034E244E759ECC701B6010E946DD6181665
:1093F0005CF4F5012081318142815381C701B601BE
:109400000E946DD6181604F120E034E244E759ECCE
:10941000C301B2010E946DD618165CF4F5012081DB
:10942000318142815381C301B2010E946AD487FD18
:109430000BC00B5C1F4FF4E0AF0EB11C84E3C83CC3
:10944000D80709F0B0CF02C08CED01C080E0DF91F9
:10945000CF911F910F91FF90EF90DF90CF90BF9031
:10946000AF907F906F905F904F9008958091BE3441
:10947000811105C08091BD348093BC3429C08230F5
:1094800031F487E08093BC348091BD3421C08330B7
:1094900031F489E08093BC348091BD3419C08430AC
:1094A00031F48AE08093BC348091BD3411C0809146
:1094B000BF34813031F485E08093BC348091BD3479
:1094C00007C0823019F486E08093BC348091BD34AB
:1094D000863019F08091BC3408958BE08093BC34C1
:1094E00008958091BD3408958093BF34813059F040
:1094F00018F0823041F008958DEE94E38093EB34C0
:109500009093EC34089585EB98E58093EB34909339
:10951000EC340895FC0184810895845B9F4FFC0125
:1095200080810895855B9F4FFC0180810895825B57
:109530009F4FFC0180810895815B9F4FFC018081DA
:109540000895875B9F4FFC01808108950C941897C4
:10955000CD96FC0160817181828193810895FC0127
:10956000648308958B5A9F4FFC01608308958F5B3D
:109570009F4FFC01408351836283738308956093FE
:10958000ED347093EE348093EF349093F03488EEA2
:1095900091E20C945162BF92CF92DF92EF92FF92D0
:1095A0000F931F93CF93DF93D0903A357C010FE553
:1095B00015E38091393590E0EC01CC0FDD1FC80F29
:1095C000D91FCC0FDD1FCC0FDD1FCC0FDD1FCA5202
:1095D000DD4C81E0D816A9F0B881A981CA80BB8092
:1095E0004091B235413091F4F801208131814281BE
:1095F00053816B2F7A2F8C2D9B2D0E94C2D29B0101
:1096000009C020E030E080E090E004C02B2F3A2F2A
:109610008C2D9B2DA901BC01F701458F568F678FBB
:1096200070A3F4E0EF0EF11C0C5F1F4F249685E34E
:109630000737180771F6DF91CF911F910F91FF90B7
:10964000EF90DF90CF90BF900895835B9F4FFC0118
:1096500060838DEE94E30C94CB4A4F925F926F92AD
:109660007F928F929F92AF92BF92CF92DF92EF92B2
:10967000FF920F931F93CF93DF93CDB7DEB7689719
:10968000CDBFDEBF8C016091B23570E080E090E02C
:109690000E940CD52B013C01F8016081718182810F
:1096A00093810E94DED470E05B01AA0CBB1CA60E65
:1096B000B71EAA0CBB1CAA0CBB1CAA0CBB1CC50168
:1096C0008A529D4C5C010FE515E3FE0131964F0176
:1096D000F501C190D190E190F1905F01F8016191A5
:1096E0007191819191918F01A30192010E940FD7F5
:1096F0009B01AC01C701B6010E94C2D2F401619383
:109700007193819391934F01F5E307371F0701F799
:10971000CE0101960E94FB968DEE94E30E94CB4A07
:109720006896CDBFDEBFDF91CF911F910F91FF9063
:10973000EF90DF90CF90BF90AF909F908F907F90F1
:109740006F905F904F9008958D5E944369F4E62F7B
:10975000F0E0EE0FFF1FEE0FFF1FE95BFA4C608198
:109760007181828193810895862F0C94F096CF9217
:10977000DF92EF92FF920F931F93CF93DF93EC0151
:1097800084E3CD3ED80709F04AC070E0FB01EE0F3C
:10979000FF1FEE0FFF1FE95BFA4CC080D180E28013
:1097A000F38080913A35813059F18091393590E0DC
:1097B000FC01EE0FFF1FE80FF91FEE0FFF1FE60F72
:1097C000F71FEE0FFF1FEE0FFF1FEA52FD4C008147
:1097D0001181B281A3812091B2352130B1F4FB0116
:1097E000EE0FFF1FEE0FFF1FE15AFA4C208131816F
:1097F00042815381B8018B2F9A2F0E94C2D208C098
:1098000060E070E080E090E003C0B8018B2F9A2FF9
:109810009B01AC01C701B6010E94C1D203C0862FD3
:109820000E940497C55BDF4F2881211106C023E306
:1098300033E34BEC51E40E9471D4DF91CF911F913F
:109840000F91FF90EF90DF90CF90089588E1E2EFC5
:10985000F4E3A7E4B5E301900D928A95E1F78091D6
:10986000363581110CC08091F134813041F4109271
:109870002A3510922B3510922C3510922D350895E3
:109880004F925F926F927F928F929F92AF92BF9210
:10989000CF92DF92EF92FF920F931F93CF93DF93BC
:1098A000CDB7DEB76997CDBFDEBF8091BE348111E1
:1098B00055C08091E334813009F050C00E9458C5F2
:1098C00081114CC01092E3349EEE692E92E3792E02
:1098D00026E3822E912C8E010E5E1F4F36EEA32EB4
:1098E00030E2B32E33C0F70181917F011F928F9335
:1098F0005F924F92BF92AF921F930F930E9432E2FA
:10990000B80187E493E20E94735F8D839E83F60122
:1099100081919191A191B1916F018A879B87AC87C9
:10992000BD87CE0101960E943B5CCDBFDEBF9EEDA0
:10993000E91690E2F906B9F6E8E16E0E711CFFEF48
:109940008F1A9F0A8CE38816910441F0240189ED57
:10995000E82E80E2F82E630188E7C8CF80E06996A0
:10996000CDBFDEBFDF91CF911F910F91FF90EF90A0
:10997000DF90CF90BF90AF909F908F907F906F902F
:109980005F904F9008952F923F924F925F926F9207
:109990007F928F929F92AF92BF92CF92DF92EF927F
:1099A000FF920F931F93CF93DF93CDB7DEB7299725
:1099B000CDBFDEBF4C015B0140903C3550903A3545
:1099C000209039356090B235709038356B0182EF58
:1099D00094E3888799875EE7E52E53E3F52E98E1B7
:1099E000299E100111248401D6016D917D918D91E4
:1099F0009D916D012CEA35EC47E257E30E946AD451
:109A000087FD80C0F70180818150823008F07AC0E4
:109A100041104CC0F1E05F1609F1E885F985E20DCF
:109A2000F31DEC51F2408081898391819D83B28145
:109A3000A381E1E06E1217C0E885F985E359FF4F75
:109A40002081318142815381BC018B2F9A2F0E944A
:109A5000C2D269837D838E839F8307C019821D8252
:109A60001E821F8202C0BE83AF8371100CC023E32D
:109A700033E34BEC51E4D8016D917D918D919C9134
:109A80000E940FD705C0F8016081718182819381A6
:109A900029813D814E815F810E94C2D2A885B9850E
:109AA0006D937D938D939C9313972CC0A885B98556
:109AB0008D919D910D90BC91A02D89839A83AB834C
:109AC000BC8371100EC023E333E34BEC51E4F80187
:109AD00060817181828193810E940FD79B01AC01CB
:109AE00005C0D8012D913D914D915C9169817A819C
:109AF0008B819C810E94C2D2E885F9856083718345
:109B0000828393838885998504968887998795E3CE
:109B1000E90EF11C0C5F1F4FA885B985AE5FB443F9
:109B200009F062CF6090383570903C35F0913A354D
:109B3000F983C09039352091B2352D838CE0A80E81
:109B4000B11CADE1B4E3A887B9874EEFE42E44E33E
:109B5000F42EB8E1CB9E600111248401F5016191DE
:109B60007191819191915F012CEA35EC47E257E3C5
:109B70000E946AD487FD8CC0A885B9858C91882302
:109B800009F486C08150823030F4F8012484358491
:109B9000468457843BC0611016C023E333E34BEC8B
:109BA00051E4D8011C966D917D918D919C911F97E8
:109BB0000E940FD720E030E044EB53E40E940FD71F
:109BC0001B012C010DC020E030E044EB53E4F80110
:109BD00064857585868597850E940FD71B012C01AA
:109BE0002BED3FE049EC50E4A885B98591966D9145
:109BF0007D918D919C9194970E940FD79B01AC0110
:109C0000C201B1010E9471D41B012C01711031C03D
:109C1000B981B130E1F0F701EC0DFD1DEC51F240DE
:109C2000A081B18192808380ED81E130A1F4F701C0
:109C3000E359FF4F2081318142815381BD01892D3C
:109C4000982D0E94C2D2DB01982E892E04C0A0E07C
:109C5000B0E0912C812CA2019101BD01892D982D9C
:109C60000E94C2D2D7016D937D938D939C931397DD
:109C70000FC0A2019101F7016081718182819381FE
:109C80000E94C2D2D7016D937D938D939C931397BD
:109C9000E885F985F596E887F987F4E0EF0EF11C81
:109CA0000C5F1F4F888599858C5B944309F056CFD4
:109CB0002996CDBFDEBFDF91CF911F910F91FF900D
:109CC000EF90DF90CF90BF90AF909F908F907F905C
:109CD0006F905F904F903F902F9008958091BA328F
:109CE0009091BB328F3E924111F08FE508958091A3
:109CF0007136909172368F3E9241B9F7809143351B
:109D0000909144358F3E924181F78091B935909181
:109D1000BA358F3E924149F780910D5990910E5975
:109D20008F3E924111F78091CA599091CB598F3E45
:109D30009241D9F680E00895CF93C82F0E9407A8DA
:109D400082E08093BD348C2FCF9108958091BE34F2
:109D5000811104C083E08093BD3403C085E080930B
:109D6000BD3480E00895CF93C82F0E944BB380E0AC
:109D70000E94E0AE8C2F0E9407A886E08093BD343D
:109D80008C2FCF9108958093373580E0089580938C
:109D9000383580E0089580933C3580E008954F92F7
:109DA0005F926F927F929F92AF92BF92CF92DF921B
:109DB000EF92FF920F931F93CF93DF93C82FB62E8E
:109DC0008A01F22ED32F8FEF8C0F863008F082C0DD
:109DD0006091453670E080E090E00E940CD52CEA5E
:109DE00035EC47E257E30E946AD487FD75C082E0F4
:109DF000B81619F0E4E1BE1271C090903835CF2C3E
:109E0000DD2E8C2F90E0EC01CC0FDD1FC80FD91F89
:109E1000CC0FDD1FCC0FDD1FCC0FDD1FCA52DD4C78
:109E2000780107E415E3AA24A394F60161917191E6
:109E3000819191916F012CEA35EC47E257E30E9442
:109E40006DD61816DCF5F2E0BF1214C091100CC0EC
:109E500023E333E34BEC51E4F701608171818281AC
:109E600093810E940FD724C0F701608171818281A4
:109E700093811EC0F80140805180628073809110F0
:109E80000EC023E333E34BEC51E4F70160817181B1
:109E9000828193810E940FD79B01AC0105C0F7011D
:109EA0002081318142815381C301B2010E94C1D21C
:109EB000688379838A839B83A092E3342496F4E0B9
:109EC000EF0EF11C0C5F1F4F85E30F35180709F0EB
:109ED000ACCF06C081EA05C08CEA03C08DEA01C0A0
:109EE00080E0DF91CF911F910F91FF90EF90DF9075
:109EF000CF90BF90AF909F907F906F905F904F906A
:109F00000895CF93DF93CDB7DEB76897CDBFDEBF9F
:109F100080933935682F70E080E090E00E940AD588
:109F200069837A838B839C831D821E821F8218869D
:109F300019861A861B861C861D861E861F86188A11
:109F4000198A1A8A1B8A1C8A1D8A1E8A1F8A188EE1
:109F5000AE014F5F5F4FBA018DE29BE40E945983CF
:109F600080E06896CDBFDEBFDF91CF910895CF939B
:109F7000DF93EDEEF4E386E5DF011D928A95E9F7C4
:109F80008BE5ABEBB5E3ED01982F19929A95E9F7C4
:109F9000A6E1B6E3ED0119928A95E9F78FEE92E119
:109FA0008093BA329093BB3280937136909372361D
:109FB00080934335909344358093B9359093BA3567
:109FC00080930D5990930E598093CA599093CB5911
:109FD000E093EB34F093EC348091D33280933835B6
:109FE0008091D1320E94814F8091D2328093373557
:109FF0008091D43280933B358091D53280933C352B
:10A0000081E0809336358093B33594E09093F134BA
:10A010001092E4341092E5341092E6348093BD340B
:10A020008093BC340E947EADDF91CF910C949B84D1
:10A03000CF92DF92EF92FF92CF93C82F6A017B01FC
:10A04000E82FF0E0DF01AA0FBB1FAA0FBB1FA95B1F
:10A05000BA4C4D935D936D937C931397EE0FFF1F56
:10A06000EE0FFF1FEE50FB4C4083518362837383DE
:10A070008C2F0E940C82B701A6018C2F0E941782A0
:10A08000CF91FF90EF90DF90CF900C9422829F921F
:10A09000AF92BF92CF92DF92EF92FF920F931F93F6
:10A0A000CF93DF93CDB7DEB76897CDBFDEBF962ED7
:10A0B000A72EC62ED72E7C0100E010E0B12CF601B1
:10A0C00061917191819191916F012CEA35EC47E298
:10A0D00057E30E946DD61816A4F58091383581118A
:10A0E0000EC023E333E34BEC51E4F701608171814F
:10A0F000828193810E940FD7AB01BC0105C0F7019B
:10A100004081518162817381E1E0F0E0EC0FFD1F3D
:10A11000E00FF11F4083518362837383C80186542B
:10A120009D4CFC01E357FD4F408351836283738351
:10A13000E555F10940835183628373838B2D0E941F
:10A140000C82B3940C5F1F4FF4E0EF0EF11C08314A
:10A15000110509F0B4CF492D5A2DBE016F5F7F4F15
:10A1600082EA97E40E94598380E06896CDBFDEBF03
:10A17000DF91CF911F910F91FF90EF90DF90CF90E3
:10A18000BF90AF909F9008954F925F926F927F9291
:10A190008F929F92AF92BF92CF92DF92EF92FF92F7
:10A1A0000F931F93CF93DF93CDB7DEB76897CDBFE3
:10A1B000DEBF21E02093B23580903935909038355C
:10A1C0005B016C0107E415E3882D90E07C01EE0C47
:10A1D000FF1CE80EF91EEE0CFF1CEE0CFF1CEE0C33
:10A1E000FF1CC7018A529D4C7C01F5016191719160
:10A1F000819191915F012CEA35EC47E257E30E948F
:10A200006DD6181664F5F7012081318142815381A2
:10A21000F80160817181828193810E94C1D22B01FA
:10A220003C0191100EC023E333E34BEC51E4F60103
:10A2300060817181828193810E940FD79B01AC0163
:10A2400005C0F6012081318142815381C301B201F1
:10A250000E94C1D2F801608F718F828F938FF4E0DA
:10A26000CF0ED11C0C5F1F4F84E0E80EF11C95E36C
:10A270000F35190709F0B9CF682D70E080E090E044
:10A280000E940AD569837A838B839C831D821E82F8
:10A290001F82188619861A861B861C861D861E86B6
:10A2A0001F86188A198A1A8A1B8A1C8A1D8A1E8A86
:10A2B0001F8A188EAE014F5F5F4FBA018DE29BE49B
:10A2C0000E94598380E06896CDBFDEBFDF91CF91B9
:10A2D0001F910F91FF90EF90DF90CF90BF90AF90C4
:10A2E0009F908F907F906F905F904F900895CF9345
:10A2F000DF93CDB7DEB76897CDBFDEBF1092B23522
:10A3000010925F351092603510926135109262356F
:10A31000109263351092643510926535109266354F
:10A3200010926735109268351092693510926A352F
:10A3300010926B3510926C3510926D3510926E350F
:10A3400010926F35109270351092713510927235EF
:10A3500010927335109274351092753510927635CF
:10A360006091393570E080E090E00E940AD5698301
:10A370007A838B839C831D821E821F821886198696
:10A380001A861B861C861D861E861F86188A198AB9
:10A390001A8A1B8A1C8A1D8A1E8A1F8A188EAE0181
:10A3A0004F5F5F4FBA018DE29BE40E94598380E0CA
:10A3B0006896CDBFDEBFDF91CF910895CF93DF9335
:10A3C000CDB7DEB76897CDBFDEBF1092B2356091D2
:10A3D000393570E080E090E00E940AD569837A8385
:10A3E0008B839C831D821E821F82188619861A8683
:10A3F0001B861C861D861E861F86188A198A1A8A45
:10A400001B8A1C8A1D8A1E8A1F8A188EAE014F5F06
:10A410005F4FBA018DE29BE40E94598380E0689609
:10A42000CDBFDEBFDF91CF910895CF93DF93CDB73E
:10A43000DEB76897CDBFDEBF81E08093B235609113
:10A44000393570E080E090E00E940AD569837A8314
:10A450008B839C831D821E821F82188619861A8612
:10A460001B861C861D861E861F86188A198A1A8AD4
:10A470001B8A1C8A1D8A1E8A1F8A188EAE014F5F96
:10A480005F4FBA018DE29BE40E94598380E0689699
:10A49000CDBFDEBFDF91CF910895CF931092F134FD
:10A4A0000E94C34C8091C432813069F482EF94E3FE
:10A4B0000E94C049C82F882331F00E9407A882E07B
:10A4C0008093BD3417C08DEE94E30E94CB4A85E0A3
:10A4D0008093BD348091BE34811105C081E08093AA
:10A4E000BE340E94F3AB8DEE94E30E9425970E9448
:10A4F000264CC0E08C2FCF91089588E1E7E4F5E386
:10A50000A7E7B5E301900D928A95E1F780E0089501
:10A510000F931F93CF93DF93CDB7DEB76A97CDBF6D
:10A52000DEBF8C0181E080933A358DEE94E3698F34
:10A530007A8F0E94CB4A698D7A8DC8010E944D5254
:10A540000E9493828823E1F388E1E0E0F0E2DE01FB
:10A55000119601900D928A95E1F7BE016F5F7F4FD2
:10A5600087E795E30E944D526A96CDBFDEBFDF912B
:10A57000CF911F910F91089588E1E7E4F5E3AFE8EB
:10A58000B5E301900D928A95E1F780E008950F936D
:10A590001F93CF93DF93CDB7DEB76A97CDBFDEBFF2
:10A5A0008C0181E080933A358DEE94E3698F7A8F48
:10A5B0000E94CB4A698D7A8DC8010E944D520E943B
:10A5C00093828823E1F388E1E0E0F0E2DE01119676
:10A5D00001900D928A95E1F7BE016F5F7F4F8FE882
:10A5E00095E30E944D526A96CDBFDEBFDF91CF91B9
:10A5F0001F910F910895FB01DC0180913635811187
:10A6000011C09B01AD0160E070E080E89FE30E9413
:10A6100071D460932A3570932B3580932C359093A9
:10A620002D3518C080913835811109C023E333E3FB
:10A630004BEC51E4CD010E940FD7FB0101C0CD01CD
:10A64000AF01BC0140932A3550932B3560932C35D4
:10A6500070932D3580E008958093363580E008951D
:10A6600080933B3580E008956093323570933335A5
:10A6700080933435909335350E94B18380E00895FE
:10A680000F931F93CF93DF93EC018B0180913635AD
:10A69000882399F080912A3590912B35A0912C3503
:10A6A000B0912D35BC01CD019F772CEA35EC47E206
:10A6B00057E30E946AD487FD30C081E08093F13473
:10A6C000B801CE010E94C34C8091C432813069F43C
:10A6D00082EF94E30E94C049C82F882331F00E9482
:10A6E00007A882E08093BD3419C08DEE94E30E94E8
:10A6F000CB4A85E08093BD348091BE34811105C082
:10A7000081E08093BE340E94F3AB8DEE94E30E940F
:10A710002597C82F0E94264C01C0CEE88C2FDF91D0
:10A72000CF911F910F910895CF93DF93CDB7DEB7EF
:10A730006897CDBFDEBF682F70E080E090E00E9498
:10A740000AD569837A838B839C831D821E821F8234
:10A75000188619861A861B861C861D861E861F86ED
:10A76000188A198A1A8A1B8A1C8A1D8A1E8A1F8ABD
:10A77000188EAE014F5F5F4FBA018EE897E40E94DA
:10A78000598380E06896CDBFDEBFDF91CF910895F9
:10A79000CF93DF93CDB7DEB76897CDBFDEBF6091B3
:10A7A0003F3570E080E090E00E940AD569837A83AB
:10A7B0008B839C831D821E821F82188619861A86AF
:10A7C0001B861C861D861E861F86188A198A1A8A71
:10A7D0001B8A1C8A1D8A1E8A1F8A188EAE014F5F33
:10A7E0005F4FBA0188E997E40E94598380E0689638
:10A7F000CDBFDEBFDF91CF910895CF93DF93CDB76B
:10A80000DEB76897CDBFDEBF682F70E080E090E0D4
:10A810000E940AD569837A838B839C831D821E8262
:10A820001F82188619861A861B861C861D861E8620
:10A830001F86188A198A1A8A1B8A1C8A1D8A1E8AF0
:10A840001F8A188EAE014F5F5F4FBA0181EE97E409
:10A850000E94598380E06896CDBFDEBFDF91CF9123
:10A860000895CF93DF93CDB7DEB76897CDBFDEBF36
:10A87000682F70E080E090E00E940AD569837A83B7
:10A880008B839C831D821E821F82188619861A86DE
:10A890001B861C861D861E861F86188A198A1A8AA0
:10A8A0001B8A1C8A1D8A1E8A1F8A188EAE014F5F62
:10A8B0005F4FBA0182EF97E40E94598380E0689667
:10A8C000CDBFDEBFDF91CF910895CF93FC016081B2
:10A8D0007181828193810E94DED46093BD34109295
:10A8E000BF348DEE94E38093EB349093EC348091FD
:10A8F000BE34813011F41092BE341092C0341092E4
:10A90000E6340E94DE96C091BD34C430C9F40E9482
:10A9100077518091D1320E94814F8091D2328093C1
:10A9200037358091D53280933C3580E00E94E0AE8F
:10A9300080E00E94315481E080933635C093F13439
:10A9400081E0CF910C94D1AA8093AF358093B0353C
:10A950008093B83580E008952CEA35EC47E257E360
:10A9600060915D3670915E3680915F369091603671
:10A970000E946DD61816B4F4809102369091033679
:10A98000A0910436B0910536BC01CD019F772CEA29
:10A9900035EC47E257E30E946AD487FF03C0109268
:10A9A000AF3503C081E08093AF3580E00895809398
:10A9B000AF358091023690910336A0910436B09164
:10A9C00005368093A7359093A835A093A935B09309
:10A9D000AA3580E008952CEA35EC47E257E3609110
:10A9E0005D3670915E3680915F36909160360E9440
:10A9F0006DD61816B4F48091023690910336A0916A
:10AA00000436B0910536BC01CD019F772CEA35ECB8
:10AA100047E257E30E946AD487FF03C01092B03523
:10AA200003C081E08093B03580E008958093B03515
:10AA30008091023690910336A0910436B09105368C
:10AA40008093AB359093AC35A093AD35B093AE35D4
:10AA500080E008952CEA35EC47E257E360915D36DB
:10AA600070915E3680915F36909160360E946DD60F
:10AA70001816B4F48091023690910336A0910436F2
:10AA8000B0910536BC01CD019F772CEA35EC47E249
:10AA900057E30E946AD487FF03C01092B83503C001
:10AAA00081E08093B83580E008958093B835809137
:10AAB000023690910336A0910436B091053680930A
:10AAC000B4359093B535A093B635B093B73580E0E3
:10AAD0000895BC018DEE90E20C94746281E0809345
:10AAE000E434089581E08093E534089581E0809313
:10AAF000E63408951F93CF93DF93CDB7DEB7689701
:10AB0000CDBFDEBF0E9418978130C9F10E9408D1E5
:10AB10000E940CC80E94168380E00E9408AC10E0DE
:10AB2000812F0E94F096AB01BC01812F0E9418502A
:10AB30001F5F1630A9F780E090E0A0E4B0E48983BD
:10AB40009A83AB83BC831D821E821F82188619865E
:10AB50001A861B861C861D861E861F86188A198AE1
:10AB60001A8A1B8A1C8A1D8A1E8A1F8A188EBE0199
:10AB70006F5F7F4FCB010E94655480E001C08AE681
:10AB80006896CDBFDEBFDF91CF911F910895809170
:10AB9000E4348130A9F42091BF34213079F48091DC
:10ABA000C03481110BC082E08093BF3485EB98E5FF
:10ABB0008093EB349093EC342093C0341092E434BF
:10ABC0008091E534813091F48091BF34882331F055
:10ABD000823061F49091C034943051F40E941897FF
:10ABE000811104C01092E5340E947A559091C034CE
:10ABF0008091E6348130C1F42091E534211114C0F4
:10AC00009150933088F01092E63495E09093C034E0
:10AC10009093BD349091BE34911104C08093BE34A2
:10AC20000E94F3AB0E948A9F80E0089585E08093A4
:10AC3000BD348091BE34811105C081E08093BE3463
:10AC40000C94F3AB0895CF93DF93CDB7DEB768973D
:10AC5000CDBFDEBF8091BE34882311F180E090E04B
:10AC6000A0E4B0E489839A83AB83BC831D821E82F7
:10AC70001F82188619861A861B861C861D861E86CC
:10AC80001F86188A198A1A8A1B8A1C8A1D8A1E8A9C
:10AC90001F8A188EBE016F5F7F4FCB010E946554E3
:10ACA0006896CDBFDEBFDF91CF910895CF93DF933C
:10ACB000CDB7DEB76897CDBFDEBF80E090E0A0E4FF
:10ACC000B0E489839A83AB83BC831D821E821F827A
:10ACD000188619861A861B861C861D861E861F8668
:10ACE000188A198A1A8A1B8A1C8A1D8A1E8A1F8A38
:10ACF000188EAE014F5F5F4FBA0185E694E50E9462
:10AD000059836896CDBFDEBFDF91CF910895CF9371
:10AD1000DF93CDB7DEB76897CDBFDEBF80E090E0B0
:10AD2000A0E8B0E489839A83AB83BC831D821E8232
:10AD30001F82188619861A861B861C861D861E860B
:10AD40001F86188A198A1A8A1B8A1C8A1D8A1E8ADB
:10AD50001F8A188EAE014F5F5F4FBA0185E694E5FA
:10AD60000E9459836896CDBFDEBFDF91CF910895D1
:10AD7000CF93DF93CDB7DEB72797CDBFDEBF97E088
:10AD8000EFEDF0E2DE01119601900D929A95E1F758
:10AD9000873050F4E1E0F0E0EC0FFD1FE80FF11D0B
:10ADA00087FDFA95808101C080E22796CDBFDEBF86
:10ADB000DF91CF9108950F931F93CF93DF93EC0111
:10ADC000042F10E020E030E009871A872B873C87AA
:10ADD00082E08F8350E0440F551F640F751FFB0105
:10ADE000659174914FE450E086E69FE30E94A4E0F1
:10ADF000BC01CE01DF91CF911F910F910C9416628F
:10AE0000CF93DF93EC010E94364A482F60E573E14F
:10AE1000CE01DF91CF910C94DB564091BD3461E1BE
:10AE200073E10C94DB564091BE3468EE72E10C94F1
:10AE3000DB564091BF3464ED72E10C94DB564091D7
:10AE4000C03466EA72E10C94DB564091C13469E883
:10AE500072E10C94DB56E091EB34F091EC34E55B5D
:10AE6000FF4F408163EB73E10C94DB56E091EB34D0
:10AE7000F091EC34E45BFF4F40816FEB71E10C9497
:10AE8000DB56E091EB34F091EC34448165E271E102
:10AE90000C94DB56E091EB34F091EC34E65BFF4F21
:10AEA000408162EF70E10C94DB56E091EB34F0915D
:10AEB000EC34E25BFF4F408168EA70E10C94DB56B2
:10AEC000E091EB34F091EC34E15BFF4F408167E6B9
:10AED00070E10C94DB56E091EB34F091EC34E75BDD
:10AEE000FF4F408168EF7FE00C94DB56E091EB343C
:10AEF000F091EC34EF5AFF4F408150E060E070E099
:10AF0000FC01418752876387748722E0278380E0B2
:10AF10000895E091EB34F091EC34408151816281ED
:10AF20007381FC01418752876387748722E02783FE
:10AF300080E00895CF93DF93EC018091BF348111BD
:10AF400005C019861A861B861C8614C00E94E796C7
:10AF500069877A878B879C872091005921110AC0C5
:10AF600025E832E441E25DE30E940FD769877A87E2
:10AF70008B879C878C819D81FC01EE0FFF1FE80F62
:10AF8000F91FEE0FFF1FEE0FFF1FEE0FFF1FE25620
:10AF9000FA4E85919491888784E08F8380E0DF91D9
:10AFA000CF910895CF93DF93EC012091EB34309152
:10AFB000EC34F901FD96608171818281938169870A
:10AFC0007A878B879C873E96208121110AC025E8CD
:10AFD00032E441E25DE30E940FD769877A878B876D
:10AFE0009C878C819D81FC01EE0FFF1FE80FF91FEC
:10AFF000EE0FFF1FEE0FFF1FEE0FFF1FE256FA4E80
:10B0000085919491888784E08F8380E0DF91CF9150
:10B010000895CF93DF93EC018C819D810E941A48A3
:10B02000682F8091EB349091EC340E94B74B698784
:10B030007A878B879C878C819D81FC01EE0FFF1F97
:10B04000E80FF91FEE0FFF1FEE0FFF1FEE0FFF1FA0
:10B05000E256FA4E85919491888784E08F8380E050
:10B06000DF91CF910895CF93DF93EC018C819D8187
:10B070000E941A482091EB343091EC342D5E344319
:10B0800069F4E82FF0E0EE0FFF1FEE0FFF1FE95B02
:10B09000FA4C608171818281938102C00E94F09696
:10B0A00069877A878B879C878C819D81FC01EE0F55
:10B0B000FF1FE80FF91FEE0FFF1FEE0FFF1FEE0F30
:10B0C000FF1FE256FA4E85919491888784E08F8322
:10B0D00080E0DF91CF910895CF93DF93EC018C81D5
:10B0E0009D810E941A48E091EB34F091EC3494E099
:10B0F000899FE00DF11D1124458D568D678D70A13E
:10B1000049875A876B877C878C819D81FC01EE0F74
:10B11000FF1FE80FF91FEE0FFF1FEE0FFF1FEE0FCF
:10B12000FF1FE256FA4E85919491888784E08F83C1
:10B1300080E0DF91CF910895CF93DF93EC010E94DF
:10B14000405D49856FED73E1CE01DF91CF910C94A5
:10B15000DB56CF93DF93EC018C819D810E941A48CE
:10B16000833054F48F3F91F407C0CE010E94195EE2
:10B1700080E016C08DE614C049855A856B857C85B4
:10B180004430510561057105A8F7EFCF49855A850F
:10B190006B857C85433051056105710558F7E5CF16
:10B1A000DF91CF91089595E3899FF0011124E15734
:10B1B000FC4C60817181828193810895CF92DF92EE
:10B1C000EF92FF92CF93DF936A017B0125E3829F89
:10B1D000C001112486549D4CFC01EB52FF4F40836B
:10B1E000518362837383EC01C352DF4F20E034E26A
:10B1F00044E759E4C701B6010E940FD79B01AC0197
:10B2000060E070E080E89FE30E9471D468837983F6
:10B210008A839B83DF91CF91FF90EF90DF90CF9057
:10B220000895CF92DF92EF92FF92CF93DF93EC01DC
:10B23000C984DA84EB84FC8420E034E244E759E4F6
:10B24000C701B6010E946DD6181664F420E034E2FE
:10B2500044E759E4C701B6010E9471D469877A872F
:10B260008B879C87CE010E943163C984DA84EB848A
:10B27000FC848C819D810E941A4825E3829FC00135
:10B28000112486549D4CFC01EB52FF4FC082D182A9
:10B29000E282F382EC01C352DF4F20E034E244E764
:10B2A00059E4C701B6010E940FD79B01AC0160E0D1
:10B2B00070E080E89FE30E9471D4688379838A8379
:10B2C0009B8380E0DF91CF91FF90EF90DF90CF9054
:10B2D0000895CF92DF92EF92FF92CF93DF93EC012C
:10B2E000C984DA84EB84FC8420E034E244E759E446
:10B2F000C701B6010E946DD6181664F420E034E24E
:10B3000044E759E4C701B6010E9471D469877A877E
:10B310008B879C87CE010E94316380E0DF91CF91C3
:10B32000FF90EF90DF90CF90089581E08093E53417
:10B3300080E00895FC0181859285A385B4850197FD
:10B34000A105B10511F40E94EB6A80E008956091B7
:10B35000E7347091E8348091E9349091EA340895AB
:10B360000E94F15E80E00E946E6D80E008950E9470
:10B37000F15E81E00E946E6D80E008950E94F15EB2
:10B3800082E00E946E6D80E008950E94F15E83E08D
:10B390000E946E6D80E00895CF93DF93EC01E09101
:10B3A000EB34F091EC34E55BFF4FE081F0E0EE0F21
:10B3B000FF1FEE5EFB4E659174914FE450E086E610
:10B3C0009FE30E94A4E0AC0161EE7FE0CE01DF913B
:10B3D000CF910C947CC0CF93DF93EC01E091EB34E0
:10B3E000F091EC34E55BFF4FE081F0E0EE0FFF1FE2
:10B3F000EE5EFB4E659174914FE450E086E69FE36C
:10B400000E94A4E0AC0169EC7FE0CE01DF91CF9116
:10B410000C947CC0CF93DF93EC0181EF90E20E940B
:10B4200005E2CE010E94CC59CE010E94EB5966EB99
:10B430007FE0CE010E94A8C06DE97FE0CE010E94AE
:10B44000F2BF64E87FE0CE010E94F2BF6BE67FE0CE
:10B45000CE010E94F2BF62E57FE0CE010E94F2BF02
:10B4600069E37FE0CE010E94F2BF60E27FE0CE019F
:10B470000E94F2BF67E07FE0CE010E94F2BF6EEE55
:10B480007EE0CE010E94F2BF65ED7EE0CE010E941B
:10B49000F2BF6CEB7EE0CE010E94F2BF63EA7EE079
:10B4A000CE010E94F2BF6AE87EE0CE010E94F2BFA8
:10B4B00061E77EE0CE010E94F2BF68E57EE0CE014A
:10B4C0000E9420C080E0DF91CF91089566EB7FE07D
:10B4D0000C94A8C06DE97FE00C94F2BF64E87FE0B3
:10B4E0000C94F2BF6BE67FE00C94F2BF62E57FE064
:10B4F0000C94F2BF69E37FE00C94F2BF60E27FE05E
:10B500000C94F2BF67E07FE00C94F2BF6EEE7EE039
:10B510000C94F2BF65ED7EE00C94F2BF6CEB7EE024
:10B520000C94F2BF63EA7EE00C94F2BF6AE87EE01E
:10B530000C94F2BF61E77EE00C94F2BF68E57EE018
:10B540000C9420C06CED7DE00C9420C06BEA7DE093
:10B550000C9420C066E77DE00C9420C06BE37DE096
:10B560000C9420C067E07DE00C9420C0CF93DF9363
:10B57000EC01E091EB34F091EC34E55BFF4FE081BE
:10B58000F0E0EE0FFF1FEE5EFB4E659174914FE40D
:10B5900050E086E69FE30E94A4E0AC0163EE7CE00D
:10B5A000CE01DF91CF910C947CC0CF93DF93EC015F
:10B5B000E091EB34F091EC34E55BFF4FE081F0E09B
:10B5C000EE0FFF1FEE5EFB4E659174914FE450E06D
:10B5D00086E69FE30E94A4E0AC0162EC7CE0CE0131
:10B5E000DF91CF910C947CC065EA7CE00C94A8C0FC
:10B5F000CF93DF93EC01E091EB34F091EC34E55B19
:10B60000FF4FE081F0E0EE0FFF1FEE5EFB4E659115
:10B6100074914FE450E086E69FE30E94A4E0AC0101
:10B6200066E87CE0CE01DF91CF910C947CC00F9353
:10B630001F93CF93DF93CDB7DEB7C058D109CDBFED
:10B64000DEBF8C01DC011996EC91F0E0EE0FFF1FDC
:10B65000E152FC4E659174914FE450E086E69FE321
:10B660000E94A4E09801235F3F4F9F938F93F801BE
:10B6700081851F928F933F932F930F5E1F4F1F93D0
:10B680000F933F932F938AE69CE09F938F938E01B5
:10B690000F5F1F4F1F930F930E945BE2C8010E9430
:10B6A000CDBFCDBFDEBFC058DF4FCDBFDEBFDF9106
:10B6B000CF911F910F91089562E47CE00C948C4827
:10B6C0006AE17CE00C948C4868EF7BE00C948C4839
:10B6D00066ED7BE00C948C4864EA7BE00C948C482B
:10B6E00063E77BE00C948C486AE37BE00C948C4825
:10B6F0006AE17BE00C948C4868ED7AE00C945A483F
:10B7000066E97AE00C945A486FE67AE00C948C482B
:10B7100069E47AE00C948C4868E27AE00C948C48F6
:10B7200068E07AE00C948C486BEE79E00C94F04879
:10B730006CEC79E00C94F048BC01675F7F4F20917E
:10B74000383542E45EE0FC01848195810C945749D0
:10B75000BC01675F7F4F21E048E25EE0FC0184812D
:10B7600095810C945749BC01675F7F4F21E04FE002
:10B770005EE0FC01848195810C9457490F931F93DF
:10B78000CF93DF93EC010C811D810E949E6408170A
:10B790001907C4F48C819D81FC01EE0FFF1FE80F97
:10B7A000F91FEE0FFF1FEE0FFF1FEE0FFF1FED55EE
:10B7B000FA4E25913491CE01F901DF91CF911F917D
:10B7C0000F91199485E1DF91CF911F910F91089509
:10B7D0000F931F93CF93DF93EC010C811D810E9487
:10B7E0009E6408171907C4F48C819D81FC01EE0F3B
:10B7F000FF1FE80FF91FEE0FFF1FEE0FFF1FEE0FE9
:10B80000FF1FEF55FA4E25913491CE01F901DF91DA
:10B81000CF911F910F91199485E1DF91CF911F91E5
:10B820000F9108950F931F93CF93DF93EC010C8139
:10B830001D810E949E6408171907C4F48C819D81A4
:10B84000FC01EE0FFF1FE80FF91FEE0FFF1FEE0FB9
:10B85000FF1FEE0FFF1FE156FA4E25913491CE01E6
:10B86000F901DF91CF911F910F911994DF91CF9141
:10B870001F910F910895CF93DF93EC018C819D81EF
:10B880000E94B1648823C9F08C819D81FC01EE0F78
:10B89000FF1FE80FF91FEE0FFF1FEE0FFF1FEE0F48
:10B8A000FF1FE356FA4EE491E1FF05C0CE01DF91A0
:10B8B000CF910C94718180E001C085E1DF91CF913F
:10B8C0000895AF92BF92CF92DF92EF92FF920F93C3
:10B8D0001F93CF93DF93EC0181E00E94C74E1C823F
:10B8E0001D8280E090E07E0121E1E20EF11C54E037
:10B8F000A52E62E0B62E51C00C811D816801CC0CD2
:10B90000DD1C9601200F311F220F331F220F331F22
:10B91000220F331F23563A4EF901849180FF38C01D
:10B92000F601E00FF11FEE0FFF1FEE0FFF1FEE0FEE
:10B93000FF1FE955FA4E659175918591949169873C
:10B940007A878B879C87F901249124FD08C00E9487
:10B95000DED469877A878B879C87BF8201C0AF82DC
:10B96000B601600F711F660F771F660F771F660F96
:10B97000771F69567A4E45E050E0C7010E94A4E067
:10B98000CE010E94BE5BCE010E943B5C0C811D81FA
:10B990000F5F1F4F0C831D83C8010E94A16481119A
:10B9A000ABCF81E00E948FA8DF91CF911F910F91C3
:10B9B000FF90EF90DF90CF90BF90AF900C9477A85E
:10B9C000CF92DF92EF92FF92CF93DF93EC01C98485
:10B9D000DA84EB84FC8481E0C816D104E104F1042C
:10B9E00049F0CE01DF91CF91FF90EF90DF90CF90A3
:10B9F0000C94037ACE010E94615C82E08F83C98639
:10BA0000DA86EB86FC8680E0DF91CF91FF90EF90A5
:10BA1000DF90CF90089580912C3C90912D3C8F3EEB
:10BA2000924111F08AE5089580916E3C90916F3CAF
:10BA30008F3E9241B9F78091FE369091FF368F3E4E
:10BA4000924181F78091243A9091253A8F3E92411C
:10BA500049F78091263A9091273A8F3E924111F70B
:10BA600080912A3C90912B3C8F3E9241D9F6809157
:10BA7000B53F8111D7CF0895FC01178289E608955B
:10BA8000CF93DF93DC0114968D919C911597FC0167
:10BA9000EE0FFF1FE80FF91FEE0FFF1FEE0FFF1F46
:10BAA000EE0FFF1FEB55FA4EC591D491488150E03F
:10BAB00060E070E019964D935D936D937C931C97B5
:10BAC00082E017968C9380E0DF91CF910895CF9319
:10BAD000DF93DC0114968D919C911597FC01EE0F7C
:10BAE000FF1FE80FF91FEE0FFF1FEE0FFF1FEE0FF6
:10BAF000FF1FEB55FA4EC591D4914881598160E002
:10BB000070E019964D935D936D937C931C9782E042
:10BB100017968C9380E0DF91CF910895CF93DF93B8
:10BB2000DC0114968D919C911597FC01EE0FFF1F7F
:10BB3000E80FF91FEE0FFF1FEE0FFF1FEE0FFF1FA5
:10BB4000EB55FA4EC591D491488159816A817B8128
:10BB500019964D935D936D937C931C9782E0179695
:10BB60008C9380E0DF91CF910895CF93DF93DC0138
:10BB700014968D919C911597FC01EE0FFF1FE80F15
:10BB8000F91FEE0FFF1FEE0FFF1FEE0FFF1FEB550C
:10BB9000FA4EC591D491488159816A817B81199669
:10BBA0004D935D936D937C931C9783E017968C93D4
:10BBB00080E0DF91CF910895CF93DF93DC0114965D
:10BBC0008D919C911597FC01EE0FFF1FE80FF91F57
:10BBD000EE0FFF1FEE0FFF1FEE0FFF1FEB55FA4E8C
:10BBE000C591D491488159816A817B8119964D9381
:10BBF0005D936D937C931C97FC01EE0FFF1FE80F84
:10BC0000F91FEE0FFF1FEE0FFF1FEE0FFF1FE25693
:10BC1000FA4E8591949118968C93189784E0179614
:10BC20008C9380E0DF91CF91089588E6089580E0BD
:10BC30000895FC0124813581F901EE0FFF1FE20F09
:10BC4000F31FEE0FFF1FEE0FFF1FEE0FFF1FEB5551
:10BC5000FA4EA591B491FC0181858C9380E0089502
:10BC6000FC0124813581F901EE0FFF1FE20FF31F64
:10BC7000EE0FFF1FEE0FFF1FEE0FFF1FEB55FA4EEB
:10BC8000A591B491FC01818592858D939C9380E070
:10BC90000895CF93DF93FC0124813581F901EE0FE4
:10BCA000FF1FE20FF31FEE0FFF1FEE0FFF1FEE0F40
:10BCB000FF1FEB55FA4EC591D491FC018185928509
:10BCC000A385B48588839983AA83BB8380E0DF91B1
:10BCD000CF910895FC01418552856385748542307A
:10BCE000510561057105A0F484819581FC01EE0F79
:10BCF000FF1FE80FF91FEE0FFF1FEE0FFF1FEE0FE4
:10BD0000FF1FEB55FA4EA591B4914C9380E0089536
:10BD10008EE60895FC014185528563857485433024
:10BD2000510561057105A0F484819581FC01EE0F38
:10BD3000FF1FE80FF91FEE0FFF1FEE0FFF1FEE0FA3
:10BD4000FF1FEB55FA4EA591B4914C9380E00895F6
:10BD50008EE60895FC0141855285638574854430E3
:10BD6000510561057105A0F484819581FC01EE0FF8
:10BD7000FF1FE80FF91FEE0FFF1FEE0FFF1FEE0F63
:10BD8000FF1FEB55FA4EA591B4914C9380E00895B6
:10BD90008EE60895CF93DF93DC0114968D919C91EC
:10BDA0001597FC01EE0FFF1FE80FF91FEE0FFF1FA5
:10BDB000EE0FFF1FEE0FFF1FEB55FA4EC591D4910A
:10BDC00019964D915D916D917C911C974883598393
:10BDD0006A837B8383E017968C9380E0DF91CF9119
:10BDE0000895CF93DF93DC0114968D919C91159764
:10BDF000FC01EE0FFF1FE80FF91FEE0FFF1FEE0F04
:10BE0000FF1FEE0FFF1FEB55FA4EC591D491199607
:10BE10004D915D916D917C911C97488359836A8304
:10BE20007B83FC01EE0FFF1FE80FF91FEE0FFF1FD2
:10BE3000EE0FFF1FEE0FFF1FE256FA4E8591949111
:10BE400018968C93189784E017968C9380E0DF9176
:10BE5000CF9108951F93CF93DF93EC018091843CA1
:10BE60008823D1F01DE10A80DB81C02D209711F4D9
:10BE700080E013C08F818F3FD9F3811104C0CE01C0
:10BE80000E94E85B06C0CE010E94BE5BCE010E940C
:10BE90003B5C115041F7ECCF85E6DF91CF911F91CC
:10BEA0000895CF93DF93EC01BC018FEF90E20E94E5
:10BEB000DDE0892B41F0BE0182E091E20E94DDE0ED
:10BEC00021E0892B09F420E0822FDF91CF910895A2
:10BED00041E020910037309101372817390709F0E8
:10BEE00040E0842F08950F931F93CF93DF93CDB736
:10BEF000DEB72997CDBFDEBF8B0144E050E0BC0127
:10BF0000CE0101960E94FDE046E050E0B801CE016E
:10BF100001960E94EDE00E949E64181619060CF02E
:10BF20003FC07981AA81BB811C810D8127E935E160
:10BF300040E050E0F9016491671327C03196E49125
:10BF4000E11103C0A11121C029C0EA131EC0F901EB
:10BF50003296E491E11103C0B11117C01FC0EB1379
:10BF600014C0F9013396E491E11103C011110DC021
:10BF700015C0E1130AC0F9013496E491E11103C040
:10BF8000011103C00BC0E01749F04F5F5F4F285EFF
:10BF90003F4F4817590709F0CDCF02C0CA0102C070
:10BFA0008FEF9FEF2996CDBFDEBFDF91CF911F911D
:10BFB0000F910895CF93DF93FC012189222371F122
:10BFC000EC016196BE0186E091E20E94DDE0892BE2
:10BFD00039F1BE018FEF90E20E94DDE0892B11F173
:10BFE000BE0189E091E20E94DDE0892BD9F0BE011B
:10BFF0008DEE90E20E94DDE0892BB1F0BE018CE075
:10C0000091E20E94DDE0892B79F0BE0188EE91E299
:10C010000E94DDE0892B51F485E009C080E007C073
:10C0200082E005C083E003C084E001C081E0DF91CD
:10C03000CF910895FC018FEF8783148215821186BA
:10C040001286138614861086118A1586178A108E1A
:10C05000A081B181109711F416820DC017968C91B2
:10C060001797873029F416968C918F5F868303C0CB
:10C0700016968C918683CF010895EF92FF920F93CD
:10C080001F93CF93DF93EC010C811D810E949E646E
:10C09000081719070CF06FC00C811D81CE010E949A
:10C0A0001A600C831D837E0181E1E80EF11CB8014A
:10C0B000660F771F600F711F660F771F660F771F60
:10C0C000660F771F69567A4EC7010E9485E08E0180
:10C0D000035F1F4F2C813D81B901660F771F620FEF
:10C0E000731F660F771F660F771F660F771F6D56DA
:10C0F0007A4EC8010E9485E08D85882311F18C81DC
:10C100009D81FC01EE0FFF1FE80FF91FEE0FFF1FCF
:10C11000EE0FFF1FEE0FFF1FE356FA4EE491E2FF12
:10C1200002C01D8610C0F80101900020E9F7BF0190
:10C13000601B710B605F7F4F6C0F7D1FC7010E94FA
:10C14000E6E08C819D81FC01EE0FFF1FE80FF91FD7
:10C15000EE0FFF1FEE0FFF1FEE0FFF1FEF55FA4E02
:10C1600025913491CE01F901DF91CF911F910F916B
:10C17000FF90EF901994DF91CF911F910F91FF9055
:10C18000EF9008958F929F92AF92BF92CF92DF92DD
:10C19000EF92FF920F931F93CF93DF9300D01F92E4
:10C1A000CDB7DEB76C015C0181E1A80EB11C87E060
:10C1B000F601878363E9E62E65E1F62E00E010E0E4
:10C1C0001DC0B701CE0101960E9485E0BE016F5FE0
:10C1D0007F4FC5010E94DDE0892B59F44601F9E14A
:10C1E0008F0E911CF601058F168FC4010E943D60D1
:10C1F00064010F5F1F4FF8E1EF0EF11CC8010E94B0
:10C20000A1648111DECF2496CDBFDEBFDF91CF9137
:10C210001F910F91FF90EF90DF90CF90BF90AF9064
:10C220009F908F900895CF93DF931092283A1092A9
:10C23000293A21E0FC013081311101C020E0ABEE50
:10C24000B6E3E4E0F7E33FEFA083B18379965B9632
:10C25000ED93FC935C975D961D921C925E97EF01A7
:10C260006397288322961882219738832A9618820A
:10C2700059964AE3E432F40739F710920D3A1092D6
:10C280000E3A1092043710920537FC0120812223C8
:10C2900069F010920A3727E020930B37BC0185E143
:10C2A00097E30E94E6E08DE197E302C084E097E324
:10C2B000DF91CF910895EF92FF920F931F93CF9349
:10C2C000DF938AE091E20E941361EC018FEE92E12C
:10C2D00080932C3C90932D3C80936E3C90936F3CCC
:10C2E0008093FE369093FF368093243A9093253ABC
:10C2F0008093263A9093273A80932A3C90932B3C44
:10C3000081E00E94C74E1C821D82CE010E9448819E
:10C310002091763C3091773C4091783C5091793C2B
:10C3200069857A858B859C850E94C1D29F772CEA8E
:10C3300035EC47E257E30E946DD6181624F4CE017F
:10C340000E94615C58C00E947CA81C821D8280E013
:10C3500090E08E010F5E1F4F42E0E42E54E0F52E78
:10C3600044C06C817D81CB01880F991FFC01E60FD1
:10C37000F71FEE0FFF1FEE0FFF1FEE0FFF1FE3561D
:10C38000FA4EE491E0FF2CC0680F791F660F771F0B
:10C39000660F771F660F771F69567A4E45E050E0AB
:10C3A000C8010E94A4E0CE010E9448818C819D8139
:10C3B000FC01EE0FFF1FE80FF91FEE0FFF1FEE0F3E
:10C3C000FF1FEE0FFF1FE356FA4EE491E4FF02C099
:10C3D000FF8201C0EF82CE010E94BE5B6C817D8135
:10C3E0006F5F7F4F6C837D83CB010E94A1648111BD
:10C3F000B8CF0E948FA860E171E287E493E20E94C7
:10C40000735F809300379093013764E171E287E4B2
:10C4100093E20E94735F8093023790930337DF911A
:10C42000CF911F910F91FF90EF900895EF92FF929F
:10C430000F931F93CF93DF938C012091283A309173
:10C44000293AEB0109900020E9F72197C61BD70B89
:10C45000AE01420F531F41305240D8F4F901E65D5E
:10C46000F54C7F01AE014F5F5F4FCF010E94BEE0F0
:10C470004091283A5091293A4F5F5F4F4C0F5D1F12
:10C480004093283A5093293AF801E78AF08E80E0E9
:10C4900001C08DE0DF91CF911F910F91FF90EF9040
:10C4A0000895CF93DF932EE1CDE1D7E33F813F3F66
:10C4B00059F00A80DB81C02D209719F480E090E0CC
:10C4C00010C0215099F7FACFBC0187E493E20E9493
:10C4D000735F8C839D83019689F3CE010E943D603A
:10C4E000CE01DF91CF910895EF92FF920F931F93AA
:10C4F000CF93DF938B012EE1CDE1D7E33F813F3F27
:10C5000059F00A80DB81C02D209719F480E090E07B
:10C510001DC0215099F7FACF7E0121E1E20EF11CF6
:10C5200045E050E0BC01C7010E94FDE0B801CE012A
:10C530000E9416628111EACFB70187E493E20E945C
:10C54000735F8C839D8385E08F83CE01DF91CF91D4
:10C550001F910F91FF90EF9008952091843C21301E
:10C5600021F42091623F213029F4BC018DEE90E24C
:10C570000C94746280E090E008959091843C913036
:10C5800019F4642F0C94F57F0C94C5BFCF93DF93FF
:10C59000EC018091773281110BC00E9400D1482FAD
:10C5A00050E060E070E049875A876B877C870AC05B
:10C5B0000E940EC8482F50E060E070E049875A871B
:10C5C0006B877C8782E08F8380E0DF91CF91089535
:10C5D0000F931F93CF93DF93CDB7DEB7C058D10928
:10C5E000CDBFDEBFDC011996EC918FEF8E0F863048
:10C5F00030F088E491E20E94AD628EE629C0E093BB
:10C60000723281E080937332F0E0EE0FFF1FE25A46
:10C61000FA4E659174914FE450E086E69FE30E94E4
:10C62000A4E09F938F9385E294E19F938F938E0173
:10C630000F5F1F4F1F930F930E945BE2C8010E9480
:10C64000AD620F900F900F900F900F900F9080E0C1
:10C65000C058DF4FCDBFDEBFDF91CF911F910F914B
:10C6600008950F931F93CF93DF93EC018DEE94E326
:10C670000E94924A882329F009851A858B859C851A
:10C6800011C023E333E34BEC51E469857A858B8554
:10C690009C850E940FD78B01AB01BC0149875A874B
:10C6A0006B877C872C813D81F901EE0FFF1FE20F24
:10C6B000F31FEE0FFF1FEE0FFF1FEE0FFF1FEB55D7
:10C6C000FA4EA591B491A801BC014D935D936D9371
:10C6D0007C931397F901EE0FFF1FE20FF31FEE0F8C
:10C6E000FF1FEE0FFF1FEE0FFF1FE256FA4E859160
:10C6F0009491888784E08F8380E0DF91CF911F91B0
:10C700000F9108956FE275E10C94A8C06BE075E19C
:10C710000C94A8C06FEC74E10C94A8C06BE974E1B0
:10C720000C94A8C06EE474E10C94A8C01F93CF933E
:10C73000DF93EC0110E08881882311F18AE091E217
:10C740000E94136145E050E0BE018EE297E30E9433
:10C75000FDE06EE277E387E493E20E94735F8093EB
:10C760002137909322378DE197E30E943D6042E0AC
:10C7700063E080E00E94BD621F5F26961D31D9F6FE
:10C7800084E0DF91CF911F910895CF93DF93CDB7D0
:10C79000DEB7EC97CDBFDEBF8CE3E8E1F0E2DE016F
:10C7A000119601900D928A95E1F7CE0101960E94B3
:10C7B0009663EC96CDBFDEBFDF91CF910895CF9306
:10C7C000DF93CDB7DEB7AA97CDBFDEBF8AE2E4E53F
:10C7D000F0E2DE01119601900D928A95E1F7CE010B
:10C7E00001960E949663AA96CDBFDEBFDF91CF91DE
:10C7F0000895CF93DF93CDB7DEB76E97CDBFDEBF81
:10C800008EE1EEE7F0E2DE01119601900D928A953D
:10C81000E1F7CE0101960E9496636E96CDBFDEBF12
:10C82000DF91CF910895CF93DF93EC0143E759E770
:10C8300063E770E0498B5A8B6B8B7C8B0E94C260E4
:10C8400042E063E080E00E94BD62CE010E94F96395
:10C85000CE010E94DF6320E731E340E0298B3A8B71
:10C860004B8BCE010E94C26042E063E080E00E94F8
:10C87000BD62CE01DF91CF910C94C563FC0181852F
:10C880009285A385B48583309105A105B105A0F4F7
:10C8900080937632892B8A2B8B2B39F064E070E001
:10C8A00080E00E94E7C580E0089568E070E080E0E5
:10C8B0000E94E7C580E008958EE60895FC01818519
:10C8C0009285A385B48582309105A105B105A0F4B8
:10C8D00080937532892B8A2B8B2B39F060E170E0C5
:10C8E00080E00E94E7C580E0089560E270E080E0AB
:10C8F0000E94E7C580E008958EE60895FC018185D9
:10C900009285A385B48582309105A105B105A0F477
:10C9100080937432892B8A2B8B2B39F060E470E082
:10C9200080E00E94E7C580E0089560E870E080E064
:10C930000E94E7C580E008958EE608958EE891E0B4
:10C94000089521E08534914008F020E0822F089579
:10C950009C012156314081E02932310508F080E008
:10C96000089521E08236914008F020E0822F08955A
:10C97000CF92DF92EF92FF92CF93DF93EC01C984C5
:10C98000DA84EB84FC84A7019601C701B6010E94FA
:10C9900030D881113CC0E894F7F82FEF3FEF4FE714
:10C9A0005FE7C701B6010E9430D881110AC02FEF9E
:10C9B0003FEF4FE75FE7C701B6010E946AD4181640
:10C9C00034F18C819D81FC01EE0FFF1FE80FF91FF0
:10C9D000EE0FFF1FEE0FFF1FEE0FFF1FE356FA4E85
:10C9E000E491E3FF14C08DEE94E30E94924A81111A
:10C9F0000EC025E832E441E25DE369857A858B85E6
:10CA00009C850E940FD769877A878B879C87DF91E7
:10CA1000CF91FF90EF90DF90CF9008958091733287
:10CA2000882349F0109273326091723280E00E9444
:10CA3000EFC580E0089583E00895CF93DF93E09100
:10CA4000A63CF091A73C04C0E093A63CF093A73C21
:10CA5000EF018191982F9D7F9032B1F38930A1F33E
:10CA60004FE750E0BE018AEA9EE30E94FDE010928B
:10CA7000A23C1092A33C1092A43C1092A53C688169
:10CA8000611105C08091843C81116FC039C0613251
:10CA900021F4DF91CF910C946E55653221F4DF9132
:10CAA000CF910C9472556E3721F4DF91CF910C9495
:10CAB00076556F3379F4FE0101900020E9F7319744
:10CAC000EC1BFD0B329780F02196C093A63CD093CF
:10CAD000A73C4BC06B3741F481E08093843CCE018E
:10CAE000DF91CF910C942A7D70E088E791E20E945B
:10CAF000D2E0892B59F01092843CCE010E94B7BD40
:10CB00006AEA7EE3DF91CF910C941FBF8091843C51
:10CB1000811109C0CE010E943A706AEA7EE3DF917A
:10CB2000CF910C941FBF8AE091E20E941361EC0147
:10CB300027E633E640E0298B3A8B4B8B6091A63C8D
:10CB40007091A73C0E94166285E08F838091A63C7D
:10CB50009091A73C0E943A7042E060E00E94BD6262
:10CB600080E0DF91CF910C94D1AADF91CF9108950D
:10CB7000FF920F931F93CF93DF931F921F92CDB716
:10CB8000DEB7F82EE0E7FCE32CEB32E0DF01C90171
:10CB90001D920197E9F72FEE32E120833183209334
:10CBA0002A3F30932B3F0DEC1CE22CED33E4009335
:10CBB000763C1093773C2093783C3093793C0CEE94
:10CBC00011E528E73FE300937A3C10937B3C2093E8
:10CBD0007C3C30937D3C81E080937E3C83E080937D
:10CBE000853C8F2D4A8369830E94FFC56981862F0A
:10CBF0000E940AC64A81842F0E9415C6F0927132A3
:10CC0000F0926F320F900F90DF91CF911F910F91A3
:10CC1000FF900895CF93DF931F921F92CDB7DEB799
:10CC200080E6F82E01E010E00E94C1788230E1F346
:10CC30000E94C8788230C1F30E94714A863009F0A0
:10CC4000D9C00E94E2C380908B3C90908C3CA09015
:10CC50008D3CB0908E3C86169706A806B90620F744
:10CC60000E94E2C36C597F4F8F4F9F4F60938B3C64
:10CC700070938C3C80938D3C90938E3C0E943778CF
:10CC8000D3CF0E949DBC882329F08CEC0E94B34E28
:10CC9000823051F20E94C755823031F20E94E49DE9
:10CCA000823011F20E940B5D8093B63F81112EC03D
:10CCB0008091703C9091713C8F3E924109F0AAC0E6
:10CCC00080912A3F90912B3F8F3E924109F0A2C064
:10CCD00097C00E94DE818093B63F811117C00E94E9
:10CCE00006B38093B63F811111C00E9405708093F6
:10CCF000B63F81110BC00E940EC58093B63F8111D3
:10CD000005C00E94FEB3823031F48ECF0E94B34E34
:10CD10008230B9F789CF0E9403AB823009F484CF07
:10CD20000E9455AC823009F47FCF0E9411AD823051
:10CD300009F47ACF09831A8368EA7CE3CE0101966D
:10CD40000E9424C68093A63C9093A73C8F3F2FEF70
:10CD5000920739F48DE00E949C4E823009F464CF32
:10CD600004C0892B11F00E941D650E94438C823003
:10CD700009F45ACF0E943A6B823009F455CF0E94D1
:10CD8000F96D823009F450CF0E94E06F823009F4CF
:10CD900049CF0E94404C823009F444CF0E949382D4
:10CDA0008430F0F53FCF8091853C843038F484E0C6
:10CDB0008093853C0E9472550E9481A883E090E098
:10CDC00089839A8368EA7CE3CE0101960E9424C697
:10CDD0008093A63C9093A73C8F3F2FEF920721F4BE
:10CDE0008DE00E949C4E1ECF892B09F41BCF0E9420
:10CDF0001D6518CF0E94714A823009F44BCF41CF94
:10CE00001092B63F0E946E4E8093B63F882309F47D
:10CE100060CF7CCFF092B63F80E60E94B34E78CFD1
:10CE20008091E4299091E5290E9474CF682F70E0E9
:10CE300080E090E00E940CD520E030E048E451E42E
:10CE40000E946DD687FFEECE0E940E65823009F0FB
:10CE5000AACFE8CE8091713280936F32089580938B
:10CE60006F320895809370320895CF93C82F8091C8
:10CE70009323882379F040E050E0BA018C2F0E9480
:10CE80001850EC2FFF27E7FDF095EE53FB4C81E0A7
:10CE900080830AC06C2F85EB98E50E94B74BAB01ED
:10CEA000BC018C2F0E9418504091BA235091BB2393
:10CEB0006091BC237091BD238C2F0E94DE5880E0CE
:10CEC00099E6809394239093952382E0CF910895DF
:10CED000CF92DF92EF92FF920F931F93CF93DF9346
:10CEE000CDB7DEB7E097CDBFDEBF98E17E01A9E107
:10CEF000EA0EF11CF701A92F1192AA95E9F7FE019C
:10CF000031966F0111929A95E9F7F60194E0890242
:10CF1000E00DF11D1124408F518F628F738F80E0DF
:10CF200090E0A0E8BFE380839183A283B383009362
:10CF30002A3510932B3520932C3530932D350E94B4
:10CF400016830E947655B601C7010E944053809314
:10CF5000B63F811101C082E0E096CDBFDEBFDF9118
:10CF6000CF911F910F91FF90EF90DF90CF90089598
:10CF70000F931F93E0918D23FF27E7FDF095E9566E
:10CF8000FD4C9381913099F400919E2310919F2341
:10CF90002091A0233091A1234091A6235091A72353
:10CFA0006091A8237091A9230E9468671DC0E09139
:10CFB0008E23FF27E7FDF095E956FD4C93819130D4
:10CFC00099F400919E2310919F232091A0233091EA
:10CFD000A1234091A6235091A7236091A82370918B
:10CFE000A92370580E9468678EEF97E68093942378
:10CFF0009093952382E01F910F9108950F931F93B3
:10D00000CF93C82F85E3C802F0011124ED56FC4CE4
:10D0100040815181628173818C2F0E94DE58009182
:10D020009E2310919F232091A0233091A123409112
:10D030009A2350919B2360919C2370919D238C2F68
:10D040000E9468678DE898E68093942390939523D7
:10D0500082E0CF911F910F9108950F931F9300913C
:10D060009E2310919F232091A0233091A1234091D2
:10D07000AA235091AB236091AC237091AD230E9401
:10D08000686785E397E6809394239093952382E0E5
:10D090001F910F9108950E9416838091B3230E94DF
:10D0A000814F8091B2230E94C74E8091B4230E9489
:10D0B000CB4E8091B5230E942C538091B623909142
:10D0C000B723A091B823B091B92380932A359093C8
:10D0D0002B35A0932C35B0932D3564E08DEE94E381
:10D0E0000E94AF4A0E9423561092BE3480E00895F9
:10D0F000CF93C82F4091BA235091BB236091BC239A
:10D100007091BD230E94DE588C2F0E944B6880E0F6
:10D110000E94D1AA80EFCF9108950F931F93E091C1
:10D120008D23FF27E7FDF095E956FD4C9381913063
:10D1300039F088E798E6809394239093952318C05C
:10D140000091A2231091A3232091A4233091A52321
:10D150004091A6235091A7236091A8237091A92301
:10D160000E9468678DE298E68093942390939523BC
:10D1700082E01F910F910895FF920F931F93CF9319
:10D18000DF93CDB7DEB7C058D109CDBFDEBFF82ED3
:10D190008AE091E20E9413618EEFF81205C08DE7DC
:10D1A00091E20E94AD6219C08F2D0E94B8561F9265
:10D1B0008F9323EE3AE33F932F938E010F5F1F4F20
:10D1C0001F930F930E945BE2C8010E94AD620F9013
:10D1D0000F900F900F900F900F9042E062E080EF61
:10D1E0000E94BD628F2D0E944B6880EFC058DF4FB8
:10D1F000CDBFDEBFDF91CF911F910F91FF900895BA
:10D200004F925F926F927F929F92AF92BF92CF9216
:10D21000DF92EF92FF920F931F93CF93DF938F3F95
:10D2200009F045C02CEA35EC47E257E3609125361A
:10D230007091263680912736909128360E946DD6BF
:10D2400018160CF469C12CEA35EC47E257E36091FB
:10D250001D3670911E3680911F36909120360E94A7
:10D260006DD618160CF45DC12CEA35EC47E257E395
:10D270006091213670912236809123369091243628
:10D280000E946DD618160CF455C12CEA35EC47E215
:10D2900057E36091293670912A3680912B36909110
:10D2A0002C360E946DD618160CF43FC171C1823025
:10D2B000A1F52CEA35EC47E257E360911D367091F9
:10D2C0001E3680911F36909120360E946DD618161A
:10D2D0000CF427C12CEA35EC47E257E36091213684
:10D2E0007091223680912336909124360E946DD61B
:10D2F00018160CF41FC12CEA35EC47E257E3609195
:10D30000293670912A3680912B3690912C360E94C6
:10D310006DD618160CF409C131C18823D9F28130B9
:10D3200051F32CC17E018DEEE80EF11CF7018081D6
:10D330009181A281B381BC01CD019F772CEA35ECAC
:10D3400047E257E30E946AD487FD46C06E01F1EFC1
:10D35000CF0ED11CF601408051806280738020E0A6
:10D3600030E0A901C301B2010E946AD487FD34C034
:10D37000FE01EF52FF4F208131814281538134976A
:10D3800060817181828193810E94C1D29B01AC0135
:10D390005F77C301B2010E94C2D22B013C019F778B
:10D3A0002CEA35EC47E257E30E946AD487FD14C0AB
:10D3B000AB2CAA0C8A2D0E9497BC80938B239924B6
:10D3C00093949A0C892D0E9497BC80938C23209172
:10D3D0008B23822780FD02C08B2DDBC0B0928A2375
:10D3E000F80180819181A281B381BF7780939E23D0
:10D3F00090939F23A093A023B093A123F701408192
:10D400005181628173817F774093A2235093A3233C
:10D410006093A4237093A52320FF2DC0A0928D2399
:10D4200090928E2377FA709477F8709440929A23B2
:10D4300050929B2360929C2370929D23F6018081E1
:10D440009181A281B3818093A6239093A723A09377
:10D45000A823B093A923CB50DF4F88819981AA815B
:10D46000BB818093AA239093AB23A093AC23B0936A
:10D47000AD238A2D2AC090928D23A0928E234092B4
:10D480009A2350929B2360929C2370929D23F601D5
:10D4900080819181A281B381B0588093A62390931B
:10D4A000A723A093A823B093A923CB50DF4F888153
:10D4B0009981AA81BB81B0588093AA239093AB2312
:10D4C000A093AC23B093AD23892D0E9497BC8D7F90
:10D4D000813039F080E099E68093942390939523EE
:10D4E00069C080918E230E9497BC811103C08FEF89
:10D4F00080938E238B2D0E94D3586093BA23709310
:10D50000BB238093BC239093BD2388EB97E6809345
:10D510009423909395234EC082E090E032E0B32EA6
:10D520000DC080E090E0B12C09C083E090E023E0E2
:10D53000B22E04C081E090E0BB24B394FC01EE5312
:10D54000FB4C108225E3289FE001299FD00D112478
:10D55000C654DD4C8E0107511F4FF8018081918127
:10D56000A281B381BC01CD019F772CEA35EC47E263
:10D5700057E30E946AD487FFD5CE2ECF81E08093F7
:10D58000C1348BE498E6809394239093952312C042
:10D590008EEFDF91CF911F910F91FF90EF90DF9071
:10D5A000CF90BF90AF909F907F906F905F904F9083
:10D5B0000C94BC6882E0DF91CF911F910F91FF9096
:10D5C000EF90DF90CF90BF90AF909F907F906F9043
:10D5D0005F904F900895CF93DF93CBEED4E3888193
:10D5E00099810E94924A8093B223888199810E94F6
:10D5F0008D4A8093B323888199810E949C4A8093AD
:10D60000B423888199810E94A14A8093B52388819F
:10D6100099810E94A84A6093B6237093B7238093A0
:10D62000B8239093B92381E00E94C74E81E00E9405
:10D63000CB4E80E00E94814F81E00E942C5381E01C
:10D64000809393238FEF80938A2380E099E68093E1
:10D6500094239093952383E08093BE341092C13439
:10D6600080E0DF91CF9108950E94EB6A109293239E
:10D6700080E008958091BE34833059F40E94A64A18
:10D68000813049F0E0919423F091952380918A2391
:10D69000199483E0089582E0089585E59BE68093E0
:10D6A000CF239093D02382E008952F923F924F9200
:10D6B0005F926F927F928F929F92AF92BF92CF9222
:10D6C000DF92EF92FF920F931F93CF93DF93CDB72B
:10D6D000DEB7CA54D109CDBFDEBF98E19E01275EF7
:10D6E0003F4F29AB3AABD901E92F1D92EA95E9F7F3
:10D6F000285131091901D9011D929A95E9F724E0C1
:10D700008202F00111242B96EEAFFFAF2B97E20DB2
:10D71000F31D80E090E0A0E8BFE380839183A283C3
:10D72000B383C090C723D090C823E090C923F09062
:10D73000CA234090C3235090C4236090C5237090A7
:10D74000C6238090BF239090C023A090C123B090A7
:10D75000C223A5019401C301B2010E946AD4181624
:10D760005CF080E090E0A0E8BFE329968CAF9DAF2D
:10D77000AEAFBFAF29970AC080E090E0A0E8BFEB52
:10D7800029968CAF9DAFAEAFBFAF2997A301920191
:10D79000C501B4010E94C1D20E94D9D49B0177FF78
:10D7A00004C022273327261B370BB901882777FDB2
:10D7B0008095982F0E940CD525966CAF7DAF8EAFCB
:10D7C0009FAF2597C0922A35D0922B35E0922C3509
:10D7D000F0922D350E9416830E94765520E030E0AD
:10D7E00040E050E425966CAD7DAD8EAD9FAD2597A4
:10D7F0000E946DD618166CF08091CB239091CC23AB
:10D80000A091CD23B091CE238BAF9CAFADAFBEAF77
:10D81000DBC02AE037ED43E25CE325966CAD7DADDD
:10D820008EAD9FAD25970E946DD618162CF709E195
:10D8300010E08AE0882E87ED982E83E2A82E8CE3F4
:10D84000B82E412C512C32012B96AEADBFAD2B978B
:10D85000A20DB31D58962196AEAFBFAF21974BAA2C
:10D860005CAA6DAA7EAA8FAA98AEA9AEBAAE299676
:10D870002CAD3DAD4EAD5FAD29976FA978AD89ADAB
:10D880009AAD0E940FD79B01AC016091C3237091A8
:10D89000C4238091C5239091C6230E94C2D22196B1
:10D8A000EEADFFAD21976083718382839383C09235
:10D8B0002A35D0922B35E0922C35F0922D35B101DE
:10D8C000CE0149960E9440538093B63F8111AAC071
:10D8D00020E030E040E85FE36BA97CA98DA99EA918
:10D8E0000E94C2D26BAB7CAB8DAB9EAB20E030E034
:10D8F00048EC51E40E9471D49B01AC0160E070E0FF
:10D9000080E291E40E9472D72B013C018091CB23ED
:10D910009091CC23A091CD23B091CE238BAF9CAF1F
:10D92000ADAFBEAFC090C723D090C823E090C9234D
:10D93000F090CA23A7019601BC01CD010E94C1D27B
:10D940004B015C0120E030E040E251E4C301B20150
:10D950000E9471D49B01AC01C501B4010E940FD794
:10D960009B01AC01C701B6010E94C2D26B017C01D0
:10D970002BA93CA94DA95EA9CA01B9010E94C2D236
:10D9800020E030E048EC51E40E9471D49B01AC01EE
:10D990006FA978AD89AD9AAD0E94C2D26FAB78AF56
:10D9A00089AF9AAF9B01AC0125966CAD7DAD8EAD74
:10D9B0009FAD25970E946DD6181634F401501109B9
:10D9C0000115110509F053CF8BAD9CADADADBEADCA
:10D9D00080932A3590932B35A0932C35B0932D3519
:10D9E0002B96EEADFFAD2B97E20DF31D8091BF237B
:10D9F0009091C023A091C123B091C223808F918FB9
:10DA0000A28FB38FB101CE0149960E9440538093FB
:10DA1000B63F811107C089E29DE68093CF239093A2
:10DA2000D02382E0C65BDF4FCDBFDEBFDF91CF9159
:10DA30001F910F91FF90EF90DF90CF90BF90AF902C
:10DA40009F908F907F906F905F904F903F902F901E
:10DA50000895CF93DF931F92CDB7DEB789830E94DD
:10DA600016834091D9235091DA236091DB23709182
:10DA7000DC2389810E94DE588091D6230E94814F49
:10DA80008091D5230E94C74E8091D7230E94CB4E10
:10DA90008091D8230E942C538091D1239091D2233E
:10DAA000A091D323B091D42380932A3590932B3522
:10DAB000A0932C35B0932D3564E08DEE94E30E9455
:10DAC000AF4A0E9423561092BE3489EA91E20E9426
:10DAD00005E280E00F90DF91CF9108950F931F939F
:10DAE000CF93C82F0BEE14E3F801808191810E943F
:10DAF000924A8093D523F801808191810E948D4ABA
:10DB00008093D623F801808191810E949C4A809362
:10DB1000D723F801808191810E94A14A8093D82364
:10DB2000F801808191810E94A84A6093D12370936B
:10DB3000D2238093D3239093D4238C2F0E94D35845
:10DB40006093D9237093DA238093DB239093DC23B3
:10DB500081E00E94C74E80E00E94CB4E80E00E9490
:10DB6000814F81E00E942C5340E050E060E271E47C
:10DB70004093C7235093C8236093C9237093CA234B
:10DB800085E3C89FF0011124ED57FC4C4081518181
:10DB9000628173814093CB235093CC236093CD2338
:10DBA0007093CE236C2F85EB98E50E94A44B609375
:10DBB000C3237093C4238093C5239093C6230E94EC
:10DBC000A7596093BF237093C0238093C123909380
:10DBD000C223C093BE238DE49BE68093CF23909312
:10DBE000D02384E08093BE3480E0CF911F910F91C9
:10DBF00008958091BE34843059F40E94A64A813041
:10DC000049F0E091CF23F091D0238091BE23199465
:10DC100083E0089582E00895E091DF23F0E0E95683
:10DC2000FD4C8381882341F087E29EE68093DD23CB
:10DC30009093DE2382E008956CE274E284E194E242
:10DC40000E9440538093B63F882371F308951F9339
:10DC5000CF93DF93E091DF23F0E0E956FD4C81E0C4
:10DC60009381913009F080E08093C834C9ECD4E30B
:10DC700010E0812F0E940497AB01BC01812F0E940C
:10DC80001850612F8091EB349091EC340E94A44B9A
:10DC900069937993899399931F5F163051F783EBBA
:10DCA00091E20E942A7D83E99EE68093DD23909392
:10DCB000DE2382E0DF91CF911F9108951F93CF93D0
:10DCC000DF930E9416838091E02380939732E09146
:10DCD000DF23F0E08091E123E956FD4C83870E9429
:10DCE000B4BCC4EED3E210E04991599169917991A5
:10DCF000812F0E94DE581F5F1630B1F78091E32319
:10DD00000E94814F8091E2230E94CB4E64E08DEE11
:10DD100094E30E94AF4A0E9423561092BE34DF91D2
:10DD2000CF911F9108950E945E6E80E008950F9339
:10DD30001F93CF93DF93CDB7DEB7C058D109CDBFC6
:10DD4000DEBF182F8AE091E20E9413611E3F29F482
:10DD500080EC91E20E94AD6219C0812F0E94B856FA
:10DD60001F928F9381E19BE39F938F938E010F5FAF
:10DD70001F4F1F930F930E945BE2C8010E94AD6288
:10DD80000F900F900F900F900F900F9042E062E075
:10DD90008AEF0E94BD620E945E6E8AEFC058DF4F1C
:10DDA000CDBFDEBFDF91CF911F910F910895FF92FC
:10DDB0000F931F93CF93DF931092C83482E0809328
:10DDC000BE3404EE13E2C3E9D3E3F12C8F2D0E949D
:10DDD000D358F80161937193819391938F01488196
:10DDE00059816A817B818F2D0E94DE586F2D809131
:10DDF000EB349091EC340E94A44BF801648B758B4A
:10DE0000868B978BF394E596F6E0FF12DFCF64E103
:10DE100074E28CEF93E20E94E5C02AE43CE042E821
:10DE20005EE30E946AD487FF03C08EEF0E94976E64
:10DE3000C8E0D4E213E069917991899199912C8994
:10DE40003D894E895F890E94C1D29F772CEA35ECCB
:10DE500047E257E30E946DD618161CF4812F0E94EA
:10DE6000976E1F5F163039F784E08093DF2380912F
:10DE7000A6328093E12381E08093A632809197328D
:10DE80008093E023109297320E94B4BC8091EB34CF
:10DE90009091EC340E948D4A8093E3238091EB347F
:10DEA0009091EC340E949C4A8093E22380E00E948F
:10DEB000CB4E80E00E94814F80E00E94E0AE8CE07B
:10DEC0009EE68093DD239093DE2382E0DF91CF9165
:10DED0001F910F91FF9008950F931F93CF93DF939E
:10DEE0008C01EB0180913635882399F080912A3599
:10DEF00090912B35A0912C35B0912D35BC01CD01E1
:10DF00009F772CEA35EC47E257E30E946AD487FDFD
:10DF10004FC088819981AA81BB81BC01CD019F77C7
:10DF20002CEA35EC47E257E30E946DD61816F4F45C
:10DF30008C819D81AE81BF81BC01CD019F772CEA90
:10DF400035EC47E257E30E946DD618167CF48885BD
:10DF50009985AA85BB85BC01CD019F772CEA35EC5C
:10DF600047E257E30E946DD6181624F188E1F801C4
:10DF7000A4E1B4E201900D928A95E1F788E1FE01F7
:10DF8000ACE2B4E201900D928A95E1F788E1E9EC08
:10DF9000F4E3DF011D928A95E9F782E08093C834AB
:10DFA00087ED9EE68093DD239093DE2380E003C01F
:10DFB0008EE801C086E8DF91CF911F910F910895FF
:10DFC0008091BE34823021F08091C834823049F48F
:10DFD0000E94A64A813039F0E091DD23F091DE23E2
:10DFE000199483E0089582E00895ECE2FFE380E273
:10DFF000DF011D928A95E9F78FEE92E180934A3F07
:10E0000090934B3F80839183089580914A3F9091F4
:10E010004B3F8F3E924111F08CE5089580912C3F4B
:10E0200090912D3F8F3E9241B9F780E00895CF93B4
:10E03000DF93C82FCB01BA010E94BED727E0C29F51
:10E04000E0011124C45DD04C0E94D9D46D837E833D
:10E050008F839887DF91CF91089597E0899FF00192
:10E060001124E45DF04C65817681878190850E9462
:10E070000CD508952F923F924F925F926F927F92AC
:10E080008F929F92AF92BF92CF92DF92EF92FF92C8
:10E090000F931F93CF93DF93CDB7DEB72797CDBFF5
:10E0A000DEBF8C011B828091BD34823009F440C7F1
:10E0B000D801BC90B11069C780E06E01B3E0CB0E0F
:10E0C000D11C3DC0F6018081811108C0B72CD70159
:10E0D0001C926E01B3E0CB0ED11C54C7883239F4C8
:10E0E000B72CF7011082FFEFCF1ADF0A4BC78B3333
:10E0F000B9F3A82EB12CC5010E9459E0892B39F43F
:10E10000B5018AEE91E20E94D2E0892B51F04701DD
:10E110008FEF881A980AC5010E947DE0D7018C9381
:10E120007401BFEFCB1ADB0AF70180818111CACFDE
:10E13000B72CD8018C916E01B3E0CB0ED11CF80145
:10E140001CC08E32E1F090E0C0970A97A0F0818168
:10E15000803391F4228130E0205331092A30310597
:10E1600058F4DF01119611968C9111978D938111BE
:10E17000FACF808102C0818131968111E2CFF60110
:10E18000A080A11007C068C0D6011196AC90BFEF67
:10E19000CB1ADB0A76018A2C912CC4010E946DE017
:10E1A000892B91F7EBE7AE122FC0D60111968C9117
:10E1B00090E00E9475E08437910531F5F601828187
:10E1C00090E00E9475E089369105F1F4D60113962E
:10E1D0008C9190E00E9475E084369105A9F4BE010F
:10E1E0006F5F7F4FC60105960E94D5DC0E94DED48A
:10E1F0006093A23C7093A33C8093A43C9093A53C75
:10E20000F601A0808A2C912CC4010E9475E08D3605
:10E210009105A1F4D60111968C9190E00E9475E0D1
:10E220008337910559F4F601828190E00E9475E0F0
:10E230008736910519F4F601339602C0FE01339634
:10E24000AA2061F08A2DD701893209F41C92119617
:10E250008C918111F9CF02C0FE0133968FE2B8167E
:10E2600009F468C68081882319F0CF010E9469559E
:10E2700080E1ECE4FFE3DF011D928A95E9F78BE58D
:10E28000E6E1F6E3DF01982F1D929A95E9F7EBEBB3
:10E29000F5E3DF011D928A95E9F78DEE94E30E9484
:10E2A0008A4A8093BC35812C912C80E8A82E8FE37C
:10E2B000B82E5524539492E0492E24E0322E23C4E4
:10E2C000C701B6010E94DED4862F90E08F359105FC
:10E2D00008F034C6FC01EC50FF4F0C94B5DC1092F2
:10E2E000BC355092173680914D3F8F5F80934D3FE4
:10E2F0000AC45092BC355092173680914D3F8F5FC3
:10E3000080934D3F00C44092BC35509217368091A7
:10E310004D3F8F5F80934D3FF6C383E08093BC35C4
:10E320005092173680914D3F8F5F80934D3FEBC3E6
:10E330008DE08093BB3550921636E5C388E0B2C0BD
:10E340001092EB355092463680914E3F8F5F80930E
:10E350004E3FD9C35092EB355092463680914E3F96
:10E360008F5F80934E3FCFC34092EB35509246363D
:10E3700080914E3F8F5F80934E3FC5C31092EC3526
:10E38000509247368091513F8F5F8093513FBBC37E
:10E390005092EC35509247368091513F8F5F809379
:10E3A000513FB1C3C701B6010E9429D86C837D8358
:10E3B0008E839F8320E030E040E251E4C701B60144
:10E3C0000E940FD76B017C0120E030E040E251E475
:10E3D0006C817D818E819F810E940FD79B01AC0152
:10E3E000C701B6010E94C1D20E94DED4623001F1A1
:10E3F00028F4662341F0613089F0A0C56330E9F06C
:10E40000643001F19BC5B5E0B093BB355092163630
:10E4100080914C3F8F5F80934C3F75C33092BB35EA
:10E420006093163680914C3F8F5F80934C3F6BC357
:10E430005092BB355092163666C34092BB3550920F
:10E44000163661C383E08093BB35509216365BC3AA
:10E45000C701B6010E9429D86C837D838E839F8378
:10E4600020E030E040E251E4C701B6010E940FD73E
:10E470006B017C0120E030E040E251E46C817D8161
:10E480008E819F810E940FD79B01AC01C701B6010D
:10E490000E94C1D20E94DED4662319F0613061F07F
:10E4A0004DC587E08093BB355092163680914C3F26
:10E4B0008F5F80934C3F27C3E6E0E093BB356093CA
:10E4C000163680914C3F8F5F80934C3F1CC3C70131
:10E4D000B6010E9429D86C837D838E839F8320E0C0
:10E4E00030E040E251E4C701B6010E940FD76B0152
:10E4F0007C0120E030E040E251E46C817D818E813E
:10E500009F810E940FD79B01AC01C701B6010E94F9
:10E51000C1D20E94DED4623009F010C58EE0809333
:10E52000BB3550921636EFC25092EE3550924936B6
:10E53000EAC25092ED35509248368091553F8F5F38
:10E540008093553FE0C24092ED355092483680911D
:10E55000553F8F5F8093553FD6C283E016C03092FF
:10E56000ED35509248368091553F8F5F8093553FEF
:10E57000CAC2F5E0F093ED35509248368091553F90
:10E580008F5F8093553FBFC286E08093ED355092F8
:10E5900048368091553F8F5F8093553FB4C2C70185
:10E5A000B6010E9429D86C837D838E839F8320E0EF
:10E5B00030E040E251E4C701B6010E940FD76B0181
:10E5C0007C0120E030E040E251E46C817D818E816D
:10E5D0009F810E940FD79B01AC01C701B6010E9429
:10E5E000C1D20E94DED4662319F0613059F0A6C46E
:10E5F0001092F03550924B368091563F8F5F80934A
:10E60000563F81C26093F03560934B368091563F00
:10E610008F5F8093563F77C24092F03550924B36D1
:10E620008091563F8F5F8093563F6DC23092BC35CC
:10E630005092173680914D3F8F5F80934D3F63C25C
:10E64000C701B6010E9429D86C837D838E839F8386
:10E6500020E030E040E251E4C701B6010E940FD74C
:10E660006B017C0120E030E040E251E46C817D816F
:10E670008E819F810E940FD79B01AC01C701B6011B
:10E680000E94C1D20E94DED4662319F0613059F095
:10E6900055C41092F13550924C3680914F3F8F5FA8
:10E6A00080934F3F30C21092F23560934D36809187
:10E6B0004F3F8F5F80934F3F26C2C701B6010E9434
:10E6C00029D86C837D838E839F8320E030E040E2F5
:10E6D00051E4C701B6010E940FD76B017C0120E015
:10E6E00030E040E251E46C817D818E819F810E9407
:10E6F0000FD79B01AC01C701B6010E94C1D20E9495
:10E70000DED4662319F0613059F018C45092F13507
:10E7100050924C3680914F3F8F5F80934F3FF3C1B3
:10E720006093F23560934D3680914F3F8F5F8093B9
:10E730004F3FE9C1C701B6010E9429D86C837D8390
:10E740008E839F8320E030E040E251E4C701B601B0
:10E750000E940FD76B017C0120E030E040E251E4E1
:10E760006C817D818E819F810E940FD79B01AC01BE
:10E77000C701B6010E94C1D20E94DED4613089F087
:10E7800028F06230A1F06330C1F0D8C399E09093D3
:10E79000BB355092163680914C3F8F5F80934C3F33
:10E7A000B2C1AAE0A093BB3560931636ACC1BBE002
:10E7B000B093BB3550921636A6C1ECE0E093BB3562
:10E7C00050921636A0C11092E63550924136809193
:10E7D000503F8F5F8093503F96C15092E6355092E4
:10E7E00041368091503F8F5F8093503F8CC1C7016D
:10E7F000B6010E94DED4862F90E08D33910508F09B
:10E800009BC3FC01ED5AFE4F0C94B5DC1092BD3554
:10E81000509218368091573F8F5F8093573F73C156
:10E820005092BD35509218368091573F8F5F80933C
:10E83000573F69C15092F835509253368091593FF5
:10E840008F5F8093593F5FC14092F83550925336A5
:10E850008091593F8F5F8093593F55C11092F83591
:10E86000509253368091593F8F5F8093593F4BC1EF
:10E870005092F5355092503646C15092F63550922E
:10E88000513680915A3F8F5F80935A3F3CC15092DE
:10E89000F7355092523680915A3F8F5F80935A3F9E
:10E8A00032C11092F7355092523680915A3F8F5FA5
:10E8B00080935A3F28C15092E93550924436809156
:10E8C0005B3F8F5F80935B3F1EC11092E935509292
:10E8D000443680915B3F8F5F80935B3F14C15092C1
:10E8E000E7355092423680915B3F8F5F80935B3F6C
:10E8F0000AC15092013650925C3680915B3F8F5F27
:10E9000080935B3F00C1C701B6010E9429D80E94D5
:10E91000DED46093F43550924F36F5C0C092DA35AC
:10E92000D092DB35E092DC35F092DD3580923536E1
:10E9300090923636A0923736B0923836E4C0C09204
:10E940000236D0920336E0920436F0920536809279
:10E950005D3690925E36A0925F36B0926036D3C03C
:10E96000C092F935D092FA35E092FB35F092FC3541
:10E970008092543690925536A0925636B0925736C1
:10E98000C2C0C092C235D092C335E092C435F09275
:10E99000C53580921D3690921E36A0921F36B092D9
:10E9A0002036B1C0C092C635D092C735E092C83586
:10E9B000F092C9358092213690922236A092233669
:10E9C000B0922436A0C0C092CA35D092CB35E09226
:10E9D000CC35F092CD358092253690922636A09295
:10E9E0002736B09228368FC0C092CE35D092CF3520
:10E9F000E092D035F092D1358092293690922A3625
:10EA0000A0922B36B0922C367EC0C092D235D092D6
:10EA1000D335E092D435F092D53580922D36909250
:10EA20002E36A0922F36B09230366DC0C092D635B9
:10EA3000D092D735E092D835F092D93580923136E0
:10EA400090923236A0923336B09234365CC0C09287
:10EA50000A36D0920B36E0920C36F0920D36809248
:10EA6000653690926636A0926736B09268364BC093
:10EA7000C0920E36D0920F36E0921036F0921136D8
:10EA80008092693690926A36A0926B36B0926C365C
:10EA90003AC0C0921236D0921336E0921436F092F9
:10EAA000153680926D3690926E36A0926F36B09287
:10EAB000703629C0C0920636D0920736E0920836EA
:10EAC000F09209368092613690926236A092633657
:10EAD000B092643618C0C701B6010E94DED46093BC
:10EAE000BE357093BF358093C0359093C13581E0BA
:10EAF00090E0A0E0B0E08093193690931A36A0938E
:10EB00001B36B0931C36D8012C90222009F424C265
:10EB1000822D90E00E9464E0892B09F42FC2380115
:10EB2000BFEF6B1A7B0AF8018181803349F482813F
:10EB3000883531F40E5F1F4FC12CD12C760100C2F5
:10EB4000BE016F5F7F4FC3010E94D5DC6B017C016A
:10EB500009811A816016710609F0F2C111C2809113
:10EB6000E6350E942C53182F01C010E06091353615
:10EB70007091363680913736909138360E94DED4C7
:10EB8000662359F06091DA357091DB358091DC3580
:10EB90009091DD350E94FB52182F609139367091AB
:10EBA0003A3680913B3690913C360E94DED4662303
:10EBB00071F06091DE357091DF358091E035909194
:10EBC000E1350E94DED4862F0E94D754182F609121
:10EBD0003D3670913E3680913F36909140360E948E
:10EBE000DED4662371F06091E2357091E335809157
:10EBF000E4359091E5350E94DED4862F0E941655AB
:10EC0000182F6091543670915536809156369091F8
:10EC100057360E94DED4662359F06091F935709121
:10EC2000FA358091FB359091FC350E9414AF182F76
:10EC3000609158367091593680915A3690915B3672
:10EC40000E94DED4662371F06091FD357091FE352F
:10EC50008091FF35909100360E94DED4862F0E946D
:10EC60005555182F80914F36882329F08091F4351F
:10EC70000E949453182F80915036882329F0809158
:10EC8000F5350E94C853182F80915336882329F0F8
:10EC90008091F8350E94E0AE182F8091513688237C
:10ECA00029F08091F6350E94FD53182F809152363D
:10ECB000882329F08091F7350E943154182F8091D4
:10ECC0004236882329F08091E7350E94AC54182FF2
:10ECD00080914336882329F08091E8350E94EB54D7
:10ECE000182F80915C36882329F0809101360E948C
:10ECF0002A55182F80914436882329F08091E935D0
:10ED00000E94A454182F8091BB358D3029F080913A
:10ED100046368823A9F00FC0609102367091033601
:10ED200080910436909105360E9434538093B63F0B
:10ED3000882369F32FC18091EB350E94C34E182FB1
:10ED400080914736882329F08091EC350E94C74E88
:10ED5000182F80914836882329F08091ED350E9444
:10ED6000814F182F80914B36882329F08091F03500
:10ED70000E943053182F80914C36882329F08091BF
:10ED8000F1350E94CB4E182F4091BB3550E04F30EB
:10ED9000510508F0B6C0FA01E057FE4F0C94B5DCFF
:10EDA0000E947D52182FADC06DE176E382EC95E3B1
:10EDB0000E948852182FA5C00E94BC52182FA1C0D3
:10EDC0006DE176E382EC95E30E94C752182F99C05B
:10EDD0000E94EB6A182F95C06DE176E382EC95E313
:10EDE0000E944750182F8DC00E94346B182F89C085
:10EDF0006DE176E382EC95E30E946C6F182F81C081
:10EE000060910236709103368091043690910536F8
:10EE10000E94DED4862F2DE136E342EC55E360916B
:10EE2000EA350E94CF4E182F6CC06DE176E382EC7C
:10EE300095E30E94C450182F64C00E947751182F88
:10EE400060C00E94DE51182F5CC00E941552182F1E
:10EE500058C06091EE358DEE94E30E94254B809171
:10EE6000BC35843038F48230D8F4882349F08130BE
:10EE700079F047C0843009F044C08093F13441C038
:10EE80006DE176E382EC95E30E944D52182F39C074
:10EE90006DE176E382EC95E30E944053182F31C078
:10EEA000A0901236B0901336C0901436D09015361C
:10EEB000E0900E36F0900F3600911036109111361A
:10EEC00020910A3630910B3640910C3650910D3618
:10EED0008F93809109368F93809108368F9380911C
:10EEE00007368F93809106368F936DE176E382EC3F
:10EEF00095E30E94A684182F0F900F900F900F900B
:10EF00000F9060E08DEE94E30E94254B80911836BF
:10EF1000813061F48091BD35811104C00E94565644
:10EF2000812F38C00E948756812F34C0812F32C074
:10EF30008BEC30C083E02EC084E82CC083E82AC06C
:10EF4000822D90E0FC01E154F109EA31F105B0F7BE
:10EF5000E156FE4F0C94B5DC1092B63F6091BE3581
:10EF60007091BF358091C0359091C1350E94BF4AE4
:10EF700080914136882309F4F8CDF1CD85E60AC0A9
:10EF800086E608C0D8018C91DAC868018B2D78011B
:10EF90007B2CA4C82796CDBFDEBFDF91CF911F91F8
:10EFA0000F91FF90EF90DF90CF90BF90AF909F9028
:10EFB0008F907F906F905F904F903F902F9008952B
:10EFC000CF93DF93EC016AEA7EE30E94166280939E
:10EFD000B63F811102C095E09F83DF91CF910895E4
:10EFE000FC018789908D0C943A7083FF06C0E091F4
:10EFF0008F32F091903290E2958382FF06C0E091CB
:10F000009132F091923290E2958381FF06C0E091B7
:10F010009332F091943290E2958380FF06C0E091A4
:10F020009532F091963280E28583089583FF06C081
:10F03000E0918F32F091903290E2968382FF06C089
:10F04000E0919132F091923290E2968381FF06C076
:10F05000E0919332F091943290E2968380FF06C063
:10F06000E0919532F091963280E286830895809106
:10F07000863C811107C084E00E94F57781E080938F
:10F08000863C089584E00E9416781092863C08958C
:10F09000CF92DF92EF92FF920F931F93CF93DF9364
:10F0A000C12C26E0D22EC0927F32D092803230EA3C
:10F0B000E32E36E0F32EE0928132F092823200E8C5
:10F0C00016E00093833210938432C0E6D6E0C093FA
:10F0D0008532D0938632C0928732D0928832C093E4
:10F0E0008932D0938A3200938B3210938C32E09223
:10F0F0008D32F0928E322DEC3CEC4CED50E40E94BF
:10F100006DD6C0928F32D0929032E0929132F092CE
:10F11000923218164CF4C0939332D09394320093E9
:10F1200095321093963208C0009393321093943224
:10F13000C0939532D0939632DF91CF911F910F916A
:10F14000FF90EF90DF90CF9008950E9414D260E07E
:10F1500070E080E091E40E9448780C9433D281E022
:10F1600080938F3C089520E093E088ED08B618BEA8
:10F1700084BF909380002091820021FDFCCF08BEC7
:10F18000FFCF80918F3C81110E94B37883E0089576
:10F190008091903C882341F0F89461E089E790E009
:10F1A0000E9416D282E0089583E00895CF93DF9302
:10F1B000CDB7DEB7AD97CDBFDEBF21E2EDEEF1E218
:10F1C000DE01119601900D922A95E1F722E020933D
:10F1D000CA01DE019296E8E0F0E024912D93319689
:10F1E000EE30F105D1F72DE228A7E0E1F0E0E4915F
:10F1F000EF7121E030E02C0F3D1F2E0F311DF90182
:10F20000208129A7E2E1F0E0E491EF719E012E0F49
:10F21000311DF90121812AA7E4E1F0E0E491EF71C9
:10F220009E012E0F311DF90121812BA71CA61092E2
:10F23000CA0125E0FC012783BE016E5D7F4F0E945D
:10F2400016628093B63FAD96CDBFDEBFDF91CF9102
:10F25000089581E08093903C80E00895CF93DF9300
:10F26000EC0120E030E040E051E469857A858B854F
:10F270009C850E946DD618166CF0CE010E94F15E3E
:10F2800069857A858B859C850E9448780E94B4BCEC
:10F2900080E001C08DE6DF91CF91089561EB7BE3C3
:10F2A0000C94A8C063E97BE30C94A8C066E77BE3F9
:10F2B0000C94A8C068E57BE30C94A8C064E47BE3ED
:10F2C0000C94A8C0CF93DF9387EF96E49F938F931E
:10F2D000CEE6DCE589818F9388818F930E9480E15F
:10F2E00081EC94E49F938F9389818F9388818F938E
:10F2F0000E9480E189E394E49F938F9389818F93A7
:10F3000088818F930E9480E18FE693E49F938F938F
:10F3100089818F9388818F930E9480E10E9481A8C8
:10F320008DB79EB740968DBF9EBF80E0DF91CF9195
:10F330000895CF93DF938AE493E49F938F93CEE66F
:10F34000DCE589818F9388818F930E9480E18CED29
:10F3500091E49F938F9389818F9388818F930E94EB
:10F3600080E181E590E49F938F9389818F938881D9
:10F370008F930E9480E189E394E49F938F93898126
:10F380008F9388818F930E9480E18FE693E49F930F
:10F390008F9389818F9388818F930E9480E18DB7AD
:10F3A0009EB744968DBF9EBF80E0DF91CF910895B8
:10F3B000CF93DF9380E390E49F938F93CEE6DCE5D9
:10F3C00089818F9388818F930E9480E182EB9CE3F7
:10F3D0009F938F9389818F9388818F930E9480E17F
:10F3E0008FE693E49F938F9389818F9388818F9386
:10F3F0000E9480E18DB79EB70C968DBF9EBF80E0C6
:10F40000DF91CF910895CF93DF938AE89CE39F9398
:10F410008F93CEE6DCE589818F9388818F930E945C
:10F4200080E189E19CE39F938F9389818F93888109
:10F430008F930E9480E18FE693E49F938F9389815D
:10F440008F9388818F930E9480E18DB79EB70C9631
:10F450008DBF9EBF80E0DF91CF910895CF93DF9362
:10F4600086EF9BE39F938F93CEE6DCE589818F93B4
:10F4700088818F930E9480E18DEC9BE39F938F9313
:10F4800089818F9388818F930E9480E18FE693E436
:10F490009F938F9389818F9388818F930E9480E1BE
:10F4A0008DB79EB70C968DBF9EBF80E0DF91CF9148
:10F4B00008952F923F924F925F926F927F928F9218
:10F4C0009F92AF92BF92CF92DF92EF92FF920F93F3
:10F4D0001F93CF93DF93CDB7DEB76E97CDBFDEBF5F
:10F4E0003C016B011F86188A198A1A8A80915F3F36
:10F4F0008F5F80935F3F833008F08BC2FB010190E8
:10F500000020E9F73197E61BF70BE130F24008F0F5
:10F5100082C2DB018C91882379F17B01BFEFEB1A6A
:10F52000FB0A8B0191E020E0211118C021E0883214
:10F5300009F020E0992321F08132C0F08F37B1F03B
:10F540005801EFEFAE1ABE0A90E02E8F0E9475E0D0
:10F55000D8018C93850190E02E8D08C021E089327E
:10F5600009F420E0F80180830F5F1F4FD7018D91D0
:10F570007D018111D9CF01C08B01F8011082109259
:10F58000B63F2AE3222E22E2322E412C3DE7832E83
:10F590003CE2932E32E2A32EB12C8BE79CE2A2E256
:10F5A000B0E08B879C87AD87BE872B8A3C8A4D8ACB
:10F5B0008F829886A986BA8686E0EEE0F2E2DE01C6
:10F5C000119601900D928A95E1F7D6016C91662310
:10F5D00009F468C170E0CE010B960E94D2E0892B3D
:10F5E00009F460C1C3010E941A607601B9E0EB0E14
:10F5F000F11C8601EFEFCE1ADE0AD8016C9170E0A3
:10F60000CE010B960E94D2E0892B41F4760198013D
:10F610002E5D3F4F088F198F890104C0CE14DF047F
:10F6200041F7FDC16701BFEFEB1AFB0AF6016081EC
:10F6300070E0CE0143960E94D2E0892BE1F0088D64
:10F64000198DD6011C927301B1E1EB0EF11C46E05D
:10F6500050E0B801C7010E94FDE0B70187E493E2E2
:10F660000E94735F888F998FF3018483958301963D
:10F6700031F484E6D9C1E016F106A1F6FACF86018D
:10F680000F5F1F4F2AE0C20ED11C6A8E7B8EEC8E5C
:10F69000FD8E3801D8015D908D01E52CF12CC7015C
:10F6A0000E9459E0892B59F4B701CE0101960E94BE
:10F6B000D2E0892B21F40C151D0559F7DACF63012F
:10F6C0006A8C7B8C9701EC8CFD8CBEE65B1649F056
:10F6D000E2E25E1209C0D60111968C91823209F0E5
:10F6E0004AC0F3011782C0C0C901C0970A9718F039
:10F6F000FDE25F1235C0E88DF98DEE0FFF1F288DFA
:10F70000398DE20FF31FEE0FFF1FEE0FFF1FEE0FFD
:10F71000FF1FE356FA4EE491E4FF17C0BE016A5E94
:10F720007F4FC6010E94D5DCD30119966D937D935E
:10F730008D939C931C978E899F898C159D0509F448
:10F7400070C184E017968C938FC0C6010E945ADF67
:10F75000F301618772878387948782E0878384C0FF
:10F76000FBE75F1254C087E0D30117968C93BFEF7D
:10F77000CB1ADB0A99C0B6016F5F7F4F85E0F301BA
:10F780008783C6018F579F4FFB01DB0120812C35FA
:10F7900031F431813232A1F43C93319612C02232DD
:10F7A00079F41C926F012FEFC21AD20AD6010D9084
:10F7B0000020E9F71197AC19BD09139740F41FC059
:10F7C0002C9331961196A817B90701F72CC18181A6
:10F7D0008033A9F48281883791F440E050E060E002
:10F7E00070E0C6010E9446DED30119966D937D93A9
:10F7F0008D939C931C9783E017968C9335C0C3011F
:10F800000E9416628093B63F882371F146C0B4E728
:10F810005B120CC081E0F301878381E090E0A0E0FF
:10F82000B0E081879287A387B4871EC0F6E65F1297
:10F830000AC081E0D30117968C93F30111861286DA
:10F840001386148611C0FBE55F12E9C086E0D30180
:10F8500017968C93B601C3010E9416628093B63F3F
:10F8600081111BC087E6E0C0BE01695F7F4FC60102
:10F870000E9417E16C01009709F4D1C0FC0180815E
:10F880008D3729F4818196012F5F3F4F69018C32BA
:10F8900059F03FEFC31AD30A07C0843008F0C4C040
:10F8A000833011F480E0C0C08F85882349F043E0A5
:10F8B00050E0BE01615F7F4FC3010D960E94FDE0E5
:10F8C000D30114968D919C9115970E94A86488236A
:10F8D00061F0C7010E94515F882339F043E050E096
:10F8E000B701CE010F960E94FDE0F301848195815E
:10F8F00020910237309103378217930711F42EEFCE
:10F9000027830E94685F882309F455C0D301579666
:10F910000D911C915897F80160816B3729F4B8015B
:10F92000C3010E94597A47C070E088E791E20E94C3
:10F93000D2E0892B61F180915D3F811103C0AEE17E
:10F94000B7E402C0A0E1B7E4BF93AF930E94E1E146
:10F950000F900F9082E08093843CC8010E94B7BD55
:10F9600011E01093843CAEE0B7E4BF93AF930E94E4
:10F97000E1E180E090E00E9413611093603FD301C9
:10F9800012968D919C9113970F900F903EC087E631
:10F9900093E6A0E0F70180839183A283C8010E94CF
:10F9A0003A706AEA7EE30E941FBFD30112968D91DE
:10F9B0009C9113972AC0F30187818F3F19F48281AC
:10F9C000938123C0811105C0C3010E94E85BF3014C
:10F9D00012C08091BD34823069F0C3010E94BE5BC9
:10F9E000C3010E943B5CF30106C027812F3F61F0F9
:10F9F000FC0101C0F301828193810097B1F782B1CC
:10FA000093B1612C712C01C03F01892B09F0C5CD48
:10FA100049CF82E709C08BE68093B63F05C08FE6E9
:10FA200003C086E601C081E76E96CDBFDEBFDF91E1
:10FA3000CF911F910F91FF90EF90DF90CF90BF90EB
:10FA4000AF909F908F907F906F905F904F903F907E
:10FA50002F900895CF93DF93EC011092603F1092A6
:10FA60005F3F8AE091E20E941361BE010E94597AD1
:10FA700042E060E00E94BD6281E0DF91CF910C9492
:10FA8000D1AA2F923F924F925F926F927F928F9264
:10FA90009F92AF92BF92CF92DF92EF92FF920F931D
:10FAA0001F93CF93DF935C011B018A01060F171F81
:10FAB000DC0116969C908091603FEB012196882393
:10FAC00021F08CE2FB01808303C08BE7DB018C9388
:10FAD00090E0412C4BE7642E55E0752E68E1C62E70
:10FAE00062E2D62E74E1E72E72E2F72EECE28E2E61
:10FAF000FDE75F2EF50187818E5F823008F4E5C057
:10FB0000992311F08882219680915D3F811113C065
:10FB1000C50141969F938F93FF92EF92DF93CF930E
:10FB20000E9432E2C80FD91F0F900F900F900F90D4
:10FB30000F900F9012C0C50141969F938F93DF9253
:10FB4000CF92DF93CF930E9432E2C80FD91F0F905C
:10FB50000F900F900F900F900F90D50117968C91EA
:10FB6000811103C0EEE1F2E2A0C0823019F5D501A7
:10FB70001C968C911C978F931B968C911B978F933F
:10FB80001A968C911A978F9319968C918F93A3E262
:10FB9000B2E2BF93AF93DF93CF930E9432E2C80FDC
:10FBA000D91FD50117968C91EDB7FEB73896EDBFEA
:10FBB000FEBF84C0833019F5D5011C968C911C972B
:10FBC0008F931B968C911B978F931A968C911A97F3
:10FBD0008F9319968C918F93A7E2B2E2BF93AF9364
:10FBE000DF93CF930E9432E2C80FD91FD501179639
:10FBF0008C91EDB7FEB73896EDBFFEBF5FC0853084
:10FC000059F4D50158968C9158978F9357968C91AB
:10FC10008F93AFE2B2E209C08630C9F4F501808D5E
:10FC20008F9387898F93A4E3B2E2BF93AF93DF935F
:10FC3000CF930E9432E2C80FD91FD50117968C913D
:10FC40000F900F900F900F900F900F9037C084304F
:10FC500091F4C5010E94B864F50141855285638520
:10FC600074852085CE010E94D9C2C80FD11DD5014F
:10FC700017968C9123C0813009F5F5018185928515
:10FC8000A385B485892B8A2B8B2B69F4E9E3F2E2F7
:10FC9000DE0186E001900D928A95E1F72596D50167
:10FCA00017968C910BC0EFE3F2E2DE01872D0190F5
:10FCB0000D928A95E1F72496F5018781873021F42A
:10FCC0006882219690E001C091E0C017D10718F03A
:10FCD0008FEF9FEF48C0D5011296AD90BC9013975F
:10FCE000A114B10441F0F50186812FEF240D841594
:10FCF0002CF0482EFFCE9414A4F01EC0FE01D501B6
:10FD0000CF010196EC01508216964C9016973FEF6A
:10FD1000320F42161CF4232FFC01F2CF5D0191E05B
:10FD2000E9CEFE012DE7CF010196EC0120834A9434
:10FD3000941414F4FC01F7CF8091603F882329F0DC
:10FD40001092603F8DE7888321968DE79AE0A0E0CE
:10FD500088839983AA8322960C171D0708F4B8CFCD
:10FD6000CE0182199309DF91CF911F910F91FF90DE
:10FD7000EF90DF90CF90BF90AF909F908F907F904B
:10FD80006F905F904F903F902F90089540E052E029
:10FD90006AEA7CE30E94417D8AEA9CE39F938F9309
:10FDA0000E94CFE10F900F900895BF92CF92DF9203
:10FDB000EF92FF920F931F93CF93DF93CDB7DEB7F0
:10FDC0006297CDBFDEBFB82E80915C3F882309F4D7
:10FDD000FFC08FE6B81214C08AE091E20E9413615E
:10FDE0006AEA7EE38091A63C9091A73C0E94B9C24A
:10FDF000BC018CE091E20E9474620DE117E332C015
:10FE00008091BD340DE117E3882361F1FF24FA945A
:10FE1000C8010E94DA5F882329F1823029F4809199
:10FE2000653F811119C016C0843029F48091623F6A
:10FE3000811112C00FC0853079F48091643F88230E
:10FE400049F0F8014185528563857485452B462B21
:10FE5000472B11F0F801F782F80102811381011597
:10FE60001105B1F6C090A23CD090A33CE090A43C18
:10FE7000F090A53CC701B6010E940AD52CEA35ECEA
:10FE800047E257E30E946DD6181654F14EC0F801B0
:10FE9000028113810115110519F581E70E9407A858
:10FEA0008091A23C9091A33CA091A43CB091A53C30
:10FEB00089B99AB9ABB9BCB984E799E6A4E6B0E0D0
:10FEC00081BB92BBA3BBB4BB82E087B916B840E04C
:10FED00052E06AEA7CE384E097E30E94417D78C0C7
:10FEE000F80187818F3F99F6C186D286E386F48632
:10FEF00084E799E6A4E6B0E0818B928BA38BB48B68
:10FF000082E087831682028113810FC0F80102818B
:10FF100013810115110549F440E052E06AEA7CE3DF
:10FF200084E097E30E94417D53C0F80187818F3FB1
:10FF300069F78091773281111AC08091A93C8F9323
:10FF40008091A83C8F931F92BF9284E492E29F938A
:10FF50008F93CE0101967C01FF928F930E9432E233
:10FF60001092A83C1092A93CCDBFDEBF13C00E94E6
:10FF70000EC81F928F931F92BF928CE492E29F93C0
:10FF80008F93CE0101967C01FF928F930E9432E203
:10FF9000CDBFDEBFB701C8010E941662F80116820C
:10FFA00086E0878386E690E0818B928B12821382B3
:10FFB00040E052E06AEA7CE384E097E30E94417DFE
:10FFC0008AEA9CE39F938F930E94CFE10F900F905A
:10FFD0006296CDBFDEBFDF91CF911F910F91FF9051
:10FFE000EF90DF90CF90BF900895613019F06230AC
:10FFF00029F0089584E097E30C94C67E0C94D57E96
:020000021000EC
:10000000FC0181859285A385B48586309105A10583
:10001000B10580F580935C3F1092613F1092623F82
:100020001092633F1092643F1092653F0097A105C4
:10003000B10511F121E02093613F81309105A105C7
:10004000B105D1F02093623F82309105A105B10541
:1000500099F02093633F83309105A105B10561F0CC
:100060002093643F0597A105B10531F42093653FC6
:1000700080E008958EE6089580E0089563EB77E4CC
:100080000C94A8C06CE577E40C94A8C068E277E40F
:100090000C94A8C0BF92CF92DF92EF92FF920F9381
:1000A0001F93CF93DF93CDB7DEB76897CDBFDEBF89
:1000B0006B0128E1FC01DE01119601900D922A9559
:1000C000E1F78EE7E82E83E3F82E8E010F5F1F4FD6
:1000D000B12CF7018081823029F4F801108211825D
:1000E000128213828091F05A8B1114C02091035B0D
:1000F0003091045B4091055B5091065BF801608193
:100100007181828193810E940FD7F6016083718390
:100110008283938380910F5B8B1114C02091225BAB
:100120003091235B4091245B5091255BF801608105
:100130007181828193810E940FD7F6016483758358
:100140008683978380912E5B8B1114C02091415B35
:100150003091425B4091435B5091445BF801608178
:100160007181828193810E940FD7F6016087718728
:100170008287938780914D5B8B1114C02091605BC7
:100180003091615B4091625B5091635BF8016081EB
:100190007181828193810E940FD7F60164877587F0
:1001A00086879787B394F5E3EF0EF11C0C5F1F4F22
:1001B00086E0B8128ECF6896CDBFDEBFDF91CF91BB
:1001C0001F910F91FF90EF90DF90CF90BF90089517
:1001D000F8940E94A5780E943F810E9433D20E9429
:1001E000CCC40E944BB30E94F56F0E94B4BC0E9425
:1001F000E8A540E060E080E00E94B8650E945B6195
:100200000E942D810E94F2820E94B74F0E942BD241
:100210008091A20084608093A2008091A2008260FD
:100220008093A2008091A20081608093A2007894C4
:100230000E9481A80E94B6BD0E940A66FDCFE82FE9
:10024000F0E0EE0FFF1FE152F84B659174914FE41F
:1002500050E086E69FE30C94A4E08091833C8230DA
:1002600041F440E060E081E00E94B86580E00E94D7
:1002700032670C9407C9682F81E00C94A9C51092CD
:10028000B73F1092B83F1092B93F1092BA3F08950D
:10029000CF93DF93EC018C819D81880F991F880F8C
:1002A000991F2091B93F3091BA3F820F931F8093DD
:1002B000BB3F9093BC3F44E050E061EC7FE30E9481
:1002C0002BD14091C13F5091C23F6091C33F70918B
:1002D000C43F49875A876B877C8780E0DF91CF9145
:1002E00008950F931F93CF93DF93EC018091BE3459
:1002F000882339F089E0DF91CF911F910F910C9401
:1003000007A849855A856B857C854093BD3F5093EE
:10031000BE3F6093BF3F7093C03FCE010E944881B3
:100320008093B63F811141C00091BD3F1091BE3F07
:100330002091BF3F3091C03F49855A856B857C85B0
:10034000401751076207730739F10093C13F1093BB
:10035000C23F2093C33F3093C43F8C819D81880F5F
:10036000991F880F991F2091B93F3091BA3F820F92
:10037000931F8093BB3F9093BC3F44E050E061ECFF
:100380007FE30E94BCD13091BD3F2091BE3F909150
:10039000BF3F8091C03F04C0342F252F962F872F59
:1003A00039872A879B878C8780E0DF91CF911F91C7
:1003B0000F9108950E94CAB880E008958091C53FCA
:1003C0009091C63F8F3E924111F08EE50895809145
:1003D000EB3F9091EC3F8F3E9241B9F78091ED3F1A
:1003E0009091EE3F8F3E924181F7809176579091A8
:1003F00077578F3E924149F780917857909179577E
:100400008F3E924111F780910B5990910C598F3E7C
:100410009241D9F680E0089594E0899FF00111247B
:10042000EB53F04C4283538364837583089594E0C7
:10043000899FF0011124E858F84A45AB56AB67ABE9
:1004400070AF08955F926F927F928F929F92AF925A
:10045000BF92CF92DF92EF92FF920F931F93CF93B1
:10046000DF93CDB7DEB76097CDBFDEBFBE016F5F54
:100470007F4F8DEA97E50E944A80CE0101964C019C
:1004800085E2A82E88E5B82E95E3C92E98E5D92EE9
:1004900025E4E22E28E5F22E05E618E537E8632E7E
:1004A0003BE5732E512CF401419151916191719171
:1004B0004F01F50141935193619371935F01F601EF
:1004C00041935193619371936F01F701419351935C
:1004D000619371937F01852D0E941770F80111922D
:1004E0001192119211928F01F301108211821282E6
:1004F00013825394F8E16F0E711C84E05812D3CF2D
:100500006096CDBFDEBFDF91CF911F910F91FF901D
:10051000EF90DF90CF90BF90AF909F908F907F90A3
:100520006F905F9008958091EF3F08951F93CF9350
:10053000DF938BE897E1EDEEFFE3DF019C011D9275
:1005400021503040E1F78FEE92E18093ED3F9093A0
:10055000EE3F8093765790937757C6EFDFE3C093D3
:10056000F03FD093F13FC093F23FD093F33FC0935D
:10057000F43FD093F53F81E090E06AEB76E520E030
:1005800030E01CEB129FA001139F500D1124FA01C3
:10059000E351F04CD90111961A9F90011B9F300D29
:1005A00011242A50304C2387348761877287BA011F
:1005B0006A50704C9C0101968032910519F78CEBC2
:1005C000829FF001839FF00D1124E351F04CC3870B
:1005D000D4876187728780E28093EF3FDF91CF916C
:1005E0001F910895CF93DF93E8E7F7E585E991E060
:1005F000DF01EC011D922197E9F7A5ECBFE388E24A
:10060000ED0119928A95E9F78FEE92E18D939C9313
:100610008093EB3F9093EC3F8083918380930B59C1
:1006200090930C59DF91CF910C9496820E940F8D7C
:100630000E94968280E00C94744AE091F03FF09121
:10064000F13F848581111BC022813381808191819A
:100650004CEBDF011D924A95E9F7228333838083B7
:10066000918381E084878091EF3F81508093EF3FB9
:10067000828193818093F03F9093F13F05C08CE19C
:100680000E9407A8E0E0F0E0CF010895A2EFBFE3E9
:10069000ED91FC911197858781E0878782E08487BF
:1006A000828193818D939C9381E00E9408AC0C948D
:1006B00010B6EF92FF920F931F93CF93DF9300D06A
:1006C0001F92CDB7DEB78C014B835C8369837A833D
:1006D0000E941D83FC014B815C8169817A810097B6
:1006E00061F48EE02496CDBFDEBFDF91CF911F91E4
:1006F0000F91FF90EF900C94B34E83E085878AEDC5
:1007000091E884839583068317838B017A0126E021
:10071000D8014D915D916D917D918D01CF018559EC
:100720009F4FDC014D935D936D937C931397D7019D
:100730004D915D916D917D917D01418B528B638BCC
:10074000748B215034962111E3CF83E02496CDBFE2
:10075000DEBFDF91CF911F910F91FF90EF900C942E
:100760004683CF92DF92EF92FF926B017C010E9451
:100770001D83009739F48EE0FF90EF90DF90CF90CB
:100780000C94B34E24E334E8FC0124833583E5560E
:10079000FF4FC082D182E282F38221E0FC012787F1
:1007A00082E00E94468380E0FF90EF90DF90CF9040
:1007B00008958091F43F9091F53FFC0124853EEF30
:1007C000320F323018F424E024870895243011F0D9
:1007D00080E090E00895E091F43FF091F53F2281B0
:1007E0003381808191814CEBDF011D924A95E9F7BD
:1007F0002283338380839183E091F43FF091F53F2E
:100800000280F381E02DE093F43FF093F53F84857F
:10081000823011F483E084878091EF3F8F5F809373
:10082000EF3F8FEF0E9408AC81E04091F03F509184
:10083000F13F2091F43F3091F53F4217530709F003
:1008400080E00895BC016F5E7F4FDC011696ED914C
:10085000FC91179785599F4F19950E94EB83811141
:100860000E94235680E0089585569F4F20E034E291
:1008700044E759E4FC0160817181828193810E9487
:100880000FD70E94DED40E940AD50E94D4B80E94DD
:10089000EB8381110E94235680E008958091F43FFC
:1008A0009091F53FFC0124853EEF320F323018F471
:1008B00024E024870895243011F080E090E008952A
:1008C000CF93DF93C091F43FD091F53F8C859EEF9D
:1008D000980F923018F484E08C8705C0843019F0AA
:1008E00080E090E010C02097D9F3DE011296ED91E0
:1008F000FC9113978785882329F0EC17FD0711F0E9
:10090000DF01F4CFCD01DF91CF910895CF93DF9335
:10091000EC012A813B81888199814CEBFB01DE014E
:1009200001900D924A95E1F72A833B83888399834E
:10093000DF91CF9108958FEE92E180930D599093BE
:100940000E598093CA599093CB5908952F923F9294
:100950004F925F926F927F928F929F92AF92BF92CF
:10096000CF92DF92EF92FF920F931F93CF93DF937B
:10097000CDB7DEB76A97CDBFDEBF4C011B012901A1
:100980003A01E986FA860B871C871A2D0B2DE8A8F9
:10099000B9A8AAA82BA9298380913635882399F074
:1009A00080912A3590912B35A0912C35B0912D3521
:1009B000BC01CD019F772CEA35EC47E257E30E945A
:1009C0006AD487FD11C78091613690916236A091FB
:1009D0006336B0916436BC01CD019F7731E03D8331
:1009E0002CEA35EC47E257E30E946DD6181614F056
:1009F0001D8210C02DEC3CEC4CEC5DE360910636A2
:100A00007091073680910836909109360E946AD419
:100A100087FDECC6F10180819181A281B381BC0187
:100A2000CD019F77F1E0FD872CEA35EC47E257E3F3
:100A30000E946DD618160CF01D86F10184819581F7
:100A4000A681B781BC01CD019F77F1E0F98B2CEA3B
:100A500035EC47E257E30E946DD618160CF0198A60
:100A6000F10180859185A285B3852091653630910D
:100A7000663640916736509168362E8B3F8B488F93
:100A8000598F2091693630916A3640916B3650917A
:100A90006C362A8B3B8B4C8B5D8B40916D36509125
:100AA0006E3660916F3670917036F0903735F11078
:100AB00021C01092555981E08093565982E080936D
:100AC00057593D81332341F04D85411195C65989D0
:100AD000511192C68CE9C1C6CB01BA019F772CEAAD
:100AE00035EC47E257E30E946DD618160CF089C624
:100AF0008BE9B3C6BC01CD019F77A1E0AA8F2CEA98
:100B000035EC47E257E30E946DD618160CF01A8EAA
:100B1000B1E0FB1216C01092555982E080935659ED
:100B2000F0925759ED81EE2339F0FD85F11164C63D
:100B30002A8D222379F260C66A897B898C899D89F6
:100B4000CDCF32E0F31217C081E080935559F09277
:100B50005659109257594D81442341F059895111EA
:100B60004BC68A8D882309F4B5CF46C66E897F8926
:100B7000888D998DB3CFB101C4010E94C34C9D8172
:100B8000992309F451C02091F2343091F33440910B
:100B9000F4345091F5346091473570914835809127
:100BA000493590914A350E94C1D29F772CEA35ECA5
:100BB00047E257E30E946AD487FF36C02091F6349B
:100BC0003091F7344091F8345091F93460914B35BD
:100BD00070914C3580914D3590914E350E94C1D227
:100BE0009F772CEA35EC47E257E30E946AD487FFEF
:100BF0001BC02091FA343091FB344091FC34509169
:100C0000FD3460914F357091503580915135909100
:100C100052350E94C1D29F772CEA35EC47E257E368
:100C20000E946AD487FDE4C58CA98093F1348DEECF
:100C300094E30E94CB4A86E5EDEEF4E3A4E7B9E540
:100C400001900D928A95E1F788E1E7E4F5E3A0E1F0
:100C5000B9E501900D928A95E1F7809138358111BF
:100C6000D5C523E333E34BEC51E46E2D7B2D8A2D68
:100C700099810E940FD74B015C016093405970939A
:100C80004159809342599093435923E333E34BEC0A
:100C900051E4C301B2010E940FD7609328597093A9
:100CA000295980932A5990932B5923E333E34BEC32
:100CB00051E469857A858B859C850E940FD7609366
:100CC0002C5970932D5980932E5990932F5923E3CB
:100CD00033E34BEC51E4612F702FC6010E940FD714
:100CE000162F072F412F502FBC014093305950939E
:100CF00031596093325970933359809102369091F3
:100D00000336A0910436B0910536BC01CD019F7722
:100D10000E9447D50E94DED4609351597093525976
:100D20008093535990935459A0915559A98BB091E0
:100D30005659BA8BEB2FF0E0ED83FE837F01EE0C6A
:100D4000FF1CEE0CFF1CF101EE0DFF1D8081918157
:100D5000A281B381BC01CD019F772CEA35EC47E23B
:100D600057E30E946AD4D82EDD1CDD24DD1C3989AE
:100D7000232F30E029833A838901000F111F000FD0
:100D8000111FF101E00FF11F80819181A281B381D8
:100D9000BC01CD019F772CEA35EC47E257E30E9476
:100DA0006AD4881F8827881F8D21809350592CEA88
:100DB00035EC47E257E3C501B4019F770E946DD639
:100DC00018160CF0F9C0F801EE50FB4CD801A95BE5
:100DD000BA4C2D913D914D915C91608171818281E0
:100DE00093810E94C1D26B017C01ED81FE81EE0FE7
:100DF000FF1FEE0FFF1FEE50FB4CAD81BE81AA0F0F
:100E0000BB1FAA0FBB1FA95BBA4C2D913D914D9101
:100E10005C9160817181828193810E94C1D26987D6
:100E20007A878B879C87A5019401C501B4010E9434
:100E30000FD720E030E040E850E40E940FD76D87E4
:100E40007E878F87988BA7019601C701B6010E9404
:100E50000FD72B013C0129853A854B855C85CA015A
:100E6000B9010E940FD79B01AC01C301B2010E94DE
:100E7000C2D29B01AC016D857E858F8598890E94C9
:100E8000C1D22B013C0120E030E0A9010E946DD6C7
:100E90001816C4F4C301B2010E94E8D72B013C012B
:100EA00029853A854B855C85C701B6010E947AD6B3
:100EB0009B01AC01C301B20190580E9471D42B0177
:100EC0003C0103C0412C512C32018091F13483301C
:100ED00021F477FA709477F8709420E030E0A9015B
:100EE000C501B4010E946AD487FF04C077FA7094E8
:100EF00077F8709409811A81000F111F000F111FDC
:100F0000A801435F564A5A01A301920169857A8577
:100F10008B859C850E940FD79B01AC01C701B60150
:100F20000E94C1D220E030E040E05FE30E940FD792
:100F3000D5015B966D937D938D939C935E97AD8069
:100F4000BE80AA0CBB1CAA0CBB1CF501E35FF64AD1
:100F50004F01A3019201C701B6010E940FD79B0167
:100F6000AC0169857A858B859C850E94C2D220E080
:100F700030E040E05FE30E940FD7D4015B966D93B1
:100F80007D938D939C935E97E0915759F0E0EE0F1F
:100F9000FF1FEE0FFF1FE35FF64A138E148E158EB0
:100FA000168EB0914059B987E0914159ED87209054
:100FB00042593090435925C05701F701E35FF64A83
:100FC000838D948DA58DB68D9C01AD015058F8018F
:100FD000E35FF64A838D948DA58DB68DBC01CD015E
:100FE00090580E947AD69B01AB01BC0140934059B6
:100FF00050934159609342597093435929873D87D3
:101000001C01D801A35FB64A5B96CD90DD90ED90B0
:10101000FC905E97E981FA81EE0FFF1FEE0FFF1F34
:10102000E758F64A13962D913D914D915C91169794
:1010300060817181828193810E94C1D2A701960152
:101040000E94C1D269837A838B839C83D501A35F7D
:10105000B64A5B964D905D906D907C905E97ED8169
:10106000FE81EE0FFF1FEE0FFF1FE758F64A1396A3
:101070002D913D914D915C91169760817181828196
:1010800093810E94C1D2A30192010E94C1D26D83BB
:101090007E838F8398879B01AC0169817A818B81E4
:1010A0009C810E947AD629853D85A1010E94C1D2EA
:1010B0004B015C01E894B7F820E030E040E85FE3E2
:1010C000C501B4010E946DD618160CF4C3C32AE002
:1010D00037ED43EA5BE3C501B4010E946DD61816F3
:1010E00094F42AE037ED43E25CE369857D85C10134
:1010F0000E940FD79B01AC01C501B4010E946DD6BF
:1011000018160CF4A7C3A30192015058C701B601E9
:1011100090580E9435D34B015C016093385970930D
:10112000395980933A5990933B59809137358130A2
:1011300039F4412C512C30E8632E3FEB732E06C05E
:10114000412C512C20E8622E2FE3722E80915059B1
:101150008823D1F16091515970915259809153591E
:10116000909154590E940AD56B017C012CEA35EC10
:1011700047E257E30E946AD487FD10C01091F13412
:101180002BED3FE049EC50E4C701B6010E940FD7B8
:101190009B01AC01C12CD12C7601B9C081E090E05B
:1011A000A0E0B0E08093515990935259A0935359C5
:1011B000B09354591091F1342BED3FE049EC50E4D9
:1011C000C12CD12C7601A3C02D813E814F81588541
:1011D00069817A818B819C810E9435D369837A836E
:1011E0008B839C8360933C5970933D5980933E5907
:1011F00090933F59A50194010E94C1D26B017C01DB
:101200009F772CEA35EC47E257E30E946AD487FFC8
:1012100018C01091F13460915159709152598091D8
:101220005359909154590E940AD52BED3FE049EC57
:1012300050E40E940FD79B01AC01C12CD12C760148
:1012400066C029813A814B815C81C501B4010E944D
:101250006DD61816F4F42BED3FE049EC50E4C301D1
:10126000B2010E940FD79B01AC0169817A818B8109
:101270009C810E94C2D260933C5970933D598093E7
:101280003E5990933F59A50194010E94C1D26B0130
:101290007C011091F134133099F0609151597091A3
:1012A000525980915359909154590E940AD52BED6F
:1012B0003FE049EC50E40E940FD79B01AC0127C0EE
:1012C0002BED3FE049EC50E4C301B2010E940FD77F
:1012D0009B01AC01C701B6010E94C1D27B018C0108
:1012E000609151597091525980915359909154592C
:1012F0000E940AD52BED3FE049EC50E40E940FD745
:101300009B01AC01C701D8016C017D010BC01230FB
:1013100049F4C301B2010E940FD7A70196010E94B0
:10132000C2D20AC0C301B2010E940FD79B01AC0117
:10133000C701B6010E94C1D27B01AB01BC01409341
:1013400044595093455960934659709347598C01BD
:1013500050905759A52DB0E0FD01EE0FFF1FEE0F85
:10136000FF1FE758F64AAA0FBB1FAA0FBB1FA35FB8
:10137000B64A13962D913D914D915C9116976081DF
:101380007181828193810E94C1D24B015C01609383
:1013900048597093495980934A5990934B599701F2
:1013A000A80169857D85C1010E940FD76B017C0171
:1013B00060934C5970934D5980934E5990934F5967
:1013C000A50194010E947AD669837A838B839C83DA
:1013D00060933459709335598093365990933759A7
:1013E00080913635811117C0F0912A35FD834090E8
:1013F0002B3520912C352E8B30912D353A8F109234
:101400002A3510922B3510922C3510922D3581E013
:101410008093363512C020912A3530912B3540917A
:101420002C3550912D3569817A818B819C810E9468
:1014300071D46D83472E8E8B9A8F598945E3549FC3
:10144000F0011124E158FC4C20813181428153810B
:10145000C701B6010E9471D4662E072F182F792E6E
:101460002D81342D4E895A8D0E946AD487FF04C085
:101470006D80042D1E897A8C9A8985E3989FF001EE
:101480001124E158FC4C2081318142815381C701F4
:10149000B6010E9471D46B017C019B01AC01662DE9
:1014A000702F812F972D0E946DD6181624F06C2C6A
:1014B0000D2D1E2D7F2C862D902FA12FB72D8093C3
:1014C000585990935959A0935A59B0935B5920E0B9
:1014D00030E0A901C501B4019F770E946DD61816AE
:1014E00084F5A5E35A9EF0011124E158FC4C2081BB
:1014F000318142815381C501B4010E9471D44B01F5
:101500005C01E894B7F8A5019401662D702F812F36
:10151000972D0E946DD6181614F4A72C04C0682CC1
:10152000092D1A2DAB2C862D902FA12FBA2D80932B
:10153000585990935959A0935A59B0935B59B62C66
:1015400002C0B62CA72CC090C032D090C132E0901F
:10155000C232F090C33220E030E040E850E4C701EE
:10156000B6010E940FD72B013C0129853D85A101C1
:1015700069857D85C1010E94C2D2A70196010E94A2
:10158000C1D29B01AC01C301B2010E940FD70E94DE
:10159000E8D72B013C0120EC31EE44E65CE46B2DF6
:1015A000702F812F9A2D0E940FD720E030E44CE15C
:1015B00056E40E9471D46B017C012091C9323091B4
:1015C000CA324091CB325091CC3269817A818B8181
:1015D0009C810E9471D44B015C01A301920169813D
:1015E0007A818B819C810E9471D487017601A5014B
:1015F00094010E94C1C10E9447D57B018C0120E06B
:1016000030E040E85FE30E946DD618163CF4B70165
:10161000C8010E94D9D44B015C0108C0812C912CD7
:1016200054018394E12CF12C00E81FE3C701D80199
:1016300080935C5990935D59A0935E59B0935F5924
:101640009701A801609158597091595980915A5940
:1016500090915B590E9471D46093A9597093AA59D3
:101660008093AB599093AC59809260599092615994
:10167000A0926259B09263599701A80160914459B0
:101680007091455980914659909147590E9471D463
:101690006093645970936559809366599093675924
:1016A0009701A801609148597091495980914A5910
:1016B00090914B590E9471D4609368597093695905
:1016C00080936A5990936B5980903859909039590A
:1016D000A0903A59B0903B59C501B4010E94DED7A1
:1016E000C0904059D0904159E0904259F0904359F0
:1016F0000091555910E0000F111F000F111F035FDB
:10170000164AA70196010E940FD79B01AC01F80170
:1017100063817481858196810E94C1D260936C59E6
:1017200070936D5980936E5990936F59C501B401B0
:101730000E946ED49B01AC010091565910E0000F3D
:10174000111F000F111F035F164AC701B6010E9447
:101750000FD79B01AC01D80113966D917D918D91AE
:101760009C9116970E94C1D26093705970937159E1
:101770008093725990937359A0915759B0E0FD012D
:10178000EE0FFF1FEE0FFF1FE758F64AAA0FBB1F11
:10179000AA0FBB1FA35FB64A13968D919D910D9022
:1017A000BC91A02D80839183A283B3831092B63F16
:1017B0008091345990913559A0913659B09137594B
:1017C000BC01CD019F772CEA35EC47E257E30E943C
:1017D0006AD487FD0FC00E94165682E080930F598D
:1017E0000E94264C80E039C08EE837C08EE935C0B3
:1017F0008FE933C089EC31C0B101C4010E94C34CF0
:10180000C2C9B101C4010E94C34C0ECA8E2D9B2DCA
:10181000AA2DB9818093405990934159A093425980
:10182000B0934359409228595092295960922A59AD
:1018300070922B5929853A854B855C8520932C59CC
:1018400030932D5940932E5950932F594C015D01DF
:10185000C60148CA8BE98093B63F6A96CDBFDEBF0A
:10186000DF91CF911F910F91FF90EF90DF90CF907C
:10187000BF90AF909F908F907F906F905F904F90B0
:101880003F902F9008958F929F92AF92BF92CF92E8
:10189000DF92EF92FF92CF93DF9380910F598823CD
:1018A00009F4B1C00E949382843010F482E0ACC08D
:1018B000209164593091655940916659509167590A
:1018C000609138597091395980913A5990913B59AA
:1018D0000E94C2D26B017C016093385970933959D0
:1018E00080933A5990933B590E94DED7809040599B
:1018F00090904159A0904259B0904359C091555988
:10190000D0E0CC0FDD1FCC0FDD1FC758D64AA50194
:1019100094010E940FD79B01AC0160916C597091AA
:101920006D5980916E5990916F590E94C2D268830F
:1019300079838A839B83C701B6010E946ED49B0181
:10194000AC01C0915659D0E0CC0FDD1FCC0FDD1F8C
:10195000C758D64AC501B4010E940FD79B01AC01FC
:101960006091705970917159809172599091735929
:101970000E94C2D2688379838A839B83C09157591E
:10198000D0E0CC0FDD1FCC0FDD1FC758D64A209109
:1019900068593091695940916A5950916B596881E1
:1019A00079818A819B810E94C2D2688379838A83EC
:1019B0009B8384E799E50E94259788E1E9E7F9E5AB
:1019C000A0E1B9E501900D928A95E1F78091605907
:1019D00090916159A0916259B09163590197A10901
:1019E000B1098093605990936159A0936259B09363
:1019F0006359181619061A061B060CF457CF1092D5
:101A00000F5980E001C083E0DF91CF91FF90EF900C
:101A1000DF90CF90BF90AF909F908F9008951092DD
:101A20000F5908954F925F926F927F928F929F927B
:101A3000AF92BF92CF92DF92EF92FF92CF93DF935C
:101A4000CDB7DEB76497CDBFDEBF69837A838B8362
:101A50009C8369017A0120E030E040E751E40E9474
:101A60000FD74B015C0120E030E040E751E4C701B3
:101A7000B6010E940FD79B01AC01C501B4010E94C1
:101A8000C1D26D877E878F87988B20E030E040E25F
:101A900051EC69817A818B819C810E940FD74B0127
:101AA0005C0120E030E040E251E4C701B6010E9451
:101AB0000FD79B01AC01C501B4010E94C2D2698B52
:101AC0007A8B8B8B9C8B20918D5830918E584091C6
:101AD0008F585091905860E070E080E89FE30E943A
:101AE00071D44B015C0120E030E040EC50EC6981A6
:101AF0007A818B819C810E940FD72B013C0120E0D1
:101B000030E040EC50E4C701B6010E940FD79B01C2
:101B1000AC01C301B2010E94C2D2A50194010E948E
:101B20000FD7A50194010E940FD7A50194010E942F
:101B30000FD7A50194010E940FD7A50194010E941F
:101B40000FD76B017C01A50194016D857E858F8582
:101B500098890E940FD7A50194010E940FD7A50173
:101B600094010E940FD7A50194010E940FD76D83A5
:101B70007E838F839887A501940169897A898B89EF
:101B80009C890E940FD7A50194010E940FD7A5013F
:101B900094010E940FD769877A878B879C8720E002
:101BA00030E042EF50E4C701B6010E940FD72B018D
:101BB0003C0120E030E040EA50E46D817E818F817D
:101BC00098850E940FD79B01AC01C301B2010E940E
:101BD000C2D22B013C0120E030E040E550E46985B1
:101BE0007A858B859C850E940FD79B01AC01C30130
:101BF000B2010E94C2D26093B1587093B2588093E0
:101C0000B3589093B45820E030E045EA52E4C7015D
